:10000000008000103D470000914700009947000024
:10001000A1470000A9470000B14700000000000010
:10002000000000000000000000000000B9470000D0
:10003000C147000000000000C9470000D147000090
:10004000D94700000179030089790300A17B0300EF
:10005000C97B0300CD8E0300D18F0300D590030030
:10006000D9910300D9470000D9470000D9470000C3
:10007000D9470000D9470000D9470000D947000000
:10008000D9470000D9470000D94700005D4800006B
:10009000D9470000D9470000D9470000D9470000E0
:1000A000D9470000D9470000D9470000D9470000D0
:1000B000D9470000D9470000D9470000D9470000C0
:1000C000D9470000D9470000D947000010D40500E7
:1000D000000000102800000010D4050000C0072018
:1000E0000000000028000010BC63000000C00720D2
:1000F0000000000080B485B000AF0346FB710B46E2
:10010000BB7113467B71FB791A04BB791B021A433E
:100110007B79134343F08063FB6018461437BD4678
:100120005DF8047B704700BF80B582B000AF034626
:10013000FB710A4A094BDB6943F40013D361FB7975
:10014000184636F0FDFE002036F0FAFE002036F0AC
:10015000F7FE00F0C9FA0837BD4680BD20C009206F
:1001600080B582B000AF78600B46FB70114A114B2E
:10017000DB6943F40013D3617B681B0CDBB263F0D3
:100180007F03DBB2184636F0DBFE7B681B0ADBB26E
:10019000184636F0D5FE7B68DBB2184636F0D0FE46
:1001A000FB78184636F0CCFE00F09EFA0837BD46C4
:1001B00080BD00BF20C0092080B582B000AF78604C
:1001C0000B467B80154A154BDB6943F40013D36162
:1001D0007B681B0CDBB263F07F03DBB2184636F0A2
:1001E000AFFE7B681B0ADBB2184636F0A9FE7B68BF
:1001F000DBB2184636F0A4FE7B88DBB2184636F038
:100200009FFE7B881B0A9BB2DBB2184636F098FE35
:1002100000F06AFA0837BD4680BD00BF20C0092043
:1002200080B582B000AF786039601B4A1A4BDB6939
:1002300043F40013D3617B681B0CDBB263F07F03D4
:10024000DBB2184636F07CFE7B681B0ADBB2184630
:1002500036F076FE7B68DBB2184636F071FE3B68FE
:10026000DBB2184636F06CFE3B689BB21B0ADBB271
:10027000184636F065FE3B681B0CDBB2184636F0BC
:100280005FFE3B681B0EDBB2184636F059FE00F0ED
:100290002BFA0837BD4680BD20C0092080B584B048
:1002A00000AF78603960224A214BDB6943F40013C8
:1002B000D3617B681B0CDBB263F07F03DBB21846B3
:1002C00036F03EFE7B681B0ADBB2184636F038FE7D
:1002D0007B68DBB2184636F033FE386839F070FCC4
:1002E0000346BB730023FB730AE0FB7B3A681344AD
:1002F0001B78DBB2184636F023FEFB7B0133FB7321
:10030000FA7BBB7B9A42F0D905E0002036F018FE5C
:10031000FB7B0133FB73FB7B03F00303DBB2002B9E
:10032000F3D100F0E1F9FB7B18461037BD4680BDE4
:1003300020C0092080B582B000AF7860124A124B0D
:10034000DB6943F40013D3617B681B0CDBB21846F6
:1003500036F0F6FD7B681B0ADBB2184636F0F0FD7E
:100360007B68DBB2184636F0EBFD002036F0E8FD86
:10037000002036F0E5FD00F0B7F9044B1B78184675
:100380000837BD4680BD00BF20C0092024020010F0
:1003900080B584B000AF7860184A184BDB6943F42D
:1003A0000013D3617B681B0CDBB2184636F0C8FD26
:1003B0007B681B0ADBB2184636F0C2FD7B68DBB2F5
:1003C000184636F0BDFD002036F0BAFD002036F0AC
:1003D000B7FD0B4B1B78FB73002036F0B1FD00F02E
:1003E00083F9074B1B781B029AB2FB7B9BB213432A
:1003F0009BB29BB218461037BD4680BD20C0092075
:100400002402001080B584B000AF78601F4A1F4BF3
:10041000DB6943F40013D3617B681B0CDBB2184625
:1004200036F08EFD7B681B0ADBB2184636F088FD7D
:100430007B68DBB2184636F083FD002036F080FD85
:10044000002036F07DFD124B1B78FB60002036F05B
:1004500077FD0F4B1B781B02FA681343FB600020EB
:1004600036F06EFD0A4B1B781B04FA681343FB60E1
:10047000002036F065FD00F037F9054B1B781A06B1
:10048000FB68134318461037BD4680BD20C00920C5
:100490002402001080B483B000AF0346FB71FA79E8
:1004A000054B1B681344C3F30B03034A13600C375B
:1004B000BD465DF8047B70472800001080B582B00F
:1004C00000AF7860064B1B6803F584131846796803
:1004D000FFF7A6FE0420FFF7DDFF0837BD4680BD0D
:1004E0002800001080B500AF5B4A5B4BDB6943F42A
:1004F0008003D36159480FF053FF574A564B9B690D
:1005000043F48003936155480FF04AFF0020FFF742
:100510000BFE4420FFF708FE6220FFF705FE50485F
:100520004FF4F071FFF748FE4E484FF48871FFF723
:1005300043FE4D484FF40971FFF73EFE4B48002142
:10054000FFF73AFE4A482921FFF736FE49482B219A
:10055000FFF732FE48484FF49271FFF72DFE4748EF
:100560000021FFF729FE46480A21FFF725FE4548EE
:100570000C21FFF721FE44480021FFF7F1FD43481D
:100580000021FFF7EDFD42484FF4DB71FFF714FE49
:1005900040480021FFF7E4FD3F480121FFF7E0FD5F
:1005A0003E483F49FFF73CFE3E480121FFF7D8FD9A
:1005B0003D484FF49661FFF733FE4FF480103B49FE
:1005C000FFF72EFE3A483B49FFF72AFE3A48002142
:1005D000FFF726FE39480221FFF7C2FD3848FC210B
:1005E000FFF7BEFD3748FF21FFF7BAFD364805216A
:1005F000FFF7B6FD35480FF0D3FE4FF47A7034495B
:10060000942200F0C1FA40F27C4032494BF27C5215
:1006100000F0BAFA6FF0FF00FFF750FF2548FFF730
:100620004DFF2D48FFF74AFF2C48FFF747FF2C48A6
:10063000FFF744FF2B48FFF741FF6FF0D400FFF7AF
:100640003DFF0820FFF73AFF4FF47A70FFF736FFBF
:1006500027F04AFC80BD00BF20C00920C0C62D0085
:1006600030241000442410002824100034241000EA
:10067000382410002C2410003C24100048241000C2
:100680004C24100040241000642410005C2410004E
:100690005824100060241000682410000C2410005E
:1006A000006CDC025424100004251000FF0000023E
:1006B000040010000700002608001000502410005D
:1006C0008C241000902410006C241000E09304008F
:1006D0009CB0030030B1030008000005B002000127
:1006E000172818071728000880B400AF00BF084B70
:1006F000DB6803F00103002BF9D0064A054B9B6928
:1007000043F400139361BD465DF8047B704700BF5E
:100710000080084020C0092090B583B000AF044697
:10072000084611461A462346FB800346BB800B460B
:100730007B8013463B806FF0D300FFF7BFFE1F4B5B
:100740001B6803F58412FB8810461946FFF734FD39
:100750000220FFF79FFE194B1B6803F58412BB882C
:1007600010461946FFF728FD0220FFF793FE134BB2
:100770001B6803F584127B8810461946FFF71CFDA1
:100780000220FFF787FE0D4B1B6803F584123B88A0
:1007900010461946FFF710FD0220FFF77BFE074BBE
:1007A0001B6803F584123B8B10461946FFF704FDC6
:1007B0000420FFF76FFE0C37BD4690BD28000010E7
:1007C00090B583B000AF0446084611461A4623464A
:1007D000FB800346BB800B467B8013463B806FF05B
:1007E000EF00FFF76BFE2B4B1B6803F58412FB88B1
:1007F00010461946FFF7E0FC0220FFF74BFE254BA1
:100800001B6803F58412BB8810461946FFF7D4FC19
:100810000220FFF73FFE1F4B1B6803F584127B8805
:1008200010461946FFF7C8FC0220FFF733FE194BAC
:100830001B6803F584123B8810461946FFF7BCFC81
:100840000220FFF727FE134B1B6803F584123B8B36
:1008500010461946FFF7B0FC0220FFF71BFE0D4BB8
:100860001B6803F58412BB8B10461946FFF7A4FCE6
:100870000220FFF70FFE074B1B6803F584123B8C29
:1008800010461946FFF798FC0420FFF703FE0C37CB
:10089000BD4690BD2800001090B583B000AF04465F
:1008A000084611461A462346FB800346BB800B468A
:1008B0007B8013463B806FF0F300FFF7FFFD1F4B7B
:1008C0001B6803F58412FB8810461946FFF774FC79
:1008D0000220FFF7DFFD194B1B6803F58412BB886C
:1008E00010461946FFF768FC0220FFF7D3FD134BB3
:1008F0001B6803F584127B8810461946FFF75CFCE1
:100900000220FFF7C7FD0D4B1B6803F584123B88DF
:1009100010461946FFF750FC0220FFF7BBFD074BBE
:100920001B6803F584131846B969FFF7B7FC034643
:100930001846FFF7AFFD0C37BD4690BD28000010EC
:1009400090B583B000AF0446084611461A462346C8
:10095000FB800346BB800B467B8013463B806FF0D9
:10096000F200FFF7ABFD2B4B1B6803F58412FB88ED
:1009700010461946FFF720FC0220FFF78BFD254BA0
:100980001B6803F58412BB8810461946FFF714FC58
:100990000220FFF77FFD1F4B1B6803F584127B8845
:1009A00010461946FFF708FC0220FFF773FD194BAC
:1009B0001B6803F584123B8810461946FFF7FCFBC1
:1009C0000220FFF767FD134B1B6803F584123B8B76
:1009D00010461946FFF7F0FB0220FFF75BFD0D4BB9
:1009E0001B6803F58412BB8B10461946FFF7E4FB26
:1009F0000220FFF74FFD074B1B6803F584131846D1
:100A0000396AFFF74BFC03461846FFF743FD0C37E6
:100A1000BD4690BD2800001090B583B000AF0446DD
:100A2000084611461A462346FB800346BB800B4608
:100A30007B8013463B806FF0D100FFF73FFD1B4BDF
:100A40001B6803F58412FB8810461946FFF7B4FBB8
:100A50000220FFF71FFD154B1B6803F58412BB88AE
:100A600010461946FFF7A8FB0220FFF713FD0F4BB6
:100A70001B6803F584127B8810461946FFF79CFB20
:100A80000220FFF707FD094B1B6803F584123B8822
:100A900010461946FFF790FB0220FFF7FBFCBB69ED
:100AA0001846FFF70BFD0C37BD4690BD280000101F
:100AB00090B583B000AF0446084611461A46234657
:100AC000FB800346BB800B467B8013463B806FF068
:100AD000ED00FFF7F3FC2B4B1B6803F58412FB883A
:100AE00010461946FFF768FB0220FFF7D3FC254BA1
:100AF0001B6803F58412BB8810461946FFF75CFBA0
:100B00000220FFF7C7FC1F4B1B6803F584127B888C
:100B100010461946FFF750FB0220FFF7BBFC194BAC
:100B20001B6803F584123B8810461946FFF744FB07
:100B30000220FFF7AFFC134B1B6803F584123B8BBD
:100B400010461946FFF738FB0220FFF7A3FC0D4BB8
:100B50001B6803F58412BB8B10461946FFF72CFB6C
:100B60000220FFF797FC074B1B6803F58413184618
:100B7000396AFFF793FB03461846FFF78BFC0C37E7
:100B8000BD4690BD2800001080B584B000AFF8606D
:100B9000B9607A60164A164BDB6943F40013D361DF
:100BA000FB681B0CDBB263F07F03DBB2184636F048
:100BB000C7F9FB681B0ADBB2184636F0C1F9FB68BF
:100BC000DBB2184636F0BCF908E0BB681B78DBB234
:100BD000184636F0B5F9BB680133BB607B685A1E16
:100BE0007A60002BF1D1FFF77FFD1037BD4680BD45
:100BF00020C00920B0B58CB000AF78604E4BBB620E
:100C00004D4B7B624D4B0022DA707B6840F6D86218
:100C1000934204DD4A4BFB62484B0122DA707B6849
:100C2000B3F5FA7F04DA474BFB62444B0222DA70D9
:100C3000424BDB78002B76D178683AF003F9044612
:100C40004FF08B40B96A39F099FF034620461946A8
:100C500039F094FF03463B62386A3B4939F030FF74
:100C600003461C46786A396A39F0E8FF0346204695
:100C7000194639F083FF03463B62344BFB61344B2A
:100C8000BB61344B7B61344B3B61386A334939F08B
:100C900075FF0346FB60F869396939F0CFFF0346F9
:100CA0001C463869F96839F00BFF0346204619469F
:100CB0003AF042F8034618463AF0D8F802460B4696
:100CC0001046194638F0B0FE04460D46B8693AF0B1
:100CD000CDF802460B462046294639F0D3FB0246A2
:100CE0000B4614461D467B69184619463AF024F80F
:100CF000034618463AF0BAF802460B462046294603
:100D000039F00AFB02460B46104619464FF0000226
:100D1000134B39F0CBFC02460B461046194639F00E
:100D200081FD0346FB62F86A0E4939F0C9FE0346AD
:100D300018463037BD46B0BD33335340A0270010AE
:100D400000009643000096C300C02845AD388238A5
:100D50001E1B013CC27CA237C27CA2380000FA44B0
:100D6000000039400000C84290B587B000AF7860FD
:100D7000374B3B61364BFB60364B0022DA707B68A9
:100D800040F63C72934204DD334B7B61314B0122D0
:100D9000DA707B68B3F5FA7F04DA304B7B612D4B58
:100DA0000222DA702B4BDB78002B39D178683AF0CD
:100DB00049F804464FF08B40396939F0DFFE0346AD
:100DC0002046194639F0DAFE0346BB60B86824496C
:100DD00039F076FE03461C46F868B96839F02EFFF4
:100DE00003462046194639F0C9FE0346BB60B86881
:100DF0001C4939F023FF034618463AF037F80246FB
:100E00000B461046194610A3D3E9002339F084FAA3
:100E100002460B461046194639F004FD03467B6135
:100E200078690D493AF072F80346002B01D00A4B5D
:100E30007B6178690C4939F043FE034618461C373C
:100E4000BD4690BDAFF30080CDCCCCCCCCCC0E4019
:100E500033335340A02700100000A043000096C386
:100E600000C0284500007A440000C842AFF300806B
:100E700090B589B000AF0023FB7703F0B7FB0346C2
:100E80001A46744B83F86120734B93F80D33012B92
:100E90001CD1704B9B78062B0FD06E4B9B78072B89
:100EA00003D06C4B9A786D4B1A706D4BDB78002B2E
:100EB00013D1684B06229A700FE0694BDB78012B47
:100EC0000BD1664B1A78634B9A7006E0614B9B78A6
:100ED000062B02D15F4B00229A705E4B9B78062B4B
:100EE00019D05C4B9B78072B0CD05A4B9A785B4BF4
:100EF0001A70584B93F86030012B0CD1554B0722D8
:100F00009A7008E0534B93F86030002B03D1534B99
:100F10001A78504B9A70534B1B680133514A136037
:100F2000504B1B68B3F5616F20DB4E4B00221A60FB
:100F30000023FB770EE0FA7FFB7F01334A495B0019
:100F40000B449888484953000B4402469A80FB7F23
:100F50000133FB77FB7F162BEDD9434BDA8E424BE7
:100F60005A86414B0022DA8603F012FE0023BB6151
:100F70000023FB770BE0FB7F3B4A5B0013449B881D
:100F80001BB2BA691344BB61FB7F0133FB77FB7F64
:100F9000172BF0D9304BD3F81C321846334939F0AF
:100FA000EDFD0346FB60B86939F058FF034618466B
:100FB000F96839F085FD03461A46264B1A612C4B19
:100FC0001B68002B04D02A4B1B68013B284A136086
:100FD000204B9A78204B83F81722264BDB7E002B80
:100FE00052D1244B5B899AB2224B9B899BB2D31A74
:100FF0009BB29AB2174BA3F840201F4B1B685A1C98
:101000001D490A600A2B13DD1C4B1B881AB2194BB1
:101010009B891BB2D31A184639F014FF0246184BAD
:101020001A60144B9A89154B1A80134B00221A60D0
:10103000134B1B68074A5364064B5B6C18461149F7
:1010400039F064FF0346002B00D129E0014B0D4A23
:101050005A6425E020270010040700102C0000101F
:1010600098270010300000101C1E00100000614581
:1010700000000010C42100103400001038000010DF
:101080003C0000100000FA433D4B4FF000021A6094
:101090003C4B4FF000025A643A4B0022A3F8402028
:1010A000384B9B78042B19D10FF0C6FE364B00222B
:1010B0005A72354B00221A72344A344BDB6943F4BE
:1010C0000023D3612F4B00229A802E4B0022DA801E
:1010D0002C4B00221A812E4B00221A80294B9B7820
:1010E000062B16D1274B00229A80264B00221A810C
:1010F000244B0022DA80274B00225A60224B002228
:10110000DA71254B1B680133234A1360234B0022FD
:101110001A601C4B9B78072B16D11A4B00229A8021
:10112000184B00221A81174B0022DA80194B00223B
:101130005A60154B0022DA71174B1B680133164AAF
:101140001360164B00221A600E4B9B78002B27D1A0
:101150000C4B00229A800B4B00221A81094B002273
:10116000DA800C4B00225A60074B0022DA710A4BDE
:101170001B680133084A1360084B00221A6012E012
:101180003C00001020270010300A001000C0092089
:10119000F421001040220010280A00104000001026
:1011A000844B00225A71844B9B78012B58D1814B80
:1011B00000229A71804B00229A807F4B0022DA80B5
:1011C0007E4B93F820321A467D4B5A607A4B1B8F28
:1011D000002B45D07B4B0122DA71774B1B8F013BF3
:1011E0009AB2754B1A87744B1B8F002B38D1754BF5
:1011F0000022DA71704BDC68704BB3F84632184647
:1012000039F02CFE034618466F4939F059FC034665
:101210001846F96839F054FC03462046194639F05F
:101220008BFD03461A46644BDA60684B9C6B634B3C
:10123000B3F84632184639F011FE034618466249A3
:1012400039F03EFC03461846F96839F039FC03468C
:101250002046194639F0F2FC03461A465B4B9A6366
:10126000554B9B78032B5CD1534B00229A80524BF9
:101270000022DA80504B00221A81514B00225A6022
:101280004D4B9B8F002B4CD04E4B0122DA714A4BB9
:101290009B8F013B9AB2484B9A87474B9B8F002B01
:1012A0003FD1484B0022DA71434B00229A70424BE7
:1012B000DC68424BB3F84432184639F0CFFD0346A0
:1012C0001846414939F0FCFB03461846F96839F0E5
:1012D000F7FB03462046194639F02EFD03461A4611
:1012E000354BDA60394B9C6B344BB3F844321846BB
:1012F00039F0B4FD03461846334939F0E1FB0346A3
:101300001846F96839F0DCFB03462046194639F0E7
:1013100095FC03461A462D4B9A6303F061FB03F0DC
:1013200037FC254B9B78052B40F06D81224B00222A
:101330001A81214B0022DA801F4B00229A80244B15
:101340005A891D4B1B8812B21BB29A4262DA1B4BA0
:1013500093F84A32012B45D11D4B1B7E002B41D106
:10136000164B93F81632072B3CD1194B5A68134B86
:10137000B3F84C32643B9A421BDA0E4B00229A7649
:101380000D4B08229A70134B00221A800B4BB3F8B6
:101390002E22114B1A80114B00221A80074BB3F8F2
:1013A00034321A461201D31A9B009AB20C4B1A809F
:1013B00030E02FE0A02700102027001004070010C5
:1013C00040220010300A0010000070421C1E001065
:1013D000C42100108827001044000010F81D0010E0
:1013E000F4060010774B08229A70774B00221A807F
:1013F000764BB3F82E22764B1A80764B00221A8059
:10140000724BB3F834321A461201D31A9B009AB2C7
:10141000714B1A806D4B93F81632082B3AD16F4BF3
:101420001B6801336D4A13606C4B1B683C2B31DD2C
:101430006B4B1A686B4B5B891BB2D31A6A4A1360F9
:10144000694B1B68312B1DDD664B5A895F4BB3F826
:10145000BC3112B21BB29A4214DA624B5B891AB2E7
:10146000584B1B881BB203F5FA739A420ADA574BA2
:10147000B3F840320E2B05D9524B08229A70524BCA
:1014800000221A80574B5B891BB2554A1360534B9D
:1014900000221A60504B1B88002B20D0534B002297
:1014A000DA71534B00225A604B4B1B88013B9AB2B6
:1014B000494B1A80484B1B88002B10D1434BB3F883
:1014C00032224C4B1A80414B93F838329AB2414B3E
:1014D0001A80494B1B8801339AB2474B1A80454BFF
:1014E0001B88002B1CD0394BB3F836321A46404BC0
:1014F0005A60404B1B88013B9AB23E4B1A803D4BD1
:101500001B88002B0CD1314BB3F834321A46120130
:10151000D31A9B009AB2304B1A80354B00225A6086
:101520002A4B93F81332012B6AD12A4B1B88002BCC
:1015300069D02E4B0122DA71264B1B88013B9AB2EF
:10154000244B1A80234B1B88002B5CD1274B002295
:10155000DA711C4BDC681D4B93F83832184639F0B1
:101560007DFC03461846F96839F0AAFA034620467E
:10157000194639F0E1FB03461A46124BDA601F4B5D
:10158000DB8E9AB2114B93F838329BB213449BB264
:101590009AB21A4BDA86194B9C6B0C4B93F8383283
:1015A000184639F05BFC03461846F96839F088FAAA
:1015B00003462046194639F041FB03461A460F4BB5
:1015C0009A6320E0202700108827001004070010ED
:1015D00044000010F81D0010F40600104800001030
:1015E0004C000010C421001050000010300A001000
:1015F00040220010601E0010540000101C1E00103D
:10160000274B0022DA71274B9B78082B38D1254BCA
:1016100000221A81234B0022DA80224B00229A807A
:10162000214B00229A76214BB3F836321A46204BD2
:101630005A601B4B0022DA711E4B1B889BB29BB277
:1016400001339BB29AB21B4B1A80184BB3F83A2263
:10165000184B1B8812B21BB29A4211DC114B0222AA
:101660009A70124BB3F82E22134B1A800F4BB3F81B
:1016700034321A461201D31A9B009AB20F4B1A80C9
:10168000084B9B78022B40F04B82054BDB79002BFB
:1016900018D10B4B1B8801339AB2094B1A8014E006
:1016A000300A001020270010A027001004070010A7
:1016B000402200108827001044000010F40600109B
:1016C00038220010814B00221A80814B1B680133A5
:1016D0007F4A13607F4B93F81632082B02D100200B
:1016E00000F0BAFA7B4B93F81632072B40F03981A1
:1016F000784BB3F830321A46774B5A60754B93F8F3
:101700001332012B40F0FA80744B1B88002B08D158
:10171000734B1B88002B04D16E4BB3F82E226F4BFA
:101720001A80704B1B7F002B22D06F4BDB79002B74
:101730001ED16D4B0122DA71664BB3F82C320133A6
:101740009AB2674B1A80694BDB8E9AB2614BB3F841
:101750002C3213449BB29AB2644BDA86614B1B7FE6
:10176000002B05D05F4B1B7F013BDAB25D4B1A7734
:101770005A4B1B88002B1ED0584B1B88013B9AB23A
:10178000564B1A80554B1B88002B14D1564B012207
:10179000DA71504BB3F82C3201339AB2504B1A80A5
:1017A000524BDB8E9AB24B4BB3F82C3213449BB2A4
:1017B0009AB24E4BDA864A4B1B88002B3DD0484BE1
:1017C0001B88013B9AB2464B1A80454B1B88002B65
:1017D00033D1454B0022DA713E4BB3F82E223F4BFA
:1017E0001A80434BDC683B4BB3F82C32184639F077
:1017F00035FB03461846F96839F062F9034620467E
:10180000194639F099FA03461A46394BDA60374BD4
:101810009C6B304BB3F82C32184639F01FFB034653
:101820001846F96839F04CF903462046194639F054
:1018300005FA03461A462D4B9A63264BB3F82E320F
:10184000002B02D1284B0122DA71224BB3F82E2251
:10185000204BB3F82C3213447B817B894FF46162B7
:1018600092FBF3F33B811B4BB3F82C323A8902FB1A
:1018700003F3FB80FB88184639F0F0FA0446F86859
:101880001C4939F01DF903462046194639F018F96C
:101890000346184639F0C2FA03469AB2144BDA806E
:1018A000134BDB881A460B4BB3F8143203FB02F3DD
:1018B000114A82FB03129210DB17D31A9AB20C4B17
:1018C0009A800B4B64221A811BE000BF3822001063
:1018D000280A0010040700104022001044000010E5
:1018E00056000010A0270010300A00101C1E001027
:1018F000202700100000C842676666666B4B002216
:10190000DA716B4B00229A766A4B93F84A32012BBC
:1019100027D1694B1B7E002B23D1674B5A68654B3F
:10192000B3F84C3264339A421BDD614B01229A7644
:10193000624B05229A705F4BB3F834321A4612019B
:10194000D31A9B009AB25E4B1A805E4B00221A801B
:101950005D4B00221A80554B0022DA715B4B00224E
:101960001A600023FB82534B93F81632082B01D1E7
:101970003223FB824F4B93F81632072B03D14D4B8A
:10198000B3F8BA31FB824C4B5B891AB24B4B1B88C4
:1019900019B2B7F916300B449A4205DD4C4B1B685F
:1019A00001334B4A136002E0494B00221A600023C6
:1019B000BB82404B93F81632082B09D13D4BB3F84C
:1019C00040321A461201D31A9B00BB820F23FB74CC
:1019D000384B93F81632072B0FD10523BB82354BBA
:1019E000B3F82E32002B02D10523FB7405E0314BF6
:1019F000B3F82E32DBB2023BFB74BA8A344B1B685D
:101A00009A4208D32C4B5A892A4BB3F8BC3112B2F4
:101A10001BB29A423DDDFB7C9AB22E4B1B889A4248
:101A200010D9254B5A89234BB3F8BC3112B21BB2E3
:101A30009A4207DCBA8AFB7C13441A46244B1B6883
:101A40009A4226D21B4B93F81632082B02D1012062
:101A500000F002F9194B05229A70164BB3F8343294
:101A60001A461201D31A9B009AB2154B1A80154BD5
:101A700000221A80144B00221A80144B00221A6094
:101A8000154B00225A60094B0022DA71104B0022DC
:101A90001A60022001F04CFE0346002B20D10F4BB0
:101AA0001B6801330D4A13601DE000BF300A0010AF
:101AB000A027001004070010C421001020270010E8
:101AC000F4060010601E0010F81D0010280A001017
:101AD0005800001038220010402200104000001072
:101AE000504B00221A60504BB3F850321A4613463E
:101AF0001B019B1A9B001A464A4B1B689A420FD245
:101B00004A4B01221A734A4B00229A70494B002219
:101B10001A60444B00221A60052000210BF03EFCA5
:101B2000434BDB68444A1360444B1B680133434A10
:101B30001360424B1B683B2B16D93D4BDB681846A4
:101B400039F06CF902463E4B1B689A4201D003F013
:101B50001FF83A4B00221A60354BDB68184639F003
:101B60005DF90246364B1A60314B9B78022B03D04D
:101B70002F4B9B78052B4AD12B4B93F80E33002B20
:101B800045D0304B1B6801332E4A1360264B93F827
:101B90000E331A4613461B019B1A9B001A46294B0B
:101BA0001B689A420BD2284B93F82830002B06D1A1
:101BB000254B012283F82820244B00221A70224B47
:101BC00093F82830012B21D1204B1B780133DAB256
:101BD0001E4B1A701E4B5B891AB2154B1B881BB229
:101BE00003F5FA739A4202DA1A4B64225A600E4BDA
:101BF00093F80F23154B1B789A4207D2114B002202
:101C00001A60114B002283F8282007E006E00D4BF4
:101C100000221A600C4B002283F828202437BD468E
:101C200090BD00BF4000001004070010140A00100F
:101C300020270010280A00101C1E00105C00001055
:101C4000600000103C220010A02700101C2700108C
:101C5000C421001040220010B0B58EB000AF034682
:101C6000FB71A34B93F83D329BB2C3F164039BB26B
:101C7000FB856423BB854FF00003BB624FF000037C
:101C80007B624FF000033B624FF000037B634FF039
:101C900000033B63964BB3F81832184639F0DEF870
:101CA0000346FB61934B1B78002B03D0924B5A8960
:101CB000924B1A808E4B93F84232012B10D18C4BF1
:101CC0008F4AC3F85C228A4B8E4AC3F86022884B45
:101CD0004FF08142C3F86422854B8B4AC3F86822D7
:101CE000834B93F84232022B11D1814B844AC3F8C3
:101CF0005C227F4B4FF08242C3F860227C4B814ACA
:101D0000C3F864227A4B4FF08342C3F86822784BC1
:101D100093F84232032B10D1754B794AC3F85C22F9
:101D2000734B7A4AC3F86022714B4FF08242C3F87A
:101D300064226F4B764AC3F868226D4B93F84232A7
:101D4000042B0FD16A4B6E4AC3F85C22684B714A70
:101D5000C3F86022664B6D4AC3F86422644B684A3C
:101D6000C3F86822624B93F84232052B0FD1604BC7
:101D7000634AC3F85C225E4B634AC3F860225C4B43
:101D8000644AC3F864225A4B634AC3F86822584B2A
:101D900093F84232062B10D1554B594AC3F85C22B6
:101DA000534B4FF08342C3F86022514B564AC3F85D
:101DB00064224F4B594AC3F868224D4B93F8423284
:101DC000072B10D14A4B4E4AC3F85C22484B504A6D
:101DD000C3F86022464B4FF08342C3F86422444B61
:101DE0004F4AC3F868224F4B1B6801334D4A1360BA
:101DF0004C4B1B68184639F025F802463C4BD3F88B
:101E00005C321046194639F0BFF80346002B00F04B
:101E1000AE83444B00221A60434B1B881AB2364BE8
:101E20005B891BB2D31A184639F00CF803463B62A3
:101E3000314B5B891AB2314B1B881BB202339A4279
:101E400002DD394B01229A642B4B5B891AB22B4B72
:101E50001B881BB2023B9A4203DA334B4FF0FF322E
:101E60009A64254B5B891AB2244B1B881BB2D31A88
:101E7000184637F075FE0346022B02DC2A4B00227F
:101E80009A641D4B5A68294B1B881BB21E339A4219
:101E900002DD254B0122DA64174B5A68234B1B885D
:101EA0001BB21E3B9A4203DA1F4B4FF0FF32DA643B
:101EB000114B5A681D4B1B881BB2D31A184637F0BA
:101EC0004FFE03461E2B02DC174B0022DA640A4B3E
:101ED0001B7E002B02D0144B0022DA64044B93F8D3
:101EE0004A32002B24D1104B0022DA6420E000BFDC
:101EF0000407001004000010C42100106E00001040
:101F00000000A0410000C0400000604100002041EE
:101F100000009041000040410000B0410000C0417D
:101F20000000D04170000010202700107400001045
:101F3000386A38F09BFF02460B461046194637F0C8
:101F4000F1FB02460B46104619464FF00002AE4B1D
:101F500038F0E2F902460B4614461D46AB4BD3F867
:101F600060321846AA4938F009FE0346184638F090
:101F70007DFF02460B462046294638F037F90246D7
:101F80000B461046194638F04DFC0246A14B1A602C
:101F9000386A38F06BFF02460B461046194637F098
:101FA000C1FB02460B46104619464FF00002964B05
:101FB00038F0B2F902460B4614461D46934BD3F84F
:101FC00064321846924938F0D9FD0346184638F075
:101FD0004DFF02460B462046294638F007F90246D7
:101FE0000B461046194638F01DFC02468A4B1A6013
:101FF000884B1B681846894938F088FF0346002B38
:1020000002D0844B854A1A60834B1B68184683496B
:1020100038F07CFF0346002B02D07F4B7F4A1A60CA
:102020007C4B1B68184638F021FF02460B461046D1
:10203000194673A3D3E9002338F090FC0346002B24
:1020400002D0744B764A1A60734B1B68184638F0FE
:102050000DFF02460B461046194669A3D3E900233B
:1020600038F07CFC0346002B02D06B4B6C4A1A60A4
:10207000684B1B686B4A5361674B1B68694A9361E5
:10208000386A4FF0804138F041FF0346002B00F0E2
:10209000D180644B9B6C012B45D1386A38F0E6FE49
:1020A00002460B461046194637F03CFB02460B46EB
:1020B000104619464FF000025B4B38F04FFC0346C8
:1020C000002B0BD0594B1A68534B1B68104619460E
:1020D00038F0B4FD03461A46544B1A60386A38F09B
:1020E000C5FE02460B461046194637F01BFB02465A
:1020F0000B46104619464FF00002434B38F02EFCB9
:102100000346002B0FD0474BDB6C012B0BD1474B09
:102110001A68414B1B681046194638F08FFD03467C
:102120001A46424B1A603F4B9B6C002B44D13D4BEF
:10213000DB6C012B1BD0354B93F83E32184638F040
:1021400081FE02463A4B1B681046194638F0DEFE07
:102150000346002B0BD0354B1A682E4B1B681046DC
:10216000194638F0E9FD03461A46304B1A60386AC2
:1021700038F07CFE02460B461046194637F0D2FA7C
:1021800002460B46104619464FF00002264B38F027
:10219000E5FB0346002B0FD0224BDB6C012B0BD150
:1021A000224B1A681C4B1B681046194638F046FD36
:1021B00003461A461D4B1A601A4B9B6CB3F1FF3F46
:1021C00038D1124B93F83E32184638F03BFE0246A7
:1021D000174B1B681046194638F098FE0346002B33
:1021E00028D0124B1A680B4B1B681046194638F062
:1021F000A3FD03461A460D4B1A601BE0AFF30080A7
:102200009A9999999999B93F00006940040700107B
:1022100000002041780000107C00001000004040C9
:10222000CDCCCC3D202700100000344080000010B1
:1022300084000010386A4FF0404138F049FE0346F0
:10224000002B00F084802B4B9B6C012B6AD1294B17
:10225000DB6CB3F1FF3F0BD0274B1A68274B1B6891
:102260001046194638F0EAFC03461A46224B1A601B
:10227000204BDB6CB3F1FF3F12D1386A204938F0B4
:1022800027FE0346002B0BD01B4B1A681B4B1B6809
:102290001046194638F0D2FC03461A46164B1A600F
:1022A000386A184938F014FE0346002B3AD0114B17
:1022B00005229A700123FB71134B0022DA71134B34
:1022C000B3F834321A461201D31A9B009AB2104B5B
:1022D0001A80104B00221A800F4B00221A800F4BDD
:1022E00000221A600E4B00225A600C4B00221A602A
:1022F00044E300BF20270010800000107C00001085
:10230000000048C20000FAC3300A001004070010A1
:10231000F4060010601E0010F81D0010280A0010BE
:1023200040220010A54B9B6C002B10D1A34BDB6C03
:10233000B3F1FF3F0BD0A24B1A68A24B1B681046AB
:10234000194638F07BFC03461A469D4B1A609E4B9B
:1023500093F83E32184638F075FD0246984B1B68DC
:102360001046194638F0B4FD0346002B08D0964BB2
:1023700093F83E32184638F071FD0246904B1A60D1
:10238000914BD3F868321846396A38F099FB034606
:1023900018468E4938F0F2FB0346BB61B86901F07C
:1023A0008FFD04468A4B1B68184601F089FD0346E1
:1023B00003FB04F3002B03DA854B4FF000021A6095
:1023C000B8694FF0000138F0A1FD0346002B1FD083
:1023D0007F4B1B681846B96938F07AFD0346002B1D
:1023E0000AD07B4B1B6818464FF07F5138F0A4FC95
:1023F00003461A46764B1A60754B1B681846B96936
:1024000038F084FD0346002B02D0714ABB6913608B
:10241000B8694FF0000138F05BFD0346002B1ED079
:102420006B4B1B681846B96938F070FD0346002BEA
:1024300009D0674B1B681846664938F0FFFB034616
:102440001A46634B1A60624B1B681846B96938F02C
:102450003FFD0346002B02D05D4ABB6913604FF07D
:102460007E537B61584BB3F88830002B4ED0534BD2
:102470005B6C184638F0FAFC02460B4610461946CB
:102480004FF00002544B37F047FF02460B4614460C
:102490001D464D4BB3F888301BB2184638F0D2FCBD
:1024A0000346184638F0E2FC02460B462046294611
:1024B00037F09CFE02460B461046194638F0B2F93A
:1024C00003467B613D4B5B6C1846444938F01EFD6A
:1024D0000346002B1AD03A4B1B6818463B4938F08C
:1024E000F7FC0346002B11D03D4B1B681846796959
:1024F00038F0E6FA03461A46314B1B681046194677
:1025000038F01AFC03461A462D4B1A60354B002250
:102510009A762D4B93F84A32012B17D1324B1B7E02
:10252000002B13D1304B5A68274BB3F84C3264332D
:102530009A420BDD244B93F83D32184638F08EFC5E
:1025400002462A4B1A60274B01229A761C4B1B68C5
:102550001A4AD3611E4B1B68184A1362224B5A89D0
:10256000234B1A80204B5B689AB2224B1A801D4B7A
:102570009B7E002B76D1144B93F83D32184638F0F1
:1025800061FC02460E4B1B681046194638F0BEFC33
:102590000346002B08D00C4B93F83D32184638F018
:1025A0005DFC0246064B1A60054B1A68084B1B6817
:1025B0001046194638F0C0FB1EE000BF202700106F
:1025C000800000107C000010040700100000C842CA
:1025D0008800001000004040000024400000A0409F
:1025E00078000010A0270010C42100108400001003
:1025F0006E0000107400001003461A46A34B1A60C8
:10260000A34B93F83D32184638F01CFC02469F4B12
:102610001B681046194638F079FC0346002B08D099
:102620009B4B93F83D32184638F018FC0246974B06
:102630001A60974B93F83E32184638F003FC024676
:10264000924B1B681046194638F042FC0346002B9B
:1026500008D08F4B93F83E32184638F0FFFB024605
:102660008A4B1A60894B1B681846F96938F028FABA
:1026700003461846874938F081FA03461A46864BC6
:102680001A60854B1C68824BB3F81832184638F034
:10269000D9FB03462046194638F070FA034618461F
:1026A0007C4938F00DFA03463B61386901F030FC93
:1026B00002467A4B5A60794B5B68002B02DC774B01
:1026C00001225A60724B93F81332012B40F01E81A5
:1026D0006F4BB3F84E321BB2184638F0B3FB0246CC
:1026E0006D4B1B681046194638F0EAF90346184648
:1026F000684938F043FA03461A46674B1B68104690
:10270000194638F019FB0346184638F0AFFB04466B
:102710000D465F4BB3F81432184638F09FFB034662
:10272000184638F0A3FB02460B46104619464FF0F8
:1027300000025B4B37F0F0FD02460B46204629466F
:1027400037F0EAFD02460B461046194638F06AF8A3
:102750000346FB60F8684F4938F0B2F90346184663
:1027600038F05CFB03469AB24E4BDA80F8684E496B
:1027700038F004FA0346BB604C4B1B681846B96836
:1027800038F0DAFA03461A46484B1A60404B93F881
:102790003C32184638F062FB03463B633C4BD3F8AF
:1027A0001C321846404938F0E9F903467B633F4B39
:1027B0001B681846796B38F0E1F903461846396B07
:1027C00038F0E2FB0346002B07D1394B1B7F002B6F
:1027D00078D0384BDB79002B74D1354B1B7F002B25
:1027E0000ED1324B1C68386B796B38F069F90346AF
:1027F0002046194638F022FA03461A462B4B1A6037
:10280000284BDC68386B796B38F05AF90346204660
:10281000194638F091FA03461A46224BDA60264BE5
:102820009C6B386B796B38F04BF9034620461946A0
:1028300038F004FA03461A461F4B9A631D4B0122D7
:10284000DA711C4B01229A71386B4FF07E5138F0CF
:1028500073FA0346184638F0E1FA03469AB2174B6A
:102860001A80154BDB8E9AB2094B93F83C329BB21F
:1028700013449BB29AB2104BDA860D4B1B7F002B90
:1028800020D00B4B1B7F013BDAB219E08400001013
:10289000040700100000C8428C0000104022001005
:1028A0000000244020270010000061459000001027
:1028B000A0270010300A00101C1E00109400001009
:1028C000304B1A77304BDB79012B1ED1386901F080
:1028D0001FFB02462D4B93F8563213442C4A53608B
:1028E0002B4B5B68642B02DD294B64225A60294B19
:1028F0001B88013B9AB2274B1A80264B1B88002B62
:1029000003D1214B0022DA7103E002E01E4B0022CA
:10291000DA71214B1B681846204938F0D1F803467C
:10292000184638F07BFA03469AB21D4B9A803869F4
:1029300038F074FA03469AB2194B1A81FB79002BCE
:1029400003D1184B1B78002B15D0104B93F83D3258
:102950000A33184638F076FA0246134B1A60386B81
:10296000796B38F0ADF803461A46104B1A60094BE4
:102970004FF47A721A800B4B00221A703837BD461A
:10298000B0BD00BFA0270010300A001004070010DF
:1029900040220010940000108C0000100000C8427B
:1029A000202700100400001080000010900000108C
:1029B00090B585B000AFA44B1A7DA44B83F83620A8
:1029C000A34BB3F81031FB81A14B93F81731022BC5
:1029D00003D101F005F90346FB819D4B93F81731B4
:1029E000002B00F0DB809A4B93F81631002B72D04D
:1029F000984B1B78022B02D1964B01221A70964BF2
:102A0000DB891AB2B7F90E10914BB3F812311BB231
:102A1000CB1A9A4235DA8F4B01221A708F4B002263
:102A20001A708B4B9B7D002B02D0884B00225A855D
:102A3000874B93F80831002B02D1884B00225A7043
:102A4000834BB3F814319AB2FB8913449BB29AB208
:102A50007E4B1A807D4B012283F851207E4B5B898F
:102A60001AB27D4BDB891BB264339A4209DD7A4B83
:102A70005B891BB240F6AC52934202DD774B0122D8
:102A80009A70744B1B78012B74D1734BDB89B7F9A7
:102A90000E201BB29A426DDC6D4BB3F8B8216B4B24
:102AA0001A806A4B93F86130012B0CD1684BB3F854
:102AB000B8319AB2664BB3F80A329BB2D31A9BB2C2
:102AC0009AB2624B1A80634B00221A705F4B00224D
:102AD00083F851204EE05F4B1B78012B02D15D4BF8
:102AE00002221A705A4BB3F8B821584B1A80574B30
:102AF00093F86130012B0CD1554BB3F8B8319AB231
:102B0000534BB3F80A329BB2D31A9BB29AB24F4BD3
:102B10001A80514B5B891AB24F4BDB891BB264336D
:102B20009A4218DD4C4BDB891AB2B7F90E10484BAC
:102B3000B3F812311BB2CB1A9A420CDA464B5B89BE
:102B40001BB240F6D862934205DD444B01229A70D5
:102B5000404B02221A70404BDB891AB2B7F90E10B3
:102B60003B4BB3F812311BB2CB1A9A4202DA3C4B00
:102B700001221A70384B5B891AB2374BDB891BB2C2
:102B800064339A4206DB344B5B891BB240F6D76252
:102B9000934223DC314B00229A701FE02D4B002220
:102BA0001A702B4BB3F8B821284B1A80274B93F897
:102BB0006130012B0CD1264BB3F8B8319AB2244BBB
:102BC000B3F80A329BB2D31A9BB29AB21F4B1A8047
:102BD000224B00229A70224B00221A701E4BDB8976
:102BE000B7F90E201BB29A4205DC1C4B00229A70EA
:102BF000184B00221A70164B93F81731032B0DD186
:102C0000154B5B891BB240F6D862934203DD134B30
:102C100001229A7002E0114B00229A700C4B93F83B
:102C2000B031002B02D10F4B00221A70084B93F8E1
:102C3000B031012B32D1064B93F8B431012B13D1B3
:102C4000084B01221A7029E0F421001020270010FF
:102C5000040700109A000010C4210010300A001070
:102C6000F02100109B000010A64BDA89A64BB3F8A8
:102C7000B23112B21BB29A4203DBA44B01221A708A
:102C80000CE0A04BDB891AB29F4BB3F8B2311BB2F8
:102C9000143B9A4202DA9D4B00221A709A4B93F829
:102CA000B031022B28D1984B93F8B431012B06D1C7
:102CB00000F0F4FF0346DAB2944B1A701CE0914B1B
:102CC000DA89914BB3F8B23112B21BB29A4206DBE9
:102CD00000F0E4FF0346DAB28C4B1A700CE0894B2B
:102CE000DB891AB2884BB3F8B2311BB2143B9A425B
:102CF00002DA864B00221A70844B1B78012B09D113
:102D0000834B1B78002B05D1824B01221A80824B0A
:102D100000221A807D4B1A787D4B1A707D4B1B88E0
:102D2000002B18D07B4B1B8801339AB2794B1A8049
:102D3000784B1B881946744B93F8B6311A461346E4
:102D40001B019B1A9B00994205DB724B00221A80E3
:102D5000714B01221A80704B1B88002B18D06E4BD0
:102D60001B8801339AB26C4B1A806B4B1B88194637
:102D7000654B93F8B7311A4613461B019B1A9B000B
:102D8000994205DB634B01221A80634B00221A80B3
:102D90005E4B1B78002B05D05E4B1B88002B01D0AF
:102DA000012300E00023DAB25C4BDA7000F0F0FCA3
:102DB0005B4B1B78012B00F0B282534BB3F8B82168
:102DC000584B1A80574B93F86130012B0CD14E4B66
:102DD000B3F8B8319AB24C4BB3F80A329BB2D31A5B
:102DE0009BB29AB24F4B1A80474B93F810325BB2AA
:102DF0004B2B1CD14B4B1B889AB24A4B9B8E9BB2E0
:102E000013449BB29AB2474B1A80464B022283F876
:102E10005120444B1A883C4BB3F8B83112B21BB264
:102E20009A4208D13F4B002283F8512003E03D4BEA
:102E3000002283F85120344B93F80831002B3AD10B
:102E400001F058FB0346002B2FD001F007FB03468F
:102E5000002B2AD02C4B93F8AF30012B09D02A4BF2
:102E600093F8AF30022B20D100F052FE0346002B26
:102E70001BD02D4B01221A70224B5B891BB2224AB8
:102E8000B2F8AC20934202DD244B01225A701D4B54
:102E90005B891AB21C4BB3F8AC30143B9A4203DA8C
:102EA0001E4B00225A7006E005E01C4B00225A70AF
:102EB0001D4B00221A70144B93F82930012B40F05F
:102EC000718101F09BFA0346002B00F06B810E4BE1
:102ED0001B7D002B00F046810B4B9B7A002B00F0F2
:102EE000B18000F055FC0346FB72104AFB7A137068
:102EF000054B93F82830012B1AD1084B01221A7088
:102F000028E000BFC4210010040700109B0000103F
:102F10009C0000109E000010A0000010300A00105D
:102F20009A0000102027001017270010E02700103B
:102F3000834B5B891BB2834AD28C934202DB824A69
:102F4000FB7A1370804B1B78002B03D17F4B4FF023
:102F500000021A607E4B1B8D9AB2794B5B8A9BB242
:102F6000D31A9BB23B81B7F90830184637F06AFF95
:102F700003461846774937F0A3FD03461A46734BBC
:102F80001B681046194637F0D7FE03461A466F4BAA
:102F90001A606E4B1B6818466F4937F0B7FF03463F
:102FA000002B02D0694B6C4A1A60684B1B681846AC
:102FB0006A4937F08DFF0346002B02D0634B674A06
:102FC0001A60624B1B68624A53625E4B9B891946CA
:102FD000B7F908305B4A527D02FB03F30B441846F5
:102FE00037F030FF0246594B1B681046194637F040
:102FF000A3FE0346184637F0F7FE0346BB81514B4C
:1030000093F811325BB24D2B06D1514B9B8E9AB285
:10301000BB8913449BB2BB81B7F90C30494A128A71
:10302000934202DD474B1B8ABB81B7F90C30454AFE
:10303000D289934202DA434BDB89BB81444ABB8984
:103040005385A4E03F4B9B8C002B2FD101F036FA27
:103050000346002B23D03D4B4FF000021A603A4B41
:1030600001221A70374B9B899AB2394B5A85354BDE
:1030700093F811325BB24D2B0AD1354B5B8D9AB26E
:10308000334B9B8E9BB213449BB29AB2304B5A8502
:1030900000F07EFB03461A46314B1A7077E02A4B4C
:1030A00000221A702E4B00221A7070E0274B4FF04E
:1030B00000021A60244B01221A7001F0FFF9034646
:1030C000002B05D01F4B9B899AB2214B5A8509E0F2
:1030D0001C4B9A891B4B9B8C9BB2D31A9BB29AB206
:1030E0001B4B5A85174B93F811325BB24D2B0AD10B
:1030F000174B5B8D9AB2164B9B8E9BB213449BB2BF
:103100009AB2134B5A85124B5B8D1BB20D4A128A31
:10311000934204DD0B4B1B8A9AB20D4B5A850C4B24
:103120005B8D1BB2074AD289934204DA054BDB89D7
:103130009AB2074B5A850A4B01221A7027E000BF4A
:10314000C421001004070010300A0010A400001071
:1031500020270010A69B443B0000FA430000FAC35E
:10316000E027001000F014FB0346FB718E4B5B89D7
:103170001BB28E4AD28C934202DB8D4AFB791370CC
:103180008C4AFB7913708C4B4FF000021A60864B0F
:103190005B891AB2854BDB8C323B9A4202DA844B54
:1031A00000221A70814B93F82930002B08D1804BF4
:1031B00000221A70814B00225A857E4B00221A7021
:1031C0007A4B93F82930022B40F0888001F016F9F1
:1031D0000346002B00F08280744B1B7D002B6CD0CB
:1031E00001F04CFA0346002B14D0704B9B899AB225
:1031F000724B5A8501F062F90346002B14D16B4BD8
:103200009A896A4B9B8C9BB2D31A9BB29AB26B4B36
:103210005A8509E0654B9A89644B9B8C9BB2D31A03
:103220009BB29AB2654B5A85604B93F811325BB2F0
:103230004D2B0AD1614B5B8D9AB2604B9B8E9BB23A
:1032400013449BB29AB25D4B5A855C4B5B8D1BB2AB
:10325000564A128A934204DD544B1B8A9AB2574B4A
:103260005A85564B5B8D1BB2504AD289934204DA81
:103270004E4BDB899AB2514B5A854C4B93F8283010
:10328000012B03D14A4B01221A701CE000F080FA96
:103290000346FB72444B5B891BB2444AD28C934277
:1032A00002DB434AFB7A1370414B1B78002B0AD197
:1032B000414B4FF000021A6005E001F0DFF90346D0
:1032C000DAB23B4B1A70384B5B891AB2374BDB8C46
:1032D000323B9A4202DA364B00221A70384BDB7EC0
:1032E000002B0DD101F08AF80346002B08D1304B9A
:1032F00000221A70314B00225A852E4B00221A7080
:103300002A4B1B7D002B0AD0294B1B78002B06D1A2
:10331000264B9B7D002B02D0284B00225A85234B45
:1033200093F80831002B10D001F078F903461A46C3
:103330001F4B5A701C4B5B891BB21C4AB2F8AC2065
:10334000934202DA1A4B00225A701C4B1A88174B10
:10335000B3F8BC3112B21BB29A4204DD134BB3F87E
:10336000BC21164B1A80154B1B881BB240F6B73296
:10337000934203DC114B40F6B8321A800C4B1B7899
:103380001A46104B1A60084B5A89084BB3F80E3294
:1033900012B21BB29A4219DB084B9B6D0A2B18D94B
:1033A000094B01225A7414E0C421001004070010D4
:1033B000300A0010E0270010A400001020270010A1
:1033C000A0270010A8000010140A0010784B00225B
:1033D0005A74784B1B891BB241F6583293422CDD4C
:1033E000754A754B9B6943F400239361704B9B7A3C
:1033F000012B22D00DF020FD704B01221A706F4B73
:1034000001225A706D4B01229A700220002109F0AE
:10341000C5FF674B01229A72694B9B78032B0CD036
:10342000674B03229A70674BB3F844321A46120175
:10343000D31A9B009AB2624B9A875E4B5B7E002B3D
:1034400018D00DF0F9FC5D4B01221A705B4B012284
:103450005A705A4B01229A70594B00229A70544B61
:10346000DB78012B03D00720002109F097FF504B98
:103470000122DA704E4BDB78002B07D14C4B9B7A44
:10348000002B03D14A4B5B7B002B05D04A4A4A4BA9
:103490009B6943F400239361454BDB78002B11D1EA
:1034A000434B9B7A002B0DD1414B5B7B002B09D109
:1034B000454B9B7D002B05D13F4A3F4BDB6943F4D5
:1034C0000023D3613A4B9B7C002B18D13F4B9C6B64
:1034D0003C4BB3F854321BB2184637F0B3FC0346EA
:1034E0002046194637F0F4FC0346002B00D11AE0C1
:1034F0002F4B01229A74344B14229A7513E0334BEC
:103500009C6B304BB3F854321BB2184637F09AFC20
:1035100003462046194637F0F9FC0346002B02D03B
:10352000234B00229A74234B5B891BB242F2283250
:10353000934226DD0DF080FC204B01221A701F4BB8
:1035400001225A701D4B01229A701C4B0122DA7025
:103550001D4B0122DA761A4B9B78032B06D0184BB1
:103560009B78002B02D0164B00229A70104B5B7B8D
:10357000012B03D00620002109F010FF0C4B012283
:103580005A730C4B5B891BB242F2971293421FDDB8
:103590000A4B01221A70094B01225A70074B012273
:1035A0009A70064B0122DA70074B0122DA7612E09C
:1035B000140A0010C421001000C00920300A0010B5
:1035C0002027001004070010A02700101C1E001068
:1035D000514B0022DA76514B9B7E002B20D00DF010
:1035E0002BFC4F4B01221A704D4B01225A704C4B51
:1035F00001229A704B4B9B78032B06D0494B9B784A
:10360000002B02D0474B00229A70474B1B79012BAD
:1036100003D00820002109F0C1FE434B01221A719A
:103620003E4BDB7F002B13D0404B1B7D012B0FD17A
:103630003E4B93F82930012B0AD13B4BDB79012B10
:1036400003D00D20002109F0A9FE374B0122DA71C9
:10365000324BDB7E002B10D0344B93F882305BB2C0
:10366000012B0AD1304B5B79012B03D011200021B3
:1036700009F094FE2C4B01225A71284B1B7F002B22
:103680000FD02A4B93F81731002B0AD0264B9B7989
:10369000012B03D00920002109F080FE224B0122DA
:1036A0009A711E4B9B7F002B0ED0204B9B7A002BD8
:1036B0000AD01D4B5B7A012B03D00C20002109F0AE
:1036C0006DFE194B01225A72184B93F84A32012BA6
:1036D0000ED1124B1B7E002B0AD0134B9B78012B73
:1036E00003D00A20002109F059FE0F4B01229A70E5
:1036F0000D4B9B7B002B03D10B4BDB7B002B07D0AF
:10370000084B00229A70064B0022DA7101F068F92A
:103710001437BD4690BD00BFA0270010C421001083
:10372000300A001020270010140A001004070010AF
:1037300080B485B000AF0346FB710123FB73124BCD
:103740005B891AB2114BB3F8B8311BB2A3F5C87339
:103750009A4212DC0D4B93F84A32012B0BD10A4BE3
:103760005B68A3F5FA72084B5B891BB29A4204DCD2
:103770000023FB7301E00023FB73FB7B1846143727
:10378000BD465DF8047B7047C4210010040700109B
:1037900080B500AF2F4B9B7A002B03D12E4B42F20A
:1037A0000F721A852B4B9B7A012B04D1294BDB8896
:1037B0009AB2294B1A85274B9B7A022B04D1254BB1
:1037C0009B889AB2244B1A85224B9B7A032B06D1F5
:1037D000002000F02BF903461A461F4B1A851F4B99
:1037E0005B8A1AB21C4B1B8D1BB21A4909895B1AE2
:1037F0009A4202DC1A4B01221A70184B5B8A1AB2E9
:10380000154B1B8D1BB2134909890B449A4202DBED
:10381000134B00221A70114B9B7F002B02D0104BD0
:1038200001221A700B4B9B7A002B07D100F046FE49
:103830000346002B02D00A4B01221A7000F03EFE14
:103840000346002B02D1064B00221A70044B1B7852
:10385000184680BD0407001020270010C421001066
:103860000500001080B485B000AF0C4BBB60142382
:10387000FB800023FB8107E0FB89BA681344002228
:103880001A70FB890133FB81FA89FB889A42F3D3D2
:103890001437BD465DF8047B704700BF140A001062
:1038A00080B485B000AF114BBB6000237B73142341
:1038B000FB800023FB810EE0FB89BA6813441B7870
:1038C0007B7197F90530002B02D07B7B01337B7332
:1038D000FB890133FB81FA89FB889A42ECD37B7B1D
:1038E00018461437BD465DF8047B7047140A001073
:1038F00080B500AF204B5B7E9AB2204B1A831E4BE3
:103900005A8A1E4B5A821C4BDB7D184637F0A6FAAA
:1039100002461A4B5A60184B1B7E184637F09EFA27
:103920000246164B9A60144B1B8CDAB2134B9A76F4
:10393000114B9A8B114B5A860F4BDA8B0F4B9A8691
:103940000D4B9A7E0D4B83F830200B4B93F82220C1
:103950000A4B83F836200A4B5A8D084B1A80074BC6
:10396000DB68074AD362002000F00CF803461A46D1
:10397000034B9A8680BD00BF04070010F42100109D
:103980002027001080B485B000AF0346FB710023F0
:10399000FB60FB79224A862101FB03F31344DB7AA7
:1039A0009BB21A46920013445B009BB27B811D4B75
:1039B0001B8A3B81B7F90830B3F57A7F02DB00231D
:1039C000FB6017E03B89A3F57A739BB23B813B898F
:1039D0005B429BB23B81B7F90830B7F90A2002FB82
:1039E00003F3FB60FB68104A82FB03125211DB17E2
:1039F000D31AFB60FB68002B01DA0023FB60FB6835
:103A000040F6B832934201DD0023FB60FB689BB2B5
:103A10001BB218461437BD465DF8047B704700BFE3
:103A200004070010C42100101F85EB5190B58DB024
:103A300000AF0346FB71002387F82B3000233B8542
:103A4000002387F82F300023BB8507F108032D489A
:103A500019460AF0EBFCBB6987F82B303B699BB237
:103A60001A461201D31A9B009AB2FB689BB2134408
:103A70003B853B8D244AA2FB03231B093B85FB7935
:103A8000224A862101FB03F31344DB88BB85002314
:103A900087F82F302BE0F87997F82F2097F82B1024
:103AA0001A4C1346DB009B1A862202FB00F21344D9
:103AB00023440B4430331B79012B13D1398D97F8F4
:103AC0002F20FB79084611461A4634F08DF903463B
:103AD0004B2B07D1FB790D4A862101FB03F31344DD
:103AE0009B88BB8597F82F30013387F82F3097F8E4
:103AF0002F30032BCFD9BB8D1BB218463437BD46B0
:103B000090BD00BF004002408988888804070010EB
:103B100090B58BB000AF012387F82330002387F8DE
:103B2000223000233B84002387F827300023BB8406
:103B30003B46284819460AF079FC3B6987F8223051
:103B4000BB689BB21A461201D31A9B009AB27B68DB
:103B50009BB213443B843B8C1F4AA2FB03231B09EB
:103B60003B840023BB84002387F8273028E097F8A4
:103B7000230097F8272097F82210184C1346DB00F3
:103B80009B1A862202FB00F2134423440B44303379
:103B90001B79012B0FD1398C97F8272097F8233008
:103BA000084611461A4634F01FF903464B2B02D142
:103BB00041F28833BB8497F82730013387F82730E8
:103BC00097F82730032BD2D9BB8C1BB218462C3761
:103BD000BD4690BD004002408988888804070010D7
:103BE00080B58AB000AF002387F8233000233B84E0
:103BF000002387F827300023BB843B46244819461E
:103C00000AF014FC3B6987F82330BB689BB21A4664
:103C10001201D31A9B009AB27B689BB213443B8477
:103C20003B8C1C4AA2FB03231B093B840023BB845F
:103C3000002387F8273021E097F8272097F82310F2
:103C400015481346DB009B1A03440B4403F58C73A1
:103C50001B78012B0DD13A8C97F827301046194666
:103C600033F0C6FF03464B2B03D10B4BB3F8103197
:103C7000BB8497F82730013387F8273097F827302F
:103C8000032BD9D9BB8C1BB218462837BD4680BD43
:103C900000400240898888880407001080B58AB0F7
:103CA00000AF002387F8233000233B84002387F8EC
:103CB00027300023BB843B46234819460AF0B6FB55
:103CC0003B6987F82330BB689BB21A461201D31AAE
:103CD0009B009AB27B689BB213443B843B8C1B4A8B
:103CE000A2FB03231B093B840023BB84002387F82A
:103CF00027301FE097F8272097F823101448134621
:103D0000DB009B1A03440B4403F5B0731B79012BB2
:103D10000BD13A8C97F827301046194633F0E6FF5E
:103D200003464B2B01D10123BB8497F82730013385
:103D300087F8273097F82730032BDBD9BB8C1BB2D1
:103D400018462837BD4680BD0040024089888888D3
:103D50000407001080B400AF534B1B78002B05D133
:103D6000524B1B680133514A136002E04F4B002253
:103D70001A604D4B5B78002B05D14D4B1B6801330E
:103D80004B4A136002E04A4B00221A60474B1B6803
:103D9000484A93420BD9444B01221A70424B0122EC
:103DA0009A72454B14229A74404B00221A60404B81
:103DB0001B68404A93420BD93B4B01225A703A4B45
:103DC0000122DA723C4B14229A74394B00221A6099
:103DD000394B9B7C002B27D0334B01221A70324B7E
:103DE00001229A72304B01225A702F4B0122DA7253
:103DF000314B9B7C013BDAB22F4B9A742E4B9B7C50
:103E0000002B11D1284B00221A70274B00229A72E6
:103E1000254B00225A70244B0022DA72234B0022D9
:103E20001A60234B00221A601F4B9B78002B05D190
:103E3000224B1B680133214A136002E01F4B002212
:103E40001A601E4B1B681B4A93420BD9164B01226A
:103E50009A70154B01221A73174B1422DA74174B00
:103E600000221A60144BDB7C002B18D00E4B012271
:103E70009A700D4B01221A730F4BDB7C013BDAB2B7
:103E80000D4BDA740C4BDB7C002B08D1064B002267
:103E90009A70054B00221A73084B00221A60BD4627
:103EA0005DF8047B704700BF300A001058220010F4
:103EB000DC270010002F0D00A0270010FC1D0010B3
:103EC00080B584B000AF786078684FF0000136F0BC
:103ED000FFFF0346002B02D04FF0FF33FB607868F2
:103EE0004FF0000137F012F80346002B01D00123F8
:103EF000FB6078684FF0000136F0DAFF0346002BD4
:103F000001D00023FB60FB6818461037BD4680BD1A
:103F10002DE9B043A2B000AF7860B34B93F82232E2
:103F20005BB2184636F08EFF0446AF4B93F8213251
:103F30005BB2184636F086FF03462046194636F037
:103F40007DFE0346BB67B86FA84936F017FE0346EF
:103F5000BB67A54B93F822325BB2184636F0F6FCED
:103F600004460D46786836F081FF02460B464FF056
:103F700000009F4936F086FA02460B469046994665
:103F8000B86F36F073FF02460B464046494636F09E
:103F90002DF902460B462046294636F073FA0246B2
:103FA0000B461046194636F03DFC0346C7F88430F0
:103FB000002387F87F300CE097F87F3007F1880204
:103FC0001344002203F87C2C97F87F30013387F8E4
:103FD0007F3097F87F300A2BEED9834B93F823324A
:103FE0005BB2184636F02EFF03461846814936F07C
:103FF000C5FD03467B67002387F873304FF000034D
:10400000C7F880300B2387F87F3019E0D7F880009D
:10401000796F36F091FE0346C7F8803097F87F40FD
:10402000D7F8800036F0E0FE0346DAB207F18803E5
:10403000234403F87C2C97F87F30013387F87F30D6
:1040400097F87F30132BE1D9674B93F8233287F829
:104050002030654B93F824325BB2184636F0F2FEFE
:104060000446614B93F823325BB2184636F0EAFE01
:1040700003462046194636F0E1FD034618465D49E1
:1040800036F07CFD03467B67002387F87330564B80
:1040900093F823325BB2184636F0D4FE0346C7F8D5
:1040A0008030152387F87F3019E0D7F88000796FCA
:1040B00036F042FE0346C7F8803097F87F40D7F8C5
:1040C000800036F091FE0346DAB207F188032344FC
:1040D00003F87C2C97F87F30013387F87F3097F80E
:1040E0007F301D2BE1D9404B93F8243287F82A30DA
:1040F0003D4B93F826325BB2184636F0A3FE0446D9
:10410000394B93F824325BB2184636F09BFE0346D7
:104110002046194636F092FD03461846364936F0D9
:104120002DFD03467B67002387F873302E4B93F8F1
:1041300024325BB2184636F085FE0346C7F880305D
:104140001F2387F87F3019E0D7F88000796F36F0A9
:10415000F3FD0346C7F8803097F87F40D7F880001A
:1041600036F042FE0346DAB207F18803234403F82F
:104170007C2C97F87F30013387F87F3097F87F30B9
:10418000312BE1D9184B93F8263287F83E30164B85
:1041900093F828325BB2184636F054FE0446124BB0
:1041A00093F826325BB2184636F04CFE03462046A2
:1041B000194636F043FD034618460F4936F0DEFC3B
:1041C00003467B67002387F87330074B93F826324A
:1041D0005BB2184636F036FE0346C7F8803033230C
:1041E00087F87F3024E000BF040700100000B442CD
:1041F00000005940000020410000A041D7F8800095
:10420000796F36F099FD0346C7F8803097F87F4004
:10421000D7F8800036F0E8FD0346DAB207F18803EC
:10422000234403F87C2C97F87F30013387F87F30E4
:1042300097F87F30452BE1D96D4B93F8283287F8FA
:1042400052306B4B93F82A325BB2184636F0FAFDC7
:104250000446674B93F828325BB2184636F0F2FDFD
:1042600003462046194636F0E9FC034618466149E4
:1042700036F084FC03467B67002387F873305C4B81
:1042800093F828325BB2184636F0DCFD0346C7F8D7
:104290008030472387F87F3019E0D7F88000796FA6
:1042A00036F04AFD0346C7F8803097F87F40D7F8CC
:1042B000800036F099FD0346DAB207F18803234403
:1042C00003F87C2C97F87F30013387F87F3097F81C
:1042D0007F30592BE1D9464B93F82A3287F8663064
:1042E000434B93F82A325BB2184636F0ABFD0346D7
:1042F000184636F0BBFD02460B464FF000004FF06B
:10430000000136F0BFF802460B46104619464FF042
:104310000002394B36F000F802460B4610461946AB
:1043200036F080FA03467B67002387F87330304B02
:1043300093F82A325BB2184636F084FD0346C7F87C
:1043400080305B2387F87F3019E0D7F88000796FE1
:1043500036F0F2FC0346C7F8803097F87F40D7F874
:10436000800036F041FD0346DAB207F188032344AA
:1043700003F87C2C97F87F30013387F87F3097F86B
:104380007F30632BE1D9002387F87030D7F88400A1
:1043900035F096F90446786836F040FD0346DBB206
:1043A00007F18802134413F87C3C5BB2184636F0E0
:1043B00049FD03462046194636F0BEFC0346C7F8C1
:1043C0008430D7F884004FF07E5136F081FD0346EB
:1043D000002B03D04FF07E53C7F88430D7F8840009
:1043E00036F002FD034618468837BD46BDE8B08367
:1043F000040700100000A0410000244080B400AF7A
:10440000134B5B7F002B03D0124B01221A7018E074
:104410000F4B1A8A104BB3F8803012B21BB29A427B
:1044200002DB0C4B00221A70094B1B8A1AB20A4B92
:10443000B3F880301BB2323B9A4202DA054B0122BC
:104440001A70044B1B781846BD465DF8047B704714
:10445000C4210010BA0000100407001080B400AF9F
:10446000134B5B7F002B03D0124B01221A7018E014
:104470000F4B1A8A104BB3F8063112B21BB29A4294
:1044800002DB0C4B00221A70094B1B8A1AB20A4B32
:10449000B3F806311BB2323B9A4202DA054B0122D5
:1044A0001A70044B1B781846BD465DF8047B7047B4
:1044B000C4210010BB0000100407001080B483B0BA
:1044C00000AF0023FB71094B93F80B33002B02D193
:1044D0000123FB7102E0064B1B78FB71FB79184648
:1044E0000C37BD465DF8047B704700BF0407001021
:1044F0009827001080B483B000AF0023FB71094BF4
:1045000093F80C33002B02D10123FB7102E0064B20
:104510005B78FB71FB7918460C37BD465DF8047B70
:10452000704700BF040700109827001080B58AB0BC
:1045300000AF012387F82330002387F822300023BF
:104540003B84002387F827300023BB843B46244864
:10455000194609F06BFF3B6987F82230BB689BB2B4
:104560001A461201D31A9B009AB27B689BB213447D
:104570003B843B8C1B4AA2FB03231B093B84002387
:10458000BB84002387F827301FE097F8272097F88F
:10459000221015481346DB009B1A03440B4403F515
:1045A000DC739B79012B0BD13A8C97F8273010469E
:1045B000194634F0F5FB03464B2B01D10123BB8494
:1045C00097F82730013387F8273097F82730032BE7
:1045D000DBD9BB8C1BB218462837BD4680BD00BF57
:1045E00000400240898888880407001080B582B0A6
:1045F00000AF0023FB71FFF799FF0346002B06D1A4
:10460000054B93F80D32022B01D10123FB71FB798D
:1046100018460837BD4680BD0407001080B400AFBF
:10462000134B9B891AB2134BB3F80A3119B2114BD1
:10463000B3F80C311BB2CB1A9A4202DA0E4B0122AC
:104640001A700D4B1B78002B0BD0094B9A89094B24
:10465000B3F80A3112B21BB29A4202DB064B0022B7
:104660001A70054B1B781846BD465DF8047B7047F1
:10467000C421001004070010BC00001080B58AB0EF
:1046800000AF012387F82330002387F8223000236E
:104690003B84002387F827300023BB843B46244813
:1046A000194609F0C3FE3B6987F82230BB689BB20C
:1046B0001A461201D31A9B009AB27B689BB213442C
:1046C0003B843B8C1B4AA2FB03231B093B84002336
:1046D000BB84002387F827301FE097F8272097F83E
:1046E000221015481346DB009B1A03440B44303359
:1046F0001B79012B0CD13A8C97F8273010461946BC
:10470000002233F071FB03464B2B01D10123BB8404
:1047100097F82730013387F8273097F82730032B95
:10472000DBD9BB8C1BB218462837BD4680BD00BF05
:1047300000400240898888880407001080B582B054
:1047400000AF0E4B7B600E4B3B6007E03B681A1DD1
:104750003A607A68111D796012681A603B68094AEC
:104760009342F3D3084809494FF000028842B8BF8A
:1047700040F8042BFADB34F099FFFEE710D4050073
:10478000000000102800001028000010E463001052
:1047900080B400AFFEE700BF80B400AFFEE700BF0B
:1047A00080B400AFFEE700BF80B400AFFEE700BFFB
:1047B00080B400AFFEE700BF80B400AFFEE700BFEB
:1047C00080B400AFFEE700BF80B400AFFEE700BFDB
:1047D00080B400AFFEE700BF80B400AFFEE700BFCB
:1047E00080B483B000AF0346FB71084997F90730E6
:1047F0005B09FA7902F01F02012000FA02F241F887
:1048000023200C37BD465DF8047B704700E100E0D3
:1048100080B500AF0F4A0F4B1B6923F400031361EF
:104820000C4A0C4B1B6943F4800313610A4A0A4B80
:10483000D3F8483143F00203C2F84831064A064B28
:10484000D3F84C3143F00203C2F84C311320FFF788
:10485000C7FF80BD00C0024000C00F4080B400AF61
:10486000054B0222C3F84021044B00221A60BD46CA
:104870005DF8047B704700BF00C00F40402200106D
:1048800080B582B000AF00233B710023FB70012391
:10489000BB701B237B7000233B703B46184609F01E
:1048A000DFFC1C237B703B46184609F0D9FC054809
:1048B000054909F01BFA0348012109F057FA0837A6
:1048C000BD4680BD00C00140C027090080B500AFD3
:1048D0000F4B50221A600E4B0E4A5A600C4B0322AB
:1048E0009A600B4B00221A61094B00225A61084B57
:1048F0000322DA6108480649002209F08FFA0346CC
:10490000012B01D1002301E04FF0FF33184680BD99
:10491000102800100800001000C0014080B500AF52
:104920000F4B50221A600E4B0E4A5A600C4B02225B
:104930009A600B4B0C4A1A61094B01225A61084BD1
:104940000322DA6109480649002209F067FA0346A2
:10495000012B01D1002301E04FF0FF33184680BD49
:10496000E4270010080000100C00001000C00140F7
:1049700080B582B000AF03460A46FB8013467B71C8
:10498000FB881B0A9BB2DAB2064B1A70FB88DAB2BC
:10499000044B5A70034A7B799370FFF797FF0837EF
:1049A000BD4680BD0800001080B582B000AF034650
:1049B000FB80FB881B0A9BB2DAB2074B1A70FB889C
:1049C000DAB2054B5A70FFF7A9FF044B1B78184663
:1049D0000837BD4680BD00BF080000100C00001065
:1049E00080B584B000AF194A184B9B6943F400238B
:1049F0009361174B9A78174B83F81722154BBB60BE
:104A00000023BB814FF44473FB800023FB810FE044
:104A1000FB89BA6813441B787B71BB895A1CBA8125
:104A20007A7918461146FFF7A3FFFB890133FB8112
:104A3000FA89FB889A42EBD3044A044BDB6943F4BE
:104A40000023D3611037BD4680BD00BF00C00920E0
:104A5000202700100407001080B584B000AF164A6C
:104A6000154B9B6943F400239361144BBB6040F6E4
:104A7000C413BB812823FB800023FB810FE0FB894B
:104A8000BA6813441B787B71BB895A1CBA817A7946
:104A900018461146FFF76CFFFB890133FB81FA8949
:104AA000FB889A42EBD3044A034BDB6943F40023AF
:104AB000D3611037BD4680BD00C00920641E0010C0
:104AC00090B585B000AF164A154B9B6943F400239F
:104AD0009361144BBB600023BB814FF44473FB8094
:104AE0000023FB810EE0FB89BA68D418BB895A1CED
:104AF000BA811846FFF758FF0346DBB22370FB89E3
:104B00000133FB81FA89FB889A42ECD3044A044BB7
:104B1000DB6943F40023D3611437BD4690BD00BF69
:104B200000C009200407001090B585B000AF164AF8
:104B3000154B9B6943F400239361144BBB6040F613
:104B4000C413BB812823FB800023FB810EE0FB897B
:104B5000BA68D418BB895A1CBA811846FFF724FFDB
:104B60000346DBB22370FB890133FB81FA89FB88A2
:104B70009A42ECD3044A044BDB6943F40023D3612B
:104B80001437BD4690BD00BF00C00920641E001050
:104B900080B584B000AF104BBB604FF40063BB81A5
:104BA0003C23FB800023FB810FE0FB89BA681344A0
:104BB0001B787B71BB895A1CBA817A7918461146D9
:104BC000FFF7D6FEFB890133FB81FA89FB889A4205
:104BD000EBD31037BD4680BD1C1E001090B585B0CC
:104BE00000AF104BBB604FF40063BB813C23FB80E4
:104BF0000023FB810EE0FB89BA68D418BB895A1CDC
:104C0000BA811846FFF7D0FE0346DBB22370FB895A
:104C10000133FB81FA89FB889A42ECD31437BD46F5
:104C200090BD00BF1C1E001080B584B000AF174AB5
:104C3000164B9B6943F400239361154BBB6040F610
:104C4000B833BB814FF47A73FB800023FB810FE004
:104C5000FB89BA6813441B787B71BB895A1CBA81E3
:104C60007A7918461146FFF783FEFB890133FB81F1
:104C7000FA89FB889A42EBD3044A044BDB6943F47C
:104C80000023D3611037BD4680BD00BF00C009209E
:104C90000003001090B585B000AF104BBB6040F62C
:104CA000B833BB814FF47A73FB800023FB810EE0A5
:104CB000FB89BA68D418BB895A1CBA811846FFF719
:104CC00073FE0346DBB22370FB890133FB81FA8953
:104CD000FB889A42ECD31437BD4690BD0003001008
:104CE00080B483B000AF0023FB800023FB8006E08C
:104CF000FB88074A0021D154FB880133FB80FB88E5
:104D0000632BF5D90C37BD465DF8047B704700BFB7
:104D1000B42D001080B483B000AF0023FB710023DA
:104D2000BB710023FB711FE00023BB710DE0FA791A
:104D3000B97911481346DB009B1A9B000B440344CE
:104D400000225A71BB790133BB71BB79132BEED9A9
:104D5000FA7909491346DB009B1A9B000B44002299
:104D60001A60FB790133FB71FB79632BDCD90C37BB
:104D7000BD465DF8047B7047182E001080B483B0E8
:104D800000AF0023FB710023BB710023FB7129E0FE
:104D90000023BB710CE0FA79BB791649462000FB71
:104DA00002F213440B4400221A70BB790133BB7129
:104DB000BB79132BEFD90023BB710DE0FA79BB79D6
:104DC0000C49462000FB02F20A441344103300222F
:104DD0001A71BB790133BB71BB79312BEED9FB79E9
:104DE0000133FB71FB79132BD2D90C37BD465DF82B
:104DF000047B70473C28001080B590B000AF78600D
:104E0000002387F83F30002387F83E30002387F8DF
:104E10003E3097F83E20DD491346DB009B1A9B008D
:104E20000B44DB4A1A6097F83E20D8491346DB0052
:104E30009B1A9B000B4463221A7197F83E2013467D
:104E4000DB009B1A9B00D14A134405331846D14915
:104E5000132234F004FF97F83E30013387F83E30D8
:104E600097F83E20C9491346DB009B1A9B000B4470
:104E7000C94A1A6097F83E20C4491346DB009B1AC2
:104E80009B000B4463221A7197F83E201346DB0007
:104E90009B1A9B00BD4A134405331846BF49132291
:104EA00034F0DDFE97F83E30013387F83E3097F856
:104EB0003E20BB4B1B681846B4491346DB009B1AC7
:104EC0009B000B44186097F83E20B0491346DB0066
:104ED0009B1A9B000B4477221A7197F83E201346C9
:104EE000DB009B1A9B00A94A134405331846AD49C1
:104EF000132234F0B4FE97F83E30013387F83E3089
:104F000097F83E20A1491346DB009B1A9B000B44F7
:104F100000221A6097F83E209C491346DB009B1A3A
:104F20009B000B4477221A7197F83E201346DB0052
:104F30009B1A9B00954A1344053318469A4913223D
:104F400034F08DFE97F83E30013387F83E3097F805
:104F50003E208E491346DB009B1A9B000B44002227
:104F60001A6097F83E2089491346DB009B1A9B0084
:104F70000B4477221A7197F83E201346DB009B1AE8
:104F80009B00824A1344053318468849132234F0A3
:104F900066FE97F83E30013387F83E3097F83E20A2
:104FA0007A491346DB009B1A9B000B44804A1A6027
:104FB00097F83E2075491346DB009B1A9B000B4473
:104FC0006D221A7197F83E201346DB009B1A9B0056
:104FD0006E4A1344053318467649132234F03FFED7
:104FE00097F83E30013387F83E3097F83E20674906
:104FF0001346DB009B1A9B000B446F4A1A6097F81C
:105000003E2062491346DB009B1A9B000B446D2235
:105010001A7197F83E201346DB009B1A9B005B4AEF
:105020001344053318466549132234F018FE97F8E7
:105030003E30013387F83E3097F83E2053491346FF
:10504000DB009B1A9B000B445D4A1A6097F83E20D8
:105050004E491346DB009B1A9B000B446D221A71CC
:1050600097F83E201346DB009B1A9B00474A1344E7
:10507000053318465349132234F0F1FD97F83E30BA
:10508000013387F83E3097F83E2040491346DB0055
:105090009B1A9B000B4400221A6097F83E203B4964
:1050A0001346DB009B1A9B000B4477221A7197F87A
:1050B0003E201346DB009B1A9B00344A1344053301
:1050C00018464149132234F0CAFD97F83E300133A7
:1050D00087F83E3097F83E202C491346DB009B1A98
:1050E0009B000B44394A1A6097F83E202749134623
:1050F000DB009B1A9B000B446D221A7197F83E202F
:105100001346DB009B1A9B00204A134405331846C4
:105110002F49132234F0A3FD97F83E30013387F86E
:105120003E3097F83E2019491346DB009B1A9B003E
:105130000B4400221A6097F83E2014491346DB0006
:105140009B1A9B000B4477221A7197F83E20134656
:10515000DB009B1A9B000D4A1344053318461D497A
:10516000132234F07CFD97F83E30013387F83E304F
:1051700097F83E2005491346DB009B1A9B000B4421
:1051800000221A6097F83E2026E000BF182E00107B
:105190008A090010AC66040096090010B466040089
:1051A0002C220010BC660400C4660400D066040013
:1051B000CE210010DC660400D0210010EC66040053
:1051C000880700100067040014670400BC08001082
:1051D0002867040038670400DD491346DB009B1A8A
:1051E0009B000B4477221A7197F83E201346DB0090
:1051F0009B1A9B00D64A134405331846D5491322FF
:1052000034F02DFD97F83E30013387F83E3097F8A3
:105210003E20CF491346DB009B1A9B000B44CE4A2D
:105220001A6097F83E20CA491346DB009B1A9B0080
:105230000B446D221A7197F83E201346DB009B1A2F
:105240009B00C34A134405331846C449132234F063
:1052500006FD97F83E30013387F83E3097F83E2040
:10526000BB491346DB009B1A9B000B44BC4A1A60E7
:1052700097F83E20B6491346DB009B1A9B000B446F
:105280006D221A7197F83E201346DB009B1A9B0093
:10529000AF4A134405331846B249132234F0DFFCF9
:1052A00097F83E30013387F83E3097F83E20A84902
:1052B0001346DB009B1A9B000B44AB4A1A6097F81D
:1052C0003E20A3491346DB009B1A9B000B446D2232
:1052D0001A7197F83E201346DB009B1A9B009C4AEC
:1052E000134405331846A149132234F0B8FC97F84B
:1052F0003E30013387F83E3097F83E2094491346FC
:10530000DB009B1A9B000B4400221A6097F83E209A
:105310008F491346DB009B1A9B000B4477221A71BE
:1053200097F83E201346DB009B1A9B00884A1344E3
:10533000053318468E49132234F091FC97F83E301D
:10534000013387F83E3097F83E2081491346DB0051
:105350009B1A9B000B4400221A6097F83E207C4960
:105360001346DB009B1A9B000B4477221A7197F8B7
:105370003E201346DB009B1A9B00754A13440533FD
:1053800018467C49132234F06AFC97F83E3001330A
:1053900087F83E3097F83E206D491346DB009B1A94
:1053A0009B000B44744A1A6097F83E2068491346E4
:1053B000DB009B1A9B000B446D221A7197F83E206C
:1053C0001346DB009B1A9B00614A134405331846C1
:1053D0006A49132234F043FC97F83E30013387F8D2
:1053E0003E3097F83E205A491346DB009B1A9B003B
:1053F0000B4400221A6097F83E2055491346DB0003
:105400009B1A9B000B4477221A7197F83E20134693
:10541000DB009B1A9B004E4A13440533184658493B
:10542000132234F01CFC97F83E30013387F83E30ED
:1054300097F83E2046491346DB009B1A9B000B441D
:10544000504A1A6097F83E2041491346DB009B1AE8
:105450009B000B446D221A7197F83E201346DB0027
:105460009B1A9B003A4A13440533184646491322B7
:1054700034F0F5FB97F83E30013387F83E3097F86B
:105480003E2033491346DB009B1A9B000B443F4AE6
:105490001A6097F83E202E491346DB009B1A9B00AA
:1054A0000B446D221A7197F83E201346DB009B1ABD
:1054B0009B00274A1344053318463549132234F01C
:1054C000CEFB97F83E30013387F83E3097F83E2008
:1054D0001F491346DB009B1A9B000B442D4A1A60A0
:1054E00097F83E201A491346DB009B1A9B000B4499
:1054F0006D221A7197F83E201346DB009B1A9B0021
:10550000134A1344053318462349132234F0A7FBEA
:1055100097F83E30013387F83E3097F83E200C492B
:105520001346DB009B1A9B000B441C4A1A6097F839
:105530003E2007491346DB009B1A9B000B446D225B
:105540001A7197F83E201346DB009B1A9B0027E058
:10555000182E001044670400D22100104C6704008C
:10556000140800105867040016080010646704004F
:10557000706704007C670400180800108C67040042
:1055800098670400D8210010A06704004A27001083
:10559000B067040010070010C06704001207001075
:1055A000DC4A134405331846DB49132234F057FB19
:1055B00097F83E30013387F83E3097F83E20D549C2
:1055C0001346DB009B1A9B000B44D44A1A6097F8E1
:1055D0003E20D0491346DB009B1A9B000B446D22F2
:1055E0001A7197F83E201346DB009B1A9B00C94AAC
:1055F000134405331846CA49132234F030FB97F898
:105600003E30013387F83E3097F83E20C1491346BB
:10561000DB009B1A9B000B44C24A1A6097F83E209D
:10562000BC491346DB009B1A9B000B446D221A7188
:1056300097F83E201346DB009B1A9B00B54A1344A3
:1056400005331846B849052234F009FB97F83E3077
:10565000013387F83E3097F83E20AE491346DB0011
:105660009B1A9B000B44B14A1A6097F83E20A94947
:105670001346DB009B1A9B000B4466221A7197F8B5
:105680003E201346DB009B1A9B00A24A13440533BD
:105690001846A749132234F0E2FA97F83E30013356
:1056A00087F83E3097F83E209A491346DB009B1A54
:1056B0009B000B449F4A1A6097F83E209549134679
:1056C000DB009B1A9B000B4469221A7197F83E205D
:1056D0001346DB009B1A9B008E4A13440533184681
:1056E0009549132234F0BBFA97F83E30013387F81E
:1056F0003E3097F83E2087491346DB009B1A9B00FB
:105700000B448E4A1A6097F83E2082491346DB000C
:105710009B1A9B000B4469221A7197F83E2013468E
:10572000DB009B1A9B007B4A1344053318468449CF
:10573000132234F094FA97F83E30013387F83E3064
:1057400097F83E2073491346DB009B1A9B000B44DD
:105750007C4A1A6097F83E206E491346DB009B1A7C
:105760009B000B4469221A7197F83E201346DB0018
:105770009B1A9B00674A134405331846724913224B
:1057800034F06DFA97F83E30013387F83E3097F8E1
:105790003E2060491346DB009B1A9B000B446B4A7A
:1057A0001A6097F83E205B491346DB009B1A9B006A
:1057B0000B4469221A7197F83E201346DB009B1AAE
:1057C0009B00544A1344053318466149132234F0B0
:1057D00046FA97F83E30013387F83E3097F83E207E
:1057E0004C491346DB009B1A9B000B4400221A60B5
:1057F00097F83E2047491346DB009B1A9B000B4459
:1058000077221A7197F83E201346DB009B1A9B0003
:10581000404A1344053318464E49132234F01FFA08
:1058200097F83E30013387F83E3097F83E203949EB
:105830001346DB009B1A9B000B44474A1A6097F8FB
:105840003E2034491346DB009B1A9B000B446D221B
:105850001A7197F83E201346DB009B1A9B002D4AD5
:105860001344053318463D49132234F0F8F997F8EC
:105870003E30013387F83E3097F83E2025491346E5
:10588000DB009B1A9B000B44354A1A6097F83E20B8
:1058900020491346DB009B1A9B000B446D221A71B2
:1058A00097F83E201346DB009B1A9B00194A1344CD
:1058B000053318462B49132234F0D1F997F83E30BE
:1058C000013387F83E3097F83E2012491346DB003B
:1058D0009B1A9B000B44244A1A6097F83E200D49FE
:1058E0001346DB009B1A9B000B446D221A7197F83C
:1058F0003E201346DB009B1A9B00064A13440533E7
:1059000018461A49132234F0AAF997F83E300133A9
:105910002EE000BF182E0010D067040014070010FE
:10592000E067040028070010F06704004C2700100F
:10593000F86704001B070010086804001C0700102B
:105940001868040019070010286804001D070010DB
:105950003468040044680400D62100105468040030
:1059600048270010646804000A07001074680400E7
:1059700087F83E3097F83E20DD491346DB009B1A3E
:105980009B000B44DB4A1A6097F83E20D849134627
:10599000DB009B1A9B000B446D221A7197F83E2086
:1059A0001346DB009B1A9B00D14A1344053318466B
:1059B000D149132234F053F997F83E30013387F878
:1059C0003E3097F83E20CA491346DB009B1A9B00E5
:1059D0000B44CA4A1A6097F83E20C5491346DB00BB
:1059E0009B1A9B000B446D221A7197F83E201346B8
:1059F000DB009B1A9B00BE4A134405331846C0497E
:105A0000132234F02CF997F83E30013387F83E30FA
:105A100097F83E20B6491346DB009B1A9B000B44C7
:105A200000221A6097F83E20B1491346DB009B1A0A
:105A30009B000B4477221A7197F83E201346DB0037
:105A40009B1A9B00AA4A134405331846AD491322FA
:105A500034F005F997F83E30013387F83E3097F877
:105A60003E20A3491346DB009B1A9B000B440022F7
:105A70001A6097F83E209E491346DB009B1A9B0054
:105A80000B4477221A7197F83E201346DB009B1ACD
:105A90009B00974A1344053318469B49132234F060
:105AA000DEF897F83E30013387F83E3097F83E2015
:105AB0008F491346DB009B1A9B000B4400221A609F
:105AC00097F83E208A491346DB009B1A9B000B4443
:105AD00077221A7197F83E201346DB009B1A9B0031
:105AE000834A1344053318468849132234F0B7F823
:105AF00097F83E30013387F83E3097F83E207C49D6
:105B00001346DB009B1A9B000B44814A1A6097F8EE
:105B10003E2077491346DB009B1A9B000B446C2206
:105B20001A7197F83E201346DB009B1A9B00704ABF
:105B30001344053318467749132234F090F897F848
:105B40003E30013387F83E3097F83E2068491346CF
:105B5000DB009B1A9B000B446F4A1A6097F83E20AB
:105B600063491346DB009B1A9B000B446D221A719C
:105B700097F83E201346DB009B1A9B005C4A1344B7
:105B8000053318466549132234F069F897F83E301A
:105B9000013387F83E3097F83E2055491346DB0025
:105BA0009B1A9B000B445E4A1A6097F83E205049AE
:105BB0001346DB009B1A9B000B446D221A7197F869
:105BC0003E201346DB009B1A9B00494A13440533D1
:105BD00018465449132234F042F897F83E30013306
:105BE00087F83E3097F83E2041491346DB009B1A68
:105BF0009B000B444C4A1A6097F83E203C491346E0
:105C0000DB009B1A9B000B446D221A7197F83E2013
:105C10001346DB009B1A9B00354A13440533184694
:105C20004249132234F01BF897F83E30013387F8CD
:105C30003E3097F83E202E491346DB009B1A9B000E
:105C40000B443B4A1A6097F83E2029491346DB0073
:105C50009B1A9B000B446D221A7197F83E20134645
:105C6000DB009B1A9B00224A134405331846314936
:105C7000132233F0F4FF97F83E30013387F83E30BB
:105C800097F83E201A491346DB009B1A9B000B44F1
:105C9000294A1A6097F83E2015491346DB009B1AE3
:105CA0009B000B4469221A7197F83E201346DB00D3
:105CB0009B1A9B000E4A1344053318461F491322B2
:105CC00033F0CDFF97F83E30013387F83E3097F838
:105CD0003E2007491346DB009B1A9B000B44002221
:105CE0001A6097F83E2002491346DB0028E000BF07
:105CF000182E001008070010846804000C0700101C
:105D000094680400A4680400B0680400C06804003B
:105D1000C8210010CC68040050090010DC680400A1
:105D2000D4210010EC68040084070010F868040017
:105D30000A080010086904000F0700101869040021
:105D40009B1A9B000B4477221A7197F83E2013464A
:105D5000DB009B1A9B00DD4A134405331846DC49DF
:105D6000132233F07CFF97F83E30013387F83E3042
:105D700097F83E20D5491346DB009B1A9B000B4445
:105D8000D44A1A6097F83E20D0491346DB009B1A8C
:105D90009B000B446D221A7197F83E201346DB00DE
:105DA0009B1A9B00C94A134405331846CA4913225B
:105DB00033F055FF97F83E30013387F83E3097F8BF
:105DC0003E20C2491346DB009B1A9B000B44002275
:105DD0001A6097F83E20BD491346DB009B1A9B00D2
:105DE0000B4477221A7197F83E201346DB009B1A6A
:105DF0009B00B64A134405331846B849132233F0C2
:105E00002EFF97F83E30013387F83E3097F83E205A
:105E1000AE491346DB009B1A9B000B4400221A601C
:105E200097F83E20A9491346DB009B1A9B000B44C0
:105E300077221A7197F83E201346DB009B1A9B00CD
:105E4000A24A134405331846A549132233F007FF2D
:105E500097F83E30013387F83E3097F83E209B4953
:105E60001346DB009B1A9B000B449E4A1A6097F86E
:105E70003E2096491346DB009B1A9B000B446D2283
:105E80001A7197F83E201346DB009B1A9B008F4A3D
:105E90001344053318469449132233F0E0FE97F873
:105EA0003E30013387F83E3097F83E20874913464D
:105EB000DB009B1A9B000B448C4A1A6097F83E202B
:105EC00082491346DB009B1A9B000B4469221A711E
:105ED00097F83E201346DB009B1A9B007B4A134435
:105EE000053318468249132233F0B9FE97F83E3045
:105EF000013387F83E3097F83E2074491346DB00A3
:105F00009B1A9B000B447B4A1A6097F83E206F490E
:105F10001346DB009B1A9B000B4469221A7197F809
:105F20003E201346DB009B1A9B00684A134405334E
:105F300018467149132233F092FE97F83E30013330
:105F400087F83E3097F83E2060491346DB009B1AE5
:105F50009B000B44694A1A6097F83E205B49134640
:105F6000DB009B1A9B000B446D221A7197F83E20B0
:105F70001346DB009B1A9B00544A13440533184612
:105F80005F49132233F06BFE97F83E30013387F8F8
:105F90003E3097F83E204D491346DB009B1A9B008C
:105FA0000B44584A1A6097F83E2048491346DB00D4
:105FB0009B1A9B000B4469221A7197F83E201346E6
:105FC000DB009B1A9B00414A1344053318464E4997
:105FD000052233F044FE97F83E30013387F83E3017
:105FE00097F83E2039491346DB009B1A9B000B446F
:105FF000464A1A6097F83E2034491346DB009B1A44
:106000009B000B4469221A7197F83E201346DB006F
:106010009B1A9B002D4A1344053318463C49132212
:1060200033F01DFE97F83E30013387F83E3097F885
:106030003E2026491346DB009B1A9B000B44354A41
:106040001A6097F83E2021491346DB009B1A9B00FB
:106050000B4469221A7197F83E201346DB009B1A05
:106060009B001A4A1344053318462B49132233F078
:10607000F6FD97F83E30013387F83E3097F83E2022
:1060800012491346DB009B1A9B000B44234A1A60FB
:1060900097F83E200D491346DB009B1A9B000B44EA
:1060A00069221A7197F83E201346DB009B1A9B0069
:1060B000064A1344053318461949132233F0CFFD1D
:1060C00097F83E30013387F83E302BE0182E001051
:1060D00024690400CC210010306904003C690400EC
:1060E0004C6904002627001058690400410900107B
:1060F0006869040042090010746904004409001032
:106100008069040046090010906904002509001008
:106110009869040026090010A46904005A090010B7
:10612000B069040097F83E20DB491346DB009B1A58
:106130009B000B44D94A1A6097F83E20D649134673
:10614000DB009B1A9B000B446D221A7197F83E20CE
:106150001346DB009B1A9B00CF4A134405331846B5
:10616000CF49132233F07BFD97F83E30013387F897
:106170003E3097F83E20C8491346DB009B1A9B002F
:106180000B44C84A1A6097F83E20C3491346DB0007
:106190009B1A9B000B446D221A7197F83E20134600
:1061A000DB009B1A9B00BC4A134405331846BE49CA
:1061B000132233F054FD97F83E30013387F83E3018
:1061C00097F83E20B4491346DB009B1A9B000B4412
:1061D00000221A6097F83E20AF491346DB009B1A55
:1061E0009B000B4477221A7197F83E201346DB0080
:1061F0009B1A9B00A84A134405331846AB49132247
:1062000033F02DFD97F83E30013387F83E3097F894
:106210003E20A1491346DB009B1A9B000B44A44A75
:106220001A6097F83E209C491346DB009B1A9B009E
:106230000B446D221A7197F83E201346DB009B1A1F
:106240009B00954A1344053318469A49132233F0AC
:1062500006FD97F83E30013387F83E3097F83E2030
:106260008D491346DB009B1A9B000B44924A1A602F
:1062700097F83E2088491346DB009B1A9B000B448D
:106280006D221A7197F83E201346DB009B1A9B0083
:10629000814A1344053318468849132233F0DFFC42
:1062A00097F83E30013387F83E3097F83E207A4920
:1062B0001346DB009B1A9B000B44814A1A6097F837
:1062C0003E2075491346DB009B1A9B000B446D2250
:1062D0001A7197F83E201346DB009B1A9B006E4A0A
:1062E0001344053318467749132233F0B8FC97F866
:1062F0003E30013387F83E3097F83E20664913461A
:10630000DB009B1A9B000B446F4A1A6097F83E20F3
:1063100061491346DB009B1A9B000B4469221A71EA
:1063200097F83E201346DB009B1A9B005A4A134401
:10633000053318466549132233F091FC97F83E3037
:10634000013387F83E3097F83E2053491346DB006F
:106350009B1A9B000B445E4A1A6097F83E204E49F8
:106360001346DB009B1A9B000B446D221A7197F8B1
:106370003E201346DB009B1A9B00474A134405331B
:1063800018465449132233F06AFC97F83E30013323
:1063900087F83E3097F83E203F491346DB009B1AB2
:1063A0009B000B444C4A1A6097F83E203A4913462A
:1063B000DB009B1A9B000B446D221A7197F83E205C
:1063C0001346DB009B1A9B00334A134405331846DF
:1063D0004249132233F043FC97F83E30013387F8EB
:1063E0003E3097F83E202C491346DB009B1A9B0059
:1063F0000B443B4A1A6097F83E2027491346DB00BE
:106400009B1A9B000B446D221A7197F83E2013468D
:10641000DB009B1A9B00204A134405331846314980
:10642000132233F01CFC97F83E30013387F83E30DE
:1064300097F83E2018491346DB009B1A9B000B443B
:10644000294A1A6097F83E2013491346DB009B1A2D
:106450009B000B446D221A7197F83E201346DB0017
:106460009B1A9B000C4A1344053318461F491322FC
:1064700033F0F5FB97F83E30013387F83E3097F85C
:106480003E2005491346DB009B1A9B000B44184A2B
:106490001A6097F83E202DE0182E00101809001001
:1064A000BC69040052090010CC690400D8690400DA
:1064B00038090010E069040036090010F069040092
:1064C0003A090010006A04003C090010106A040038
:1064D00030090010206A040032090010306A0400FC
:1064E00034090010406A0400BE080010506A04001D
:1064F00054090010DD491346DB009B1A9B000B4436
:106500006D221A7197F83E201346DB009B1A9B0000
:10651000D64A134405331846D549132233F09FFB5E
:1065200097F83E30013387F83E3097F83E20CF4948
:106530001346DB009B1A9B000B44CE4A1A6097F867
:106540003E20CA491346DB009B1A9B000B446D2278
:106550001A7197F83E201346DB009B1A9B00C34A32
:10656000134405331846C449132233F078FB97F8D7
:106570003E30013387F83E3097F83E20BB49134642
:10658000DB009B1A9B000B4400221A6097F83E2008
:10659000B6491346DB009B1A9B000B4477221A7105
:1065A00097F83E201346DB009B1A9B00AF4A13442A
:1065B00005331846B149132233F051FB97F83E30AA
:1065C000013387F83E3097F83E20A8491346DB0098
:1065D0009B1A9B000B44AA4A1A6097F83E20A349D5
:1065E0001346DB009B1A9B000B4469221A7197F833
:1065F0003E201346DB009B1A9B009C4A1344053344
:106600001846A049132233F02AFB97F83E30013395
:1066100087F83E3097F83E2094491346DB009B1ADA
:106620009B000B44984A1A6097F83E208F49134606
:10663000DB009B1A9B000B4469221A7197F83E20DD
:106640001346DB009B1A9B00884A13440533184607
:106650008E49132233F003FB97F83E30013387F85D
:106660003E3097F83E2081491346DB009B1A9B0081
:106670000B44874A1A6097F83E207C491346DB009A
:106680009B1A9B000B4469221A7197F83E2013460F
:10669000DB009B1A9B00754A1344053318467D495D
:1066A000132233F0DCFA97F83E30013387F83E309E
:1066B00097F83E206D491346DB009B1A9B000B4464
:1066C00000221A6097F83E2068491346DB009B1AA7
:1066D0009B000B4477221A7197F83E201346DB008B
:1066E0009B1A9B00614A1344053318466A490522E8
:1066F00033F0B5FA97F83E30013387F83E3097F81B
:106700003E205A491346DB009B1A9B000B44634A08
:106710001A6097F83E2055491346DB009B1A9B00F0
:106720000B446D221A7197F83E201346DB009B1A2A
:106730009B004E4A1344053318465949052233F04D
:106740008EFA97F83E30013387F83E3097F83E20B6
:1067500046491346DB009B1A9B000B44514A1A60C2
:1067600097F83E2041491346DB009B1A9B000B44DF
:106770006D221A7197F83E201346DB009B1A9B008E
:106780003A4A1344053318464749052233F067FA5D
:1067900097F83E30013387F83E3097F83E20334972
:1067A0001346DB009B1A9B000B4400221A6097F8EB
:1067B0003E202E491346DB009B1A9B000B44772298
:1067C0001A7197F83E201346DB009B1A9B00274A5C
:1067D0001344053318463549132233F040FA97F82D
:1067E0003E30013387F83E3097F83E201F4913466C
:1067F000DB009B1A9B000B4400221A6097F83E2096
:106800001A491346DB009B1A9B000B4477221A712E
:1068100097F83E201346DB009B1A9B00134A134453
:10682000053318462249132233F019FA97F83E30FF
:10683000013387F83E3097F83E200C491346DB00C1
:106840009B1A9B000B4400221A6097F83E200749D0
:106850001346DB009B1A9B000B4477221A7197F8B2
:106860003E201346DB009B1A9B0023E0182E0010ED
:106870005C6A04001C090010706A04007C6A040051
:10688000400900108C6A0400120A00109C6A04007F
:10689000130A0010AC6A0400BC6A04005609001018
:1068A000C46A04003E090010CC6A0400D46A0400E3
:1068B000E06A0400DF4A134405331846DE49132218
:1068C00033F0CDF997F83E30013387F83E3097F832
:1068D0003E20D8491346DB009B1A9B000B44002244
:1068E0001A6097F83E20D3491346DB009B1A9B00A1
:1068F0000B4477221A7197F83E201346DB009B1A4F
:106900009B00CC4A134405331846CC49132233F07C
:10691000A6F997F83E30013387F83E3097F83E20CD
:10692000C4491346DB009B1A9B000B4400221A60EB
:1069300097F83E20BF491346DB009B1A9B000B448F
:1069400077221A7197F83E201346DB009B1A9B00B2
:10695000B84A134405331846B949132233F07FF976
:1069600097F83E30013387F83E3097F83E20B14922
:106970001346DB009B1A9B000B4400221A6097F819
:106980003E20AC491346DB009B1A9B000B44772248
:106990001A7197F83E201346DB009B1A9B00A54A0C
:1069A000134405331846A749132233F058F997F8D2
:1069B0003E30013387F83E3097F83E209D4913461C
:1069C000DB009B1A9B000B4400221A6097F83E20C4
:1069D00098491346DB009B1A9B000B4477221A71DF
:1069E00097F83E201346DB009B1A9B00914A134404
:1069F000053318469449132233F031F997F83E30A5
:106A0000013387F83E3097F83E208A491346DB0071
:106A10009B1A9B000B4400221A6097F83E20854980
:106A20001346DB009B1A9B000B4477221A7197F8E0
:106A30003E201346DB009B1A9B007E4A134405331D
:106A400018468249132233F00AF997F83E30013391
:106A500087F83E3097F83E2076491346DB009B1AB4
:106A60009B000B4400221A6097F83E2071491346A0
:106A7000DB009B1A9B000B4477221A7197F83E208B
:106A80001346DB009B1A9B006A4A134405331846E1
:106A90006F49132233F0E3F897F83E30013387F85B
:106AA0003E3097F83E2063491346DB009B1A9B005B
:106AB0000B4400221A6097F83E205E491346DB0023
:106AC0009B1A9B000B4477221A7197F83E201346BD
:106AD000DB009B1A9B00574A1344053318465D4957
:106AE000132233F0BCF897F83E30013387F83E307C
:106AF00097F83E204F491346DB009B1A9B000B443E
:106B0000554A1A6097F83E204A491346DB009B1A03
:106B10009B000B446D221A7197F83E201346DB0050
:106B20009B1A9B00434A1344053318464B491322D2
:106B300033F095F897F83E30013387F83E3097F8F8
:106B40003E203C491346DB009B1A9B000B44444A01
:106B50001A6097F83E2037491346DB009B1A9B00CA
:106B60000B4469221A7197F83E201346DB009B1AEA
:106B70009B00304A1344053318463A49132233F038
:106B80006EF897F83E30013387F83E3097F83E2094
:106B900028491346DB009B1A9B000B44324A1A60BB
:106BA00097F83E2023491346DB009B1A9B000B44B9
:106BB00069221A7197F83E201346DB009B1A9B004E
:106BC0001C4A1344053318462849132233F047F86A
:106BD00097F83E30013387F83E3097F83E2015494C
:106BE0001346DB009B1A9B000B4400221A6097F8A7
:106BF0003E2010491346DB009B1A9B000B44772272
:106C00001A7197F83E201346DB009B1A9B00094A35
:106C10001344053318461649132233F020F897F829
:106C20003E30013387F83E3097F83E200149134645
:106C3000DB001FE0182E0010EC6A0400F86A040064
:106C4000046B0400106B04001C6B0400286B040030
:106C5000346B0400406B0400B6080010506B040055
:106C6000BA0800105C6B0400BB080010686B0400DD
:106C7000746B04009B1A9B000B445F4A1A6097F8E0
:106C80003E205E491346DB009B1A9B000B446D229D
:106C90001A7197F83E201346DB009B1A9B00574A57
:106CA0001344053318465649052232F0D8FF97F8A9
:106CB0003E30013387F83E3097F83E204F49134667
:106CC000DB009B1A9B000B4400221A6097F83E20C1
:106CD0004A491346DB009B1A9B000B4477221A712A
:106CE00097F83E201346DB009B1A9B00434A13444F
:106CF000053318464349052232F0B1FF97F83E307C
:106D0000013387F83E3097F83E203C491346DB00BC
:106D10009B1A9B000B4400221A6097F83E203749CB
:106D20001346DB009B1A9B000B4477221A7197F8DD
:106D30003E201346DB009B1A9B00304A1344053368
:106D400018463149052232F08AFF97F83E30013368
:106D500087F83E3097F83E2028491346DB009B1AFF
:106D60009B000B44294A1A6097F83E20234913469A
:106D7000DB009B1A9B000B4469221A7197F83E2096
:106D80001346DB009B1A9B001C4A1344053318462C
:106D90001F49052232F063FF97F83E30013387F830
:106DA0003E3097F83E2015491346DB009B1A9B00A6
:106DB0000B44184A1A6097F83E2010491346DB002E
:106DC0009B1A9B000B446D221A7197F83E201346C4
:106DD000DB009B1A9B00094A1344053318460E49F1
:106DE000052232F03CFF97F83E30013387F83E3001
:106DF0004037BD4680BD00BF20270010182E001070
:106E0000806B0400886B0400906B04001109001073
:106E1000986B04000E090010A06B040090B597B0A9
:106E200000AF0346FB710023A7F856300023A7F8F4
:106E30005430002387F85330002387F85230B94B81
:106E40001B7A012B40F096820023A7F85630B64BF0
:106E50001B78002B0ED1B7F856305A1CA7F85620D5
:106E60001A46B24B7B219954AF4B01221A70B04B9A
:106E700000221A80002387F852303FE2002387F86F
:106E80005330B7F856305A1CA7F856201A46A74B6D
:106E9000222199541DE0B7F856305A1CA7F8562005
:106EA0001846A34B1B88194697F853305A1C87F88D
:106EB00053201C469F4A0B46DB005B1A9B00234471
:106EC00013445A79994B1A5497F85330132B00D91D
:106ED0000EE0974B1B88184697F8532095490346B8
:106EE000DB001B1A9B0013440B445B79002BD2D1AF
:106EF000B7F856305A1CA7F856201A468B4B222159
:106F00009954B7F856305A1CA7F856201A46874BA2
:106F10003A219954864B1B881946864A0B46DB005A
:106F20005B1A9B0013441B795BB2692B12D1804B17
:106F30001B8819467F4A0B46DB005B1A9B001344F3
:106F40001B681B781A4607F10C03104619460A22E3
:106F500032F04AFC764B1B881946764A0B46DB001A
:106F60005B1A9B0013441B795BB26D2B14D1704BE1
:106F70001B8819466F4A0B46DB005B1A9B001344C3
:106F80001B68FB64FB6C1B881AB207F10C031046EC
:106F900019460A2232F028FC654B1B881946654ABF
:106FA0000B46DB005B1A9B0013441B795BB26C2B16
:106FB00013D15F4B1B8819465E4A0B46DB005B1AF8
:106FC0009B0013441B68BB64BB6C1A6807F10C037D
:106FD000104619460A2232F007FC554B1B88194609
:106FE000544A0B46DB005B1A9B0013441B795BB2CF
:106FF000662B17D14E4B1B8819464E4A0B46DB00B9
:107000005B1A9B0013441B687B647B6C1B681846EF
:1070100033F0EAFE024607F10C03104619460A2235
:1070200032F0E2FB424B1B881946424A0B46DB001A
:107030005B1A9B0013441B795BB2772B27D100238B
:10704000A7F854300023A7F854300CE0B7F85430B8
:1070500007F158021344002203F84C2CB7F85430BF
:107060000133A7F85430B7F85430312BEED9304BF8
:107070001B881A461346DB009B1A9B002D4A1344BB
:107080005A1D07F10C031046194600F0B9FD284BB4
:107090001B881946274A0B46DB005B1A9B001344EA
:1070A0001B795BB2632B53D1214B1B881946214AB4
:1070B0000B46DB005B1A9B0013441B683B640023F8
:1070C000A7F854300023A7F854300CE0B7F8543038
:1070D00007F158021344002203F84C2CB7F854303F
:1070E0000133A7F85430B7F85430312BEED90023D0
:1070F000A7F8543020E0B7F85430B7F85420396C72
:107100000A441278D2B207F158010B4403F84C2C10
:10711000B7F854300133A7F85430B7F85430142B73
:107120000AD910E02C220010C0000010B42D00106D
:10713000C2000010182E0010B7F854303A6C1344F7
:107140001B78002BD7D107F10C03184630F0E8F973
:107150008A4B1B8819468A4A0B46DB005B1A9B0048
:1071600013441B795BB2732B44D1844B1B881946A3
:10717000834A0B46DB005B1A9B0013441B683B648D
:107180000023A7F854300023A7F854300CE0B7F8D8
:10719000543007F158021344002203F84C2CB7F87E
:1071A00054300133A7F85430B7F85430312BEED9AE
:1071B0000023A7F8543016E0B7F85430B7F854203D
:1071C000396C0A441278D2B207F158010B4403F823
:1071D0004C2CB7F854300133A7F85430B7F854307A
:1071E000142B00D906E0B7F854303A6C13441B78DE
:1071F000002BE1D1002387F85330B7F856305A1CE2
:10720000A7F856201A465F4B2221995416E0B7F88A
:1072100056305A1CA7F856201A4697F85330591C76
:1072200087F8531007F158010B4413F84C1C554BC9
:10723000995497F85330312B00D908E097F8533020
:1072400007F15802134413F84C3C002BDFD1B7F878
:1072500056305A1CA7F856201A464A4B22219954F8
:10726000464B1B885A1C46491346DB009B1A9B0061
:107270000B445B79002B08D0B7F856305A1CA7F89E
:1072800056201A463F4B2C219954B7F8563000200F
:107290003C491A4632F08EF90023A7F85630374B96
:1072A0001B88632B06D9354B00221A80364B0222ED
:1072B0001A7030E0314B1B885A1C31491346DB00F1
:1072C0009B1A9B000B445B79002B06D12B4B0022B1
:1072D0001A802D4B02221A701DE0284B1B880133A7
:1072E0009AB2264B1A8097F85230013387F8523001
:1072F00097F85220FB799A4200D10CE01F4B1B8873
:1073000019461F4A0B46DB005B1A9B0013445B794E
:10731000002B7FF4B3AD1C4B1B78022B2AD1B7F89E
:1073200056305A1CA7F856201A46164B7D21995400
:10733000B7F856305A1CA7F856201A46114B0D21A3
:107340009954B7F856305A1CA7F856201A460D4BD8
:107350000A219954B7F8563000200A491A4632F0EB
:1073600029F90023A7F85630074B00221A70074B63
:1073700000221A725C37BD4690BD00BFC2000010EB
:10738000182E0010B42D0010C00000102C22001088
:1073900090B585B000AF786039600023FB600023B2
:1073A000FB720023FB606AE1FB687A6813441A7879
:1073B000974B1A70964B1B785BB2184632F0A8F9BF
:1073C0000346002B00D057E1924B1B68072B00F2BD
:1073D000488101A252F823F0F973000023740000E1
:1073E00073740000C7740000637600000975000024
:1073F0006B75000039760000854B1B785BB27B2BE8
:107400000ED1854B00225A77824B01221A60834BA2
:1074100000221A60824B1B680133814A13602BE102
:107420001FE17B4B1B785BB2222B05D17D4B0022E9
:107430001A60784B02221A60754B1B785BB27D2B69
:1074400016D1774B1B68013B754A1360744B1B6860
:10745000002B05D1704B01225A776E4B00221A6027
:107460006F4B1B68002B03DD6A4B07221A60F8E0A4
:10747000F7E0674B1B785BB2222B18D1694B1B6876
:10748000694A0021D154654B1B68462202FB03F375
:10749000664A9C18644832F093FB034620466249D2
:1074A0001A4632F0DCFB5B4B03221A60D9E05D4BDD
:1074B0001B68574A11785C4AD1545A4B1B680133F8
:1074C000584A1360CDE0524B1B785BB23A2B03D184
:1074D000574B00221A60CFE04D4B1B785BB2222B3A
:1074E00003D14C4B05221A60BBE04A4B06221A60BE
:1074F0004F4B1B68464A11784E4AD1544C4B1B687F
:1075000001334B4A1360ACE0414B1B785BB2222B3A
:107510001FD1474B1B68474A0021D1543F4B1B6882
:10752000462202FB03F31033404A13441C1D41481A
:1075300032F046FB034620463E491A4632F08FFBA6
:10754000364B1B680133354A1360324B01221A60F7
:1075500087E0374B1B682E4A1178364AD154344B9A
:107560001B680133324A13607BE0294B1B785BB206
:107570002C2B04D0264B1B785BB27D2B3BD12C4BA4
:107580001B682C4A0021D154244B1B68462202FB65
:1075900003F31033254A134404331846254932F0C7
:1075A000EFFA1E4B1B6801331C4A1360184B1B7803
:1075B0005BB22C2B02D1174B01221A60144B1B78A3
:1075C0005BB27D2B16D1164B1B68013B144A13602E
:1075D000134B1B68002B05D10F4B01225A770D4B23
:1075E00000221A600E4B1B68002B03DD094B0122A1
:1075F0001A600CE00BE00E4B1B68054A11780D4A2F
:10760000D1540B4B1B680133094A136029E028E071
:10761000C4000010C8000010A0270010CC0000100B
:10762000D0000010D4000010D80000103C2800103A
:10763000F8000010FC000010154B1B785BB27D2B8E
:107640000ED1144B1B68013B124A1360114B1B688F
:10765000002B05D1104B01225A77104B00221A60E3
:1076600000BF0F4B1B68122B06DD0D4B00221A606A
:107670000A4B00221A6007E0FB680133FB60FA68DE
:107680003B689A42FFF690AE1437BD4690BD00BFEE
:10769000C4000010D0000010A0270010C800001087
:1076A000CC00001080B588B000AF78600023FB7775
:1076B000B24B9B78022B0FD1B14B93F81632082BAB
:1076C0000AD17B684D221A707B6801334F221A70F1
:1076D0007B68023344221A70A84B9B78022B0FD18F
:1076E000A74B93F81632072B0AD17B6850221A70E9
:1076F0007B68013352221A707B68023341221A7070
:107700009E4B9B78002B0AD17B6853221A707B68B2
:10771000013354221A707B6802334F221A70974B40
:107720009B78052B0AD17B6843221A707B68013352
:107730005A221A707B68023355221A708F4B9B783D
:10774000012B0AD17B6852221A707B6801334F22C9
:107750001A707B6802335A221A70884B9B78032B6D
:107760000AD17B6857221A707B68013359221A703C
:107770007B68023347221A70804B9B78042B0AD116
:107780007B684F221A707B68013346221A707B682F
:10779000023346221A70794B9B78082B0AD17B68FA
:1077A0004B221A707B6801334F221A707B680233B8
:1077B0004E221A70714B9B78072B0AD17B6850229E
:1077C0001A707B68013341221A707B68023355229C
:1077D0001A700023FB7709E0FB7F07F120021344B6
:1077E000002203F8182CFB7F0133FB77FB7F132B60
:1077F000F2D9624B1B891A4607F108031046194655
:107800000A2231F0F1FF07F10803184632F0D8F9E7
:107810000346012B05D13B7ABB7230233B723023E8
:107820007B7207F10803184632F0CAF90346022BAF
:1078300005D17B7ABB723B7A7B7230233B727B68CB
:1078400003333A7A1A707B6804337A7A1A707B6849
:107850000533BA7A1A700023FB7709E0FB7F07F142
:1078600020021344002203F8182CFB7F0133FB771E
:10787000FB7F132BF2D9434B5A6807F108031046DC
:1078800019460A2231F0B0FF07F10803184632F01A
:1078900097F90346012B05D13B7ABB7230233B722B
:1078A00030237B7207F10803184632F089F903464A
:1078B000022B05D17B7ABB723B7A7B7230233B7201
:1078C0007B6806333A7A1A707B6807337A7A1A70C3
:1078D0007B680833BA7A1A702B4BDA792A4B5B7CB7
:1078E0001343DBB2002B04D07B68093331221A70BA
:1078F00003E07B68093330221A70234B1A78224B3D
:107900009B7A1343DBB2002B04D07B680A3331220D
:107910001A7003E07B680A3330221A701A4B5A78C7
:10792000194BDB7A1343DBB2002B04D07B680B339B
:1079300031221A7003E07B680B3330221A70124B2D
:107940009A78114B1B7B1343DBB2002B04D07B686E
:107950000C3331221A7003E07B680C3330221A702A
:10796000094BDA78084B5B7B1343DBB2002B0DD05D
:107970007B680D3331221A700CE000BF2027001005
:107980000407001040220010300A00107B680D33FD
:1079900030221A707B680E3300221A702037BD46E1
:1079A00080BD00BF80B483B000AF7860924B5B7B3A
:1079B000002B03D07B6841221A7002E07B683022E2
:1079C0001A708D4B9B7A002B04D07B6801334222C6
:1079D0001A7003E07B68013330221A70864B1B7BE0
:1079E000002B04D07B68023343221A7003E07B68CB
:1079F000023330221A70804B1B79002B04D07B6835
:107A0000033344221A7003E07B68033330221A7078
:107A1000794BDB78002B04D07B68043345221A7045
:107A200003E07B68043330221A70734B9B78002B81
:107A300004D07B68053346221A7003E07B68053367
:107A400030221A706C4BDB79002B04D07B68063334
:107A500047221A7003E07B68063330221A70664BA7
:107A60009B79002B04D07B68073348221A7003E00F
:107A70007B68073330221A70604BDB7F002B04D009
:107A80007B68083349221A7003E07B680833302290
:107A90001A705A4B9B7F002B04D07B6809334A2213
:107AA0001A7003E07B68093330221A70534B5B7FF6
:107AB000002B04D07B680A334B221A7003E07B68EA
:107AC0000A3330221A704D4BDB7E002B04D07B68CA
:107AD0000B334C221A7003E07B680B3330221A7090
:107AE000464B1B7F002B04D07B680C334D221A7051
:107AF00003E07B680C3330221A70404B1B7E002B56
:107B000004D07B680D334E221A7003E07B680D337E
:107B100030221A70384B5B79002B04D07B680E330F
:107B20004F221A7003E07B680E3330221A70324BFA
:107B30005B7A002B04D07B680F3350221A7003E06D
:107B40007B680F3330221A702B4B9B7B002B04D0A9
:107B50007B68103352221A7003E07B6810333022A6
:107B60001A70254BDB7B002B04D07B68113353222A
:107B70001A7003E07B68113330221A701E4BDB7AD7
:107B8000002B04D07B68123354221A7003E07B6808
:107B9000123330221A70184B9B7C002B04D07B6868
:107BA000133355221A7003E07B68133330221A70A6
:107BB000114B1B7C002B04D07B68143357221A70A6
:107BC00003E07B68143330221A700B4B5B7C002B74
:107BD00004D07B68153358221A7003E07B68143395
:107BE00030221A707B68163300221A700C37BD469B
:107BF0005DF8047B704700BF140A0010C421001018
:107C000080B584B000AF786039607868B3490722E6
:107C100031F0FBFF0346002B02D1386830F080F9C9
:107C20007868AF49092231F0F0FF0346002B04D1F8
:107C30003868AC490A2232F012F87868AA49092259
:107C400031F0E3FF0346002B0BD13868012108F027
:107C5000BBF83B6802332D221A703B6805332D2296
:107C60001A707868A149052231F0CFFF0346002B36
:107C70000BD19F4B1B68FB60FB68184639680A22D2
:107C800031F0B2FD38682FF04BFC78689949092231
:107C900031F0BBFF0346002B02D13868FFF702FD2D
:107CA00078689549062231F0B0FF0346002B02D1D7
:107CB0003868FFF777FE78689049072231F0A5FF12
:107CC0000346002B27D18E4B93F81731012B04D19B
:107CD00038688C49132231F0C2FF894B93F8173171
:107CE000022B04D138688849132231F0B8FF844B45
:107CF00093F81731002B04D138688449132231F0EE
:107D0000AEFF7F4B93F81731032B04D138688049BD
:107D1000132231F0A4FF78687E490B2231F075FF01
:107D20000346002B13D1764B93F81631012B04D167
:107D300038687949132231F092FF714B93F816316C
:107D4000002B04D138687549132231F088FF786818
:107D500073490C2231F059FF0346002B11D1684BB7
:107D60001B7D012B04D138686B49132231F077FF5A
:107D7000634B1B7D002B04D138686849132231F016
:107D80006EFF78686749102231F03FFF0346002BF1
:107D900014D15B4B93F882305BB2012B04D138686D
:107DA0005D49132231F05BFF554B93F88230002B75
:107DB00004D138685949132231F051FF78685A4983
:107DC000072231F022FF0346002B13D14C4B93F8CE
:107DD0002930012B04D138685449132231F03FFF78
:107DE000474B93F82930002B04D1386847491322B8
:107DF00031F035FF78684E490B2231F006FF03461B
:107E0000002B23D13E4B9B7A012B04D13868494982
:107E1000132231F024FF3A4B9B7A022B04D13868AD
:107E20004549132231F01BFF354B9B7A032B04D1BC
:107E300038683549132231F012FF314B9B7A002B01
:107E400004D138683549132231F009FF78683B497D
:107E5000072231F0DAFE0346002B1DD1284B93F8A0
:107E6000AF30012B04D138683049132231F0F7FECE
:107E7000234B93F8AF30002B04D1386823491322E9
:107E800031F0EDFE1E4B93F8AF30022B04D1386871
:107E90001D49132231F0E3FE786829490B2231F0A5
:107EA000B4FE0346002B0FD1264BDB68184626494B
:107EB00032F006FE0346184632F096FF0346184697
:107EC00039680A2231F090FC78682049092231F0A3
:107ED0009CFE0346002B4BD13AE000BFB86B040078
:107EE000C06B0400CC6B0400D86B0400E46B04008E
:107EF0002C220010EC6B0400F86B0400006C0400F2
:107F000004070010086C0400146C04001C6C0400CE
:107F1000246C0400346C0400406C0400446C0400C5
:107F20004C6C04005C6C0400706C0400786C040001
:107F3000806C04008C6C0400986C0400A46C040039
:107F4000AC6C0400202700100000C842B86C04008C
:107F50009E4B1B6918469E4932F0B2FD03461846F7
:107F600032F042FF0346184639680A2231F03CFCE1
:107F7000786898490A2231F048FE0346002B04D164
:107F800038689549032231F06AFE786893490622E1
:107F900031F03BFE0346002B13D1914B93F8163280
:107FA000082B04D138688F49132231F058FE8C4BCE
:107FB00093F81632072B04D138688B49132231F01D
:107FC0004EFE786889490B2231F01FFE0346002BD4
:107FD00010D1834BD3F81C3218467D4932F070FD26
:107FE0000346184632F000FF0346184639680A2255
:107FF00031F0FAFB78687E49042231F006FE034630
:10800000002B0FD17B4B9B6B18467B4932F058FD00
:108010000346184632F0E8FE0346184639680A223D
:1080200010F082FB78687549072231F0EEFD0346B7
:10803000002B02D138682FF073FF7868704908224E
:1080400031F0E3FD0346002B02D138682FF0B6FF74
:1080500078686C49072231F0D8FD0346002B02D125
:10806000386830F0B1F878686749082231F0CDFD02
:108070000346002B02D1386830F0F4F87868634981
:10808000082231F0C2FD0346002B02D1386830F0DF
:10809000EFF978685E49092231F0B7FD0346002BFD
:1080A00002D1386830F032FA78685A49072231F044
:1080B000ACFD0346002B02D1386830F037FB7868FE
:1080C0005549082231F0A1FD0346002B02D1386842
:1080D00030F07AFB78685149082231F096FD03466A
:1080E000002B1DD13E4B93F8B031012B04D13868E1
:1080F0004B49132231F0B3FD394B93F8B031002BCB
:1081000004D138684749132231F0A9FD344B93F864
:10811000B031022B04D138684349132231F09FFD5E
:10812000786842490C2231F070FD0346002B13D1D0
:108130002B4B93F8B431012B04D138683C491322FE
:1081400031F08DFD264B93F8B431002B04D1386803
:108150003849132231F083FD78683749072231F01E
:1081600054FD0346002B09D1344831F029FD034664
:108170000133386831491A4631F071FD7868304969
:10818000062231F042FD0346002B05D10F4B9B6DBB
:10819000184639682FF0AEF878682A49042231F081
:1081A00034FD0346002B02D1386830F0A1FC78681A
:1081B0002549042231F029FD0346002B02D13868FD
:1081C00030F0E4FC1037BD4680BD00BF2027001012
:1081D0000000C842C46C040014090010D06C0400F4
:1081E00004070010D86C0400E06C0400EC6C040080
:1081F000BC6A04001C1E001000002041B86B040083
:10820000F86C0400046D0400106D04001C6D040083
:10821000286D0400346D04003C6D0400486D0400BA
:10822000786C04001C6C0400146C0400546D040091
:10823000406C0400446C0400646D04006C6D040028
:10824000886D0400886B0400906B040080B483B0D8
:1082500000AF0023FB800023FB8006E0FB88084A78
:108260000021D154FB880133FB80FB8840F6B732F4
:108270009342F3D90C37BD465DF8047B704700BFCD
:10828000E84E001080B483B000AF0023FB710023E0
:10829000BB710023FB712AE00023BB710DE0FA796A
:1082A000B97917481346DB009B1ADB000B440344E3
:1082B00000221A70BB790133BB71BB79052BEED953
:1082C0000023BB710DE0FA79B9790D481346DB0044
:1082D0009B1ADB000B44034400229A71BB790133E3
:1082E000BB71BB79312BEED9FB790133FB71FB7983
:1082F000312BD1D90C37BD465DF8047B704700BFE8
:10830000F843001080B483B000AF0023FB7100235A
:10831000BB710023FB712AE00023BB710DE0FA79E9
:10832000B97917481346DB009B1ADB000B44034462
:1083300000221A70BB790133BB71BB79052BEED9D2
:108340000023BB710DE0FA79B9790D481346DB00C3
:108350009B1ADB000B44034400229A71BB79013362
:10836000BB71BB79312BEED9FB790133FB71FB7902
:10837000312BD1D90C37BD465DF8047B704700BF67
:108380000839001090B591B000AF7860002387F8ED
:108390003F307868E949062231F037FC0346002B6C
:1083A00040F0608197F83F201346DB009B1ADB000A
:1083B000E34A13441846E349052231F050FC07F123
:1083C0000C03184630F094FB97F83F201346DB006F
:1083D0009B1ADB00DA4A13449C1D07F10C03184674
:1083E00031F0EEFB0346013307F10C022046114643
:1083F0001A4631F034FC97F83F30013387F83F30AC
:1084000097F83F201346DB009B1ADB00CC4A13444D
:108410001846CD49052231F022FC07F10C0318461D
:1084200030F0B4FB97F83F201346DB009B1ADB00CB
:10843000C34A13449C1D07F10C03184631F0C0FBDE
:108440000346013307F10C02204611461A4631F06B
:1084500006FC97F83F30013387F83F3097F83F200C
:108460001346DB009B1ADB00B54A13441846B74994
:10847000052231F0F4FBB64B93F80D321A4607F1A2
:108480000C03104619460A2231F0AEF997F83F2046
:108490001346DB009B1ADB00A94A13449C1D07F11D
:1084A0000C03184631F08CFB0346013307F10C0234
:1084B000204611461A4631F0D2FB97F83F3001337F
:1084C00087F83F3097F83F201346DB009B1ADB000C
:1084D0009B4A134418469F49052231F0C0FB9C4B30
:1084E000B3F80A321AB207F10C03104619460A22F1
:1084F00031F07AF997F83F201346DB009B1ADB0036
:108500008F4A13449C1D07F10C03184631F058FBA9
:108510000346013307F10C02204611461A4631F09A
:108520009EFB97F83F30013387F83F3097F83F20A4
:108530001346DB009B1ADB00814A13441846864928
:10854000052231F08CFB824BB3F80E321AB207F1E0
:108550000C03104619460A2231F046F997F83F20DD
:108560001346DB009B1ADB00754A13449C1D07F180
:108570000C03184631F024FB0346013307F10C02CB
:10858000204611461A4631F06AFB97F83F30013316
:1085900087F83F3097F83F201346DB009B1ADB003B
:1085A000674A134418466D49052231F058FB684B61
:1085B000B3F8B8311AB207F10C03104619460A2273
:1085C00031F012F997F83F201346DB009B1ADB00CD
:1085D0005B4A13449C1D07F10C03184631F0F0FA76
:1085E0000346013307F10C02204611461A4631F0CA
:1085F00036FB97F83F30013387F83F3097F83F203C
:108600001346DB009B1ADB004D4A134418465449BD
:10861000052231F024FB4E4BB3F8BC311AB207F1FE
:108620000C03104619460A2231F0DEF897F83F2075
:108630001346DB009B1ADB00414A13449C1D07F1E3
:108640000C03184631F0BCFA0346013307F10C0263
:10865000204611461A4631F002FB97F83F300133AD
:1086600087F83F3078683F49082231F0CEFA034658
:10867000002B40F0DB81002387F83F3097F83F2044
:108680001346DB009B1ADB002D4A1344184636497B
:10869000052231F0E4FA07F10C03184633490B22A6
:1086A00031F0DDFA97F83F201346DB009B1ADB0020
:1086B000234A13449C1D07F10C03184631F080FA3D
:1086C0000346013307F10C02204611461A4631F0E9
:1086D000C6FA97F83F30013387F83F3097F83F20CC
:1086E0001346DB009B1ADB00154A13441846204949
:1086F000052231F0B4FA07F10C0318461D490A228D
:1087000031F0ADFA97F83F201346DB009B1ADB00EF
:108710000B4A13449C1D07F10C03184631F050FA24
:108720000346013307F10C02204611461A4631F088
:1087300096FA97F83F3001331EE000BF906D0400B9
:10874000F8430010986D0400A06D0400A86D0400AB
:1087500004070010B06D0400B86D0400C06D040083
:10876000C86D0400D06D0400DC6D04008A0900109F
:10877000E46D04009609001087F83F3097F83F2019
:108780001346DB009B1ADB00B14A13441846B1497B
:10879000052231F064FA07F10C031846AE491322A2
:1087A00031F05DFA97F83F201346DB009B1ADB009F
:1087B000A74A13449C1D07F10C03184631F000FA38
:1087C0000346013307F10C02204611461A4631F0E8
:1087D00046FA97F83F30013387F83F3097F83F204B
:1087E0001346DB009B1ADB00994A134418469B4949
:1087F000052231F034FA07F10C0318469849072294
:1088000031F02DFA97F83F201346DB009B1ADB006E
:108810008F4A13449C1D07F10C03184631F0D0F920
:108820000346013307F10C02204611461A4631F087
:1088300016FA97F83F30013387F83F3097F83F201A
:108840001346DB009B1ADB00814A13441846854916
:10885000052231F004FA844B93F8B9321A4607F135
:108860000C03104619460A2230F0BEFF97F83F204D
:108870001346DB009B1ADB00754A13449C1D07F16D
:108880000C03184631F09CF90346013307F10C0242
:10889000204611461A4631F0E2F997F83F3001338D
:1088A00087F83F3097F83F201346DB009B1ADB0028
:1088B000674A134418466D49052231F0D0F907F193
:1088C0000C0318466A49132231F0C9F997F83F2082
:1088D0001346DB009B1ADB005D4A13449C1D07F125
:1088E0000C03184631F06CF90346013307F10C0212
:1088F000204611461A4631F0B2F997F83F3001335D
:1089000087F83F3097F83F201346DB009B1ADB00C7
:108910004F4A134418465749052231F0A0F907F190
:108920000C0318465449132231F099F997F83F2067
:108930001346DB009B1ADB00454A13449C1D07F1DC
:108940000C03184631F03CF90346013307F10C02E1
:10895000204611461A4631F082F997F83F3001332C
:1089600087F83F3097F83F201346DB009B1ADB0067
:10897000374A134418464149052231F070F907F18E
:108980000C0318463E49132231F069F997F83F204D
:108990001346DB009B1ADB002D4A13449C1D07F194
:1089A0000C03184631F00CF90346013307F10C02B1
:1089B000204611461A4631F052F997F83F300133FC
:1089C00087F83F3097F83F201346DB009B1ADB0007
:1089D0001F4A134418462B49052231F040F9224B17
:1089E00093F80A331A4607F10C03104619460A2277
:1089F00030F0FAFE97F83F201346DB009B1ADB00AD
:108A0000134A13449C1D07F10C03184631F0D8F8A3
:108A10000346013307F10C02204611461A4631F095
:108A20001EF997F83F30013387F83F3078681649D0
:108A3000042231F0EAF80346002B5DD1002387F8C9
:108A40003F30002387F83E30002387F83E302AE08D
:108A5000F8430010EC6D0400A2090010F46D04004E
:108A6000B6090010FC6D040004070010046E040039
:108A7000BE0900100C6E0400E6090010146E04001C
:108A8000FA0900101C6E0400246E040097F83E30B2
:108A900007F140021344002203F8342C97F83E30CB
:108AA000013387F83E3097F83E30302BEED997F8F7
:108AB0003F201346DB009B1ADB00EA4A13441846AA
:108AC000E949052231F0CBF897F83F201346DB0047
:108AD0009B1ADB00E34A13449C1DE44831F070F814
:108AE000034603332046E1491A4631F0B8F897F8B7
:108AF0003F30013387F83F307868DD49062231F096
:108B000084F80346002B41F01981002387F83F3099
:108B100097F83F201346DB009B1ADB00D14A134431
:108B20001846D449052231F09AF8D34BB3F81832DD
:108B30001A4607F10C03104619460A2230F054FE7B
:108B400097F83F201346DB009B1ADB00C54A13440D
:108B50009C1D07F10C03184631F032F8034601332F
:108B600007F10C02204611461A4631F078F897F8C2
:108B70003F30013387F83F3097F83F201346DB0042
:108B80009B1ADB00B74A13441846BC49052231F052
:108B900066F8B94B93F84A321A4607F10C031846A7
:108BA000114604F079F897F83F201346DB009B1A32
:108BB000DB00AC4A13449C1D07F10C03184630F04F
:108BC000FFFF0346013307F10C02204611461A4607
:108BD00031F045F897F83F30013387F83F3097F888
:108BE0003F201346DB009B1ADB009E4A13441846C5
:108BF000A349052231F033F89F4BB3F84C321A46A3
:108C000007F10C03104619460A2230F0EDFD97F8E3
:108C10003F201346DB009B1ADB00924A13449C1D45
:108C200007F10C03184630F0CBFF0346013307F180
:108C30000C02204611461A4631F011F897F83F30E1
:108C4000013387F83F3097F83F201346DB009B1A2B
:108C5000DB00844A134418468A49052230F0FFFF9E
:108C6000854BB3F848321A4607F10C0310461946F3
:108C70000A2230F0B9FD97F83F201346DB009B1A1B
:108C8000DB00784A13449C1D07F10C03184630F0B2
:108C900097FF0346013307F10C02204611461A469E
:108CA00030F0DDFF97F83F30013387F83F3097F819
:108CB0003F201346DB009B1ADB006A4A1344184628
:108CC0007149052230F0CBFF6B4B93F83D321A46C9
:108CD00007F10C03104619460A2230F085FD97F87B
:108CE0003F201346DB009B1ADB005E4A13449C1DA9
:108CF00007F10C03184630F063FF0346013307F118
:108D00000C02204611461A4630F0A9FF97F83F3072
:108D1000013387F83F3097F83F201346DB009B1A5A
:108D2000DB00504A134418465849052230F097FF9B
:108D3000514B93F83E321A4607F10C031046194680
:108D40000A2230F051FD97F83F201346DB009B1AB2
:108D5000DB00444A13449C1D07F10C03184630F015
:108D60002FFF0346013307F10C02204611461A4635
:108D700030F075FF97F83F30013387F83F3097F8B0
:108D80003F201346DB009B1ADB00364A134418468B
:108D90003F49052230F063FF374BB3F840321A46A3
:108DA00007F10C03104619460A2230F01DFD97F812
:108DB0003F201346DB009B1ADB002A4A13449C1D0C
:108DC00007F10C03184630F0FBFE0346013307F1B0
:108DD0000C02204611461A4630F041FF97F83F300A
:108DE000013387F83F3097F83F201346DB009B1A8A
:108DF000DB001C4A134418462649052230F02FFF99
:108E00001D4B93F842321A4607F10C0310461946DF
:108E10000A2230F0E9FC97F83F201346DB009B1A4A
:108E2000DB00104A13449C1D07F10C03184630F078
:108E3000C7FE0346013307F10C02204611461A46CD
:108E400030F00DFF97F83F30013387F83F3097F847
:108E50003F201346DB009B1ADB00024A13441846EE
:108E60001AE000BFF84300102C6E0400346E0400BA
:108E7000506E0400586E040004070010606E040079
:108E8000686E0400706E0400786E0400806E04004A
:108E9000886E0400906E0400E449052230F0DFFE85
:108EA000E34BB3F814321A4607F10C031046194687
:108EB0000A2230F099FC97F83F201346DB009B1AFA
:108EC000DB00DC4A13449C1D07F10C03184630F00C
:108ED00077FE0346013307F10C02204611461A467D
:108EE00030F0BDFE97F83F30013387F83F3097F8F8
:108EF0003F201346DB009B1ADB00CE4A1344184682
:108F0000CD49052230F0ABFEC94BB3F84E321AB250
:108F100007F10C03104619460A2230F065FC97F859
:108F20003F201346DB009B1ADB00C24A13449C1D02
:108F300007F10C03184630F043FE0346013307F1F6
:108F40000C02204611461A4630F089FE97F83F3051
:108F5000013387F83F3097F83F201346DB009B1A18
:108F6000DB00B44A13441846B449052230F077FEBA
:108F7000AF4B93F81632082B06D107F10C031846B5
:108F8000AF49132230F06BFEA94B93F81632072B32
:108F900006D107F10C031846AA49132230F05FFEF0
:108FA00097F83F201346DB009B1ADB00A14A1344CD
:108FB0009C1D07F10C03184630F002FE03460133F6
:108FC00007F10C02204611461A4630F048FE97F889
:108FD0003F30013387F83F3097F83F201346DB00DE
:108FE0009B1ADB00934A134418469749052230F038
:108FF00036FE8F4B93F81332012B06D107F10C0389
:10900000184692490A2230F02AFE894B93F813320F
:10901000002B06D107F10C0318468D490A2230F0C7
:109020001EFE97F83F201346DB009B1ADB00814AA7
:1090300013449C1D07F10C03184630F0C1FD034694
:10904000013307F10C02204611461A4630F007FEA4
:1090500097F83F30013387F83F3097F83F201346A9
:10906000DB009B1ADB00734A13441846794905223A
:1090700030F0F5FD6E4B93F821325AB207F10C0334
:10908000104619460A2230F0AFFB97F83F201346EE
:10909000DB009B1ADB00674A13449C1D07F10C039D
:1090A000184630F08DFD0346013307F10C022046CF
:1090B00011461A4630F0D3FD97F83F30013387F858
:1090C0003F3097F83F201346DB009B1ADB00594ADC
:1090D000134418466049052230F0C1FD544B93F803
:1090E00022325AB207F10C03104619460A2230F018
:1090F0007BFB97F83F201346DB009B1ADB004D4AB1
:1091000013449C1D07F10C03184630F059FD03462B
:10911000013307F10C02204611461A4630F09FFD3C
:1091200097F83F30013387F83F3097F83F201346D8
:10913000DB009B1ADB003F4A1344184647490522CF
:1091400030F08DFD3A4B93F823325AB207F10C03FD
:10915000104619460A2230F047FB97F83F20134685
:10916000DB009B1ADB00334A13449C1D07F10C0300
:10917000184630F025FD0346013307F10C02204666
:1091800011461A4630F06BFD97F83F30013387F8EF
:109190003F3097F83F201346DB009B1ADB00254A3F
:1091A000134418462E49052230F059FD204B93F800
:1091B00024325AB207F10C03104619460A2230F045
:1091C00013FB97F83F201346DB009B1ADB00194A7C
:1091D00013449C1D07F10C03184630F0F1FC0346C4
:1091E000013307F10C02204611461A4630F037FDD4
:1091F00097F83F30013387F83F3097F83F20134608
:10920000DB009B1ADB000B4A134418461549052264
:1092100030F025FD064B93F826325AB207F10C03C5
:10922000104619460A2230F0DFFA1DE0986E04005D
:1092300004070010F8430010A06E0400A86E04009C
:10924000B06E0400B86E0400C46E0400CC6E04005E
:10925000D46E0400DC6E0400E46E0400EC6E0400C6
:10926000F46E0400FC6E040097F83F201346DB0008
:109270009B1ADB00E94A13449C1D07F10C031846B6
:1092800030F09EFC0346013307F10C0220461146E4
:109290001A4630F0E4FC97F83F30013387F83F304E
:1092A00097F83F201346DB009B1ADB00DB4A134490
:1092B0001846DB49052230F0D2FCDA4B93F828320D
:1092C0005AB207F10C03104619460A2230F08CFA04
:1092D00097F83F201346DB009B1ADB00CF4A13446C
:1092E0009C1D07F10C03184630F06AFC034601335D
:1092F00007F10C02204611461A4630F0B0FC97F8F0
:109300003F30013387F83F3097F83F201346DB00AA
:109310009B1ADB00C14A13441846C349052230F0AA
:109320009EFCC04B93F82A325AB207F10C03104648
:1093300019460A2230F058FA97F83F201346DB000E
:109340009B1ADB00B54A13449C1D07F10C03184619
:1093500030F036FC0346013307F10C02204611467B
:109360001A4630F07CFC97F83F30013387F83F30E5
:1093700097F83F201346DB009B1ADB00A74A1344F3
:109380001846AA49052230F06AFCA64B93F85632DB
:109390001A4607F10C03104619460A2230F024FA47
:1093A00097F83F201346DB009B1ADB009B4A1344CF
:1093B0009C1D07F10C03184630F002FC03460133F4
:1093C00007F10C02204611461A4630F048FC97F887
:1093D0003F30013387F83F3097F83F201346DB00DA
:1093E0009B1ADB008D4A134418469149052230F040
:1093F00036FC8C4BD3F81C3218468E4931F060FB9A
:109400000346184631F00AFD024607F10C031046E8
:1094100019460A220FF088F997F83F201346DB001F
:109420009B1ADB007D4A13449C1D07F10C03184670
:1094300030F0C6FB0346013307F10C02204611460B
:109440001A4630F00CFC97F83F30013387F83F3074
:1094500097F83F201346DB009B1ADB006F4A13444A
:1094600018467549052230F0FAFB6E4B93F83C32F2
:109470001A4607F10C03104619460A220FF054F958
:1094800097F83F201346DB009B1ADB00634A134426
:109490009C1D07F10C03184630F092FB0346013384
:1094A00007F10C02204611461A4630F0D8FB97F817
:1094B0003F30013387F83F3097F83F201346DB00F9
:1094C0009B1ADB00554A134418465C49052230F0CC
:1094D000C6FB544BB3F834321A4607F10C0310465E
:1094E00019460A220FF020F997F83F201346DB00B7
:1094F0009B1ADB00494A13449C1D07F10C031846D4
:1095000030F05EFB0346013307F10C0220461146A2
:109510001A4630F0A4FB97F83F30013387F83F300C
:1095200097F83F201346DB009B1ADB003B4A1344AD
:1095300018464349052230F092FB3A4BB3F83232D9
:109540001A4607F10C03104619460A220FF0ECF8F0
:1095500097F83F201346DB009B1ADB002F4A134489
:109560009C1D07F10C03184630F02AFB034601331B
:1095700007F10C02204611461A4630F070FB97F8AE
:109580003F30013387F83F3097F83F201346DB0028
:109590009B1ADB00214A134418462A49052230F061
:1095A0005EFB204BB3F836321A4607F10C03104627
:1095B00019460A220FF0B8F897F83F201346DB004F
:1095C0009B1ADB00154A13449C1D07F10C03184637
:1095D00030F0F6FA0346013307F10C02204611463B
:1095E0001A4630F03CFB97F83F30013387F83F30A4
:1095F00097F83F201346DB009B1ADB00074A134411
:1096000018461149052230F02AFB064B93F83832F0
:109610001A4607F10C03104618E000BFF84300108B
:10962000046F0400040700100C6F0400146F0400A2
:109630001C6F040000002041246F04002C6F040004
:10964000346F04003C6F0400446F040019460A2282
:109650000FF06AF897F83F201346DB009B1ADB00F7
:10966000EA4A13449C1D07F10C03184630F0A8FA8F
:109670000346013307F10C02204611461A4630F02A
:10968000EEFA97F83F30013387F83F3097F83F20E4
:109690001346DB009B1ADB00DC4A13441846DC4906
:1096A000052230F0DCFADB4BB3F83A321AB207F19C
:1096B0000C03104619460A220FF036F897F83F209F
:1096C0001346DB009B1ADB00D04A13449C1D07F1B4
:1096D0000C03184630F074FA0346013307F10C020C
:1096E000204611461A4630F0BAFA97F83F30013357
:1096F00087F83F3097F83F201346DB009B1ADB00CA
:10970000C24A13441846C449052230F0A8FAC14B96
:10971000B3F82C321A4607F10C03104619460A22F8
:109720000FF002F897F83F201346DB009B1ADB008E
:10973000B64A13449C1D07F10C03184630F040FA5A
:109740000346013307F10C02204611461A4630F059
:1097500086FA97F83F30013387F83F3097F83F207B
:109760001346DB009B1ADB00A84A13441846AB499A
:10977000052230F074FAA74BB3F82E321A4607F1DF
:109780000C03104619460A220EF0CEFF97F83F2030
:109790001346DB009B1ADB009C4A13449C1D07F117
:1097A0000C03184630F00CFA0346013307F10C02A3
:1097B000204611461A4630F052FA97F83F300133EE
:1097C00087F83F3097F83F201346DB009B1ADB00F9
:1097D0008E4A134418469249052230F040FA8D4BC8
:1097E000B3F830321A4607F10C03104619460A2224
:1097F0000EF09AFF97F83F201346DB009B1ADB0020
:10980000824A13449C1D07F10C03184630F0D8F926
:109810000346013307F10C02204611461A4630F088
:109820001EFA97F83F30013387F83F3097F83F2012
:109830001346DB009B1ADB00744A1344184679492F
:10984000052230F00CFA734BB3F8BA311AB207F1B3
:109850000C03104619460A220EF066FF97F83F20C7
:109860001346DB009B1ADB00684A13449C1D07F17A
:109870000C03184630F0A4F90346013307F10C023B
:10988000204611461A4630F0EAF997F83F30013386
:1098900087F83F3097F83F201346DB009B1ADB0028
:1098A0005A4A134418466049052230F0D8F9594BFA
:1098B000B3F850321A4607F10C03104619460A2233
:1098C0000EF032FF97F83F201346DB009B1ADB00B7
:1098D0004E4A13449C1D07F10C03184630F070F9F2
:1098E0000346013307F10C02204611461A4630F0B8
:1098F000B6F997F83F30013387F83F3097F83F20AB
:109900001346DB009B1ADB00404A134418464749C4
:10991000052230F0A4F93F4B93F80D331A4607F1B6
:109920000C03104619460A220EF0FEFE97F83F205F
:109930001346DB009B1ADB00344A13449C1D07F1DD
:109940000C03184630F03CF90346013307F10C02D2
:10995000204611461A4630F082F997F83F3001331D
:1099600087F83F3097F83F201346DB009B1ADB0057
:10997000264A134418462E49052230F070F9254B2B
:1099800093F80E331A4607F10C03104619460A22C3
:109990000EF0CAFE97F83F201346DB009B1ADB004F
:1099A0001A4A13449C1D07F10C03184630F008F9BD
:1099B0000346013307F10C02204611461A4630F0E7
:1099C0004EF997F83F30013387F83F3097F83F2042
:1099D0001346DB009B1ADB000C4A1344184615495A
:1099E000052230F03CF90B4B93F80F331A4607F180
:1099F0000C03104619460A220EF096FE97F83F20F7
:109A00001346DB009B1ADB0016E000BFF843001092
:109A10004C6F040004070010546F04005C6F0400D6
:109A2000646F04006C6F0400746F04007C6F0400AA
:109A3000846F04008C6F0400E94A13449C1D07F1F5
:109A40000C03184630F0BCF80346013307F10C0252
:109A5000204611461A4630F002F997F83F3001339C
:109A600087F83F3097F83F201346DB009B1ADB0056
:109A7000DB4A13441846DB49052230F0F0F8DA4B94
:109A8000B3F846321A4607F10C03104619460A226B
:109A90000EF04AFE97F83F201346DB009B1ADB00CE
:109AA000CF4A13449C1D07F10C03184630F088F888
:109AB0000346013307F10C02204611461A4630F0E6
:109AC000CEF897F83F30013387F83F3097F83F20C2
:109AD0001346DB009B1ADB00C14A13441846C349F6
:109AE000052230F0BCF8C04B93F820321A4607F13B
:109AF0000C03104619460A220EF016FE97F83F2076
:109B00001346DB009B1ADB00B54A13449C1D07F18A
:109B10000C03184630F054F80346013307F10C02E9
:109B2000204611461A4630F09AF897F83F30013334
:109B300087F83F3097F83F201346DB009B1ADB0085
:109B4000A74A13441846AA49052230F088F8A64BC4
:109B5000B3F844321A4607F10C03104619460A229C
:109B60000EF0E2FD97F83F201346DB009B1ADB0066
:109B70009B4A13449C1D07F10C03184630F020F853
:109B80000346013307F10C02204611461A4630F015
:109B900066F897F83F30013387F83F3097F83F2059
:109BA0001346DB009B1ADB008D4A1344184691498B
:109BB000052230F054F88C4BB3F852321AB207F148
:109BC0000C03104619460A220EF0AEFD97F83F200E
:109BD0001346DB009B1ADB00814A13449C1D07F1EE
:109BE0000C0318462FF0ECFF0346013307F10C027B
:109BF000204611461A4630F032F897F83F300133CC
:109C000087F83F3097F83F201346DB009B1ADB00B4
:109C1000734A134418467849052230F020F8724BF5
:109C2000B3F854321AB207F10C03104619460A224F
:109C30000EF07AFD97F83F201346DB009B1ADB00FD
:109C4000674A13449C1D07F10C0318462FF0B8FF18
:109C50000346013307F10C02204611461A462FF045
:109C6000FEFF97F83F30013387F83F3097F83F20E9
:109C70001346DB009B1ADB00594A134418465F4920
:109C800005222FF0ECFF584BB3F870321A4607F15B
:109C90000C03104619460A222FF0A6FD97F83F2024
:109CA0001346DB009B1ADB004D4A13449C1D07F151
:109CB0000C0318462FF084FF0346013307F10C0212
:109CC000204611461A462FF0CAFF97F83F3001335D
:109CD00087F83F3097F83F201346DB009B1ADB00E4
:109CE0003F4A13441846464905222FF0B8FF3E4B21
:109CF000B3F872321A4607F10C03104619460A22CD
:109D00002FF072FD97F83F201346DB009B1ADB0013
:109D1000334A13449C1D07F10C0318462FF050FFE3
:109D20000346013307F10C02204611461A462FF074
:109D300096FF97F83F30013387F83F307868314914
:109D400003222FF062FF0346002B41F0898000239D
:109D500087F83F3097F83F201346DB009B1ADB0063
:109D60001F4A13441846284905222FF078FF1E4B3E
:109D700093F829301A4607F10C03104619460A22B7
:109D80002FF032FD97F83F201346DB009B1ADB00D3
:109D9000134A13449C1D07F10C0318462FF010FFC3
:109DA0000346013307F10C02204611461A462FF0F4
:109DB00056FF97F83F30013387F83F3097F83F2040
:109DC0001346DB009B1ADB00054A134418460F4973
:109DD00005222FF044FF044B9B881A4618E000BF71
:109DE000F8430010946F0400040700109C6F0400F7
:109DF000A46F0400AC6F0400B46F0400BC6F0400D7
:109E0000C46F0400CC6F0400D06F0400D86F04004E
:109E100007F10C03104619460A222FF0E5FC97F8CB
:109E20003F201346DB009B1ADB00E24A13449C1DD3
:109E300007F10C0318462FF0C3FE0346013307F168
:109E40000C02204611461A462FF009FF97F83F30C2
:109E5000013387F83F3097F83F201346DB009B1A09
:109E6000DB00D44A13441846D34905222FF0F7FEED
:109E7000D24BDB881A4607F10C03104619460A221A
:109E80002FF0B2FC97F83F201346DB009B1ADB0053
:109E9000C84A13449C1D07F10C0318462FF090FE8E
:109EA0000346013307F10C02204611461A462FF0F3
:109EB000D6FE97F83F30013387F83F3097F83F20C0
:109EC0001346DB009B1ADB00BA4A13441846BC4910
:109ED00005222FF0C4FEB94B1B891A4607F10C036B
:109EE000104619460A222FF07FFC97F83F201346B0
:109EF000DB009B1ADB00AF4A13449C1D07F10C03E7
:109F000018462FF05DFE0346013307F10C02204690
:109F100011461A462FF0A3FE97F83F30013387F819
:109F20003F3097F83F201346DB009B1ADB00A14A25
:109F300013441846A34905222FF091FE9F4B9B7AAC
:109F4000002B06D107F10C0318469F4913222FF06E
:109F500086FE9A4B9B7A012B06D107F10C0318461B
:109F60009A4913222FF07BFE944B9B7A022B06D149
:109F700007F10C031846964913222FF070FE8F4B01
:109F80009B7A032B06D107F10C0318469149132243
:109F90002FF065FE97F83F201346DB009B1ADB008D
:109FA000844A13449C1D07F10C0318462FF008FE49
:109FB0000346013307F10C02204611461A462FF0E2
:109FC0004EFE97F83F30013387F83F3097F83F2037
:109FD0001346DB009B1ADB00764A134418467E4981
:109FE00005222FF03CFE754B93F874321A4607F1A8
:109FF0000C031846114602F04FFE97F83F20134617
:10A00000DB009B1ADB006B4A13449C1D07F10C0319
:10A0100018462FF0D5FD0346013307F10C02204608
:10A0200011461A462FF01BFE97F83F30013387F890
:10A030003F3097F83F201346DB009B1ADB005D4A58
:10A0400013441846654905222FF009FE5B4BDB7A65
:10A050001A4607F10C03104619460A222FF0C4FBDA
:10A0600097F83F201346DB009B1ADB00514A13444C
:10A070009C1D07F10C0318462FF0A2FD0346013387
:10A0800007F10C02204611461A462FF0E8FD97F81A
:10A090003F30013387F83F3097F83F201346DB000D
:10A0A0009B1ADB00434A134418464D4905222FF002
:10A0B000D6FD97F83F201346DB009B1ADB003D4A94
:10A0C000134406331846474903222FF0C8FD97F87A
:10A0D0003F30013387F83F3097F83F201346DB00CD
:10A0E0009B1ADB00334A134418463F4905222FF0E0
:10A0F000B6FD324B1B7D1A4607F10C03184611467C
:10A1000002F0CAFD97F83F201346DB009B1ADB00E4
:10A11000284A13449C1D07F10C0318462FF050FDEC
:10A120000346013307F10C02204611461A462FF070
:10A1300096FD97F83F30013387F83F3097F83F207E
:10A140001346DB009B1ADB001A4A134418462749C2
:10A1500005222FF084FD194B9B7D1A4607F10C0355
:10A160001846114602F098FD97F83F201346DB0091
:10A170009B1ADB000F4A13449C1D07F10C03184681
:10A180002FF01EFD0346013307F10C022046114655
:10A190001A462FF064FD97F83F30013387F83F30BF
:10A1A00097F83F201346DB009B1ADB00014A13445B
:10A1B00018461DE0F8430010E06F0400040700108B
:10A1C000E86F0400F06F0400F86F040000700400F2
:10A1D000107004001C70040028700400307004002B
:10A1E0003870040014090010407004004870040026
:10A1F000E74905222FF033FDE64B5B8A1A4607F14B
:10A200000C03104619460A222FF0EEFA97F83F2069
:10A210001346DB009B1ADB00DF4A13449C1D07F149
:10A220000C0318462FF0CCFC0346013307F10C0257
:10A23000204611461A462FF012FD97F83F300133A1
:10A2400087F83F3097F83F201346DB009B1ADB006E
:10A25000D14A13441846D14905222FF000FDCD4BB9
:10A26000DB7D1A4607F10C03104619460A222FF02F
:10A27000BBFA97F83F201346DB009B1ADB00C64A67
:10A2800013449C1D07F10C0318462FF099FC03465C
:10A29000013307F10C02204611461A462FF0DFFC6D
:10A2A00097F83F30013387F83F3097F83F20134647
:10A2B000DB009B1ADB00B84A13441846B849052254
:10A2C0002FF0CDFCB34B1B7E1A4607F10C03104652
:10A2D00019460A222FF088FA97F83F201346DB0030
:10A2E0009B1ADB00AC4A13449C1D07F10C03184673
:10A2F0002FF066FC0346013307F10C02204611469D
:10A300001A462FF0ACFC97F83F30013387F83F3006
:10A3100097F83F201346DB009B1ADB009E4A13444C
:10A320001846A04905222FF09AFC9A4B5B7D1A46ED
:10A3300007F10C03104619460A222FF055FA97F838
:10A340003F201346DB009B1ADB00934A13449C1DFD
:10A3500007F10C0318462FF033FC0346013307F1D5
:10A360000C02204611461A462FF079FC97F83F3030
:10A37000013387F83F3097F83F201346DB009B1AE4
:10A38000DB00854A13441846874905222FF067FCF5
:10A39000804B5B7E1A4607F10C03104619460A22D1
:10A3A0002FF022FA97F83F201346DB009B1ADB00C0
:10A3B000794A13449C1D07F10C0318462FF000FC4A
:10A3C0000346013307F10C02204611461A462FF0CE
:10A3D00046FC97F83F30013387F83F3097F83F202D
:10A3E0001346DB009B1ADB006B4A134418466F4987
:10A3F00005222FF034FC674B9B7D1A4607F10C03B6
:10A400001846114602F048FC97F83F201346DB003F
:10A410009B1ADB00604A13449C1D07F10C0318468D
:10A420002FF0CEFB0346013307F10C022046114604
:10A430001A462FF014FC97F83F30013387F83F306D
:10A4400097F83F201346DB009B1ADB00524A134467
:10A450001846574905222FF002FC4E4B9B891A469D
:10A4600007F10C03104619460A222FF0BDF997F8A0
:10A470003F201346DB009B1ADB00474A13449C1D18
:10A4800007F10C0318462FF09BFB0346013307F13D
:10A490000C02204611461A462FF0E1FB97F83F3098
:10A4A000013387F83F3097F83F201346DB009B1AB3
:10A4B000DB00394A134418463E4905222FF0CFFBF2
:10A4C000344BDB891A4607F10C03104619460A2261
:10A4D0002FF08AF997F83F201346DB009B1ADB0028
:10A4E0002D4A13449C1D07F10C0318462FF068FBFE
:10A4F0000346013307F10C02204611461A462FF09D
:10A50000AEFB97F83F30013387F83F3097F83F2094
:10A510001346DB009B1ADB001F4A134418462649EA
:10A5200005222FF09CFB1B4B1B8A1A4607F10C03DC
:10A53000104619460A222FF057F997F83F20134684
:10A54000DB009B1ADB00144A13449C1D07F10C032B
:10A5500018462FF035FB0346013307F10C02204665
:10A5600011461A462FF07BFB97F83F30013387F8EE
:10A570003F3097F83F201346DB009B1ADB00064A6A
:10A58000134418460D4905222FF069FB18E000BF5F
:10A590005070040004070010F843001058700400C5
:10A5A000607004006870040070700400487004005B
:10A5B00078700400807004008870040090700400BB
:10A5C000E74BB3F884301AB207F10C031046194672
:10A5D0000A222FF009F997F83F201346DB009B1A57
:10A5E000DB00E04A13449C1D07F10C0318462FF0D2
:10A5F000E7FA0346013307F10C02204611461A46DA
:10A600002FF02DFB97F83F30013387F83F3097F854
:10A610003F201346DB009B1ADB00D24A1344184646
:10A62000D14905222FF01BFBCD4B93F882305BB252
:10A6300007F10C021046194602F02EFB97F83F2056
:10A640001346DB009B1ADB00C64A13449C1D07F12E
:10A650000C0318462FF0B4FA0346013307F10C023D
:10A66000204611461A462FF0FAFA97F83F30013388
:10A6700087F83F3097F83F201346DB009B1ADB003A
:10A68000B84A13441846B94905222FF0E8FAB44BEA
:10A69000B3F888301AB207F10C03104619460A22A3
:10A6A0002FF0A2F897F83F201346DB009B1ADB003F
:10A6B000AC4A13449C1D07F10C0318462FF080FA96
:10A6C0000346013307F10C02204611461A462FF0CB
:10A6D000C6FA97F83F30013387F83F3097F83F20AC
:10A6E0001346DB009B1ADB009E4A13441846A04920
:10A6F00005222FF0B4FA9A4BDB8C1A4607F10C03B3
:10A70000104619460A222FF06FF897F83F2013469B
:10A71000DB009B1ADB00934A13449C1D07F10C03DA
:10A7200018462FF04DFA0346013307F10C0220467C
:10A7300011461A462FF093FA97F83F30013387F805
:10A740003F3097F83F201346DB009B1ADB00854A19
:10A7500013441846874905222FF081FA804B93F85D
:10A7600028301A4607F10C031846114602F094FAF5
:10A7700097F83F201346DB009B1ADB00794A13440D
:10A780009C1D07F10C0318462FF01AFA03460133FB
:10A7900007F10C02204611461A462FF060FA97F88E
:10A7A0003F30013387F83F3097F83F201346DB00F6
:10A7B0009B1ADB006B4A134418466F4905222FF0A1
:10A7C0004EFA674BB3F878321AB207F10C03104611
:10A7D00019460A222FF008F897F83F201346DB00AD
:10A7E0009B1ADB005F4A13449C1D07F10C031846BB
:10A7F0002FF0E6F90346013307F10C02204611461B
:10A800001A462FF02CFA97F83F30013387F83F3083
:10A8100097F83F201346DB009B1ADB00514A134494
:10A820001846564905222FF01AFA4D4BB3F87632E6
:10A830001AB207F10C03104619460A222EF0D4FF73
:10A8400097F83F201346DB009B1ADB00454A134470
:10A850009C1D07F10C0318462FF0B2F90346013393
:10A8600007F10C02204611461A462FF0F8F997F826
:10A870003F30013387F83F3097F83F201346DB0025
:10A880009B1ADB00374A134418463D4905222FF036
:10A89000E6F9334BB3F87E321AB207F10C031046D7
:10A8A00019460A222EF0A0FF97F83F201346DB003E
:10A8B0009B1ADB002B4A13449C1D07F10C0318461E
:10A8C0002FF07EF90346013307F10C0220461146B2
:10A8D0001A462FF0C4F997F83F30013387F83F301C
:10A8E00097F83F201346DB009B1ADB001D4A1344F8
:10A8F0001846244905222FF0B2F9194BB3F87A32E1
:10A900001AB207F10C03104619460A222EF06CFF0A
:10A9100097F83F201346DB009B1ADB00114A1344D3
:10A920009C1D07F10C0318462FF04AF9034601332A
:10A9300007F10C02204611461A462FF090F997F8BD
:10A940003F30013387F83F3097F83F201346DB0054
:10A950009B1ADB00034A134418460B49052215E0F5
:10A9600004070010F843001098700400A070040061
:10A97000A8700400B0700400B8700400C070040037
:10A98000C8700400D0700400D87004002FF067F97C
:10A99000E84BB3F87C321AB207F10C0310461946A3
:10A9A0000A222EF021FF97F83F201346DB009B1A66
:10A9B000DB00E14A13449C1D07F10C0318462FF0FD
:10A9C000FFF80346013307F10C02204611461A46F0
:10A9D0002FF045F997F83F30013387F83F3097F86B
:10A9E0003F201346DB009B1ADB00D34A1344184672
:10A9F000D24905222FF033F9CE4BB3F880301AB28A
:10AA000007F10C03104619460A222EF0EDFE97F8C6
:10AA10003F201346DB009B1ADB00C74A13449C1DF2
:10AA200007F10C0318462FF0CBF80346013307F16A
:10AA30000C02204611461A462FF011F997F83F30C4
:10AA4000013387F83F3097F83F201346DB009B1A0D
:10AA5000DB00B94A13441846B94905222FF0FFF824
:10AA6000B44BB3F806311AB207F10C03104619467D
:10AA70000A222EF0B9FE97F83F201346DB009B1AFE
:10AA8000DB00AD4A13449C1D07F10C0318462FF060
:10AA900097F80346013307F10C02204611461A4687
:10AAA0002FF0DDF897F83F30013387F83F3097F803
:10AAB0003F201346DB009B1ADB009F4A13441846D5
:10AAC000A04905222FF0CBF807F10C0318462DF012
:10AAD000CFFC97F83F201346DB009B1ADB00964A19
:10AAE00013449C1D07F10C0318462FF069F8034628
:10AAF000013307F10C02204611461A462FF0AFF839
:10AB000097F83F30013387F83F3097F83F201346DE
:10AB1000DB009B1ADB00884A134418468A49052249
:10AB20002FF09DF807F10C0318462DF0EFFC97F875
:10AB30003F201346DB009B1ADB007F4A13449C1D19
:10AB400007F10C0318462FF03BF80346013307F1D9
:10AB50000C02204611461A462FF081F897F83F3034
:10AB6000013387F83F3097F83F201346DB009B1AEC
:10AB7000DB00714A13441846744905222FF06FF820
:10AB80006C4B93F80B331A4607F10C031846114629
:10AB900002F082F897F83F201346DB009B1ADB0097
:10ABA000654A13449C1D07F10C0318462FF008F862
:10ABB0000346013307F10C02204611461A462FF0D6
:10ABC0004EF897F83F30013387F83F3097F83F2031
:10ABD0001346DB009B1ADB00574A134418465C49B6
:10ABE00005222FF03CF8534B9B8C1AB207F10C0353
:10ABF000104619460A222EF0F7FD97F83F2013461B
:10AC0000DB009B1ADB004C4A13449C1D07F10C032C
:10AC100018462EF0D5FF0346013307F10C022046FB
:10AC200011461A462FF01BF897F83F30013387F88A
:10AC30003F3097F83F201346DB009B1ADB003E4A6B
:10AC400013441846434905222FF009F8394BDB8B92
:10AC50001A4607F10C03104619460A222EF0C4FDCD
:10AC600097F83F201346DB009B1ADB00324A13445F
:10AC70009C1D07F10C0318462EF0A2FF034601337A
:10AC800007F10C02204611461A462EF0E8FF97F80D
:10AC90003F30013387F83F3097F83F201346DB0001
:10ACA0009B1ADB00244A134418462B4905222EF038
:10ACB000D6FF204B9B8B1A4607F10C031046194612
:10ACC0000A222EF091FD97F83F201346DB009B1AD5
:10ACD000DB00194A13449C1D07F10C0318462EF0A3
:10ACE0006FFF0346013307F10C02204611461A4656
:10ACF0002EF0B5FF97F83F30013387F83F3097F8D3
:10AD00003F201346DB009B1ADB000B4A1344184616
:10AD1000124905222EF0A3FF064B9B7E1A4607F12F
:10AD20000C03104619460A222EF05EFD97F83F20CC
:10AD3000134615E004070010F8430010E07004000B
:10AD4000E8700400F0700400F87004000071040062
:10AD500008710400107104001871040020710400CF
:10AD6000DB009B1ADB00E84A13449C1D07F10C032F
:10AD700018462EF025FF0346013307F10C0220464A
:10AD800011461A462EF06BFF97F83F30013387F8D3
:10AD90003F3097F83F201346DB009B1ADB00DA4A6E
:10ADA00013441846D94905222EF059FFD84B1B8C65
:10ADB0001AB207F10C03104619460A222EF014FDB0
:10ADC00097F83F201346DB009B1ADB00CE4A134462
:10ADD0009C1D07F10C0318462EF0F2FE03460133CA
:10ADE00007F10C02204611461A462EF038FF97F85C
:10ADF0003F30013387F83F3097F83F201346DB00A0
:10AE00009B1ADB00C04A13441846C24905222EF0A3
:10AE100026FFBF4B93F822301A4607F10C03104669
:10AE200019460A222EF0E0FC97F83F201346DB007B
:10AE30009B1ADB00B44A13449C1D07F10C0318460F
:10AE40002EF0BEFE0346013307F10C0220461146E8
:10AE50001A462EF004FF97F83F30013387F83F3051
:10AE60007868AD4903222EF0D0FE0346002B40F057
:10AE7000CC81002387F83F3097F83F201346DB0052
:10AE80009B1ADB00A04A13441846A44905222EF061
:10AE9000E6FE9F4B93F8AF30012B06D107F10C0370
:10AEA00018469F490F222EF0DAFE994B93F8AF30E7
:10AEB000002B06D107F10C0318469A490F222EF0F9
:10AEC000CEFE934B93F8AF30022B06D107F10C0363
:10AED000184695490F222EF0C2FE97F83F201346E0
:10AEE000DB009B1ADB00884A13449C1D07F10C030E
:10AEF00018462EF065FE0346013307F10C0220468A
:10AF000011461A462EF0ABFE97F83F30013387F812
:10AF10003F3097F83F201346DB009B1ADB007A4A4C
:10AF200013441846814905222EF099FE784BB3F858
:10AF3000AC301A4607F10C03104619460A222EF0CF
:10AF400053FC97F83F201346DB009B1ADB006E4A48
:10AF500013449C1D07F10C0318462EF031FE0346E6
:10AF6000013307F10C02204611461A462EF077FEF7
:10AF700097F83F30013387F83F3097F83F2013466A
:10AF8000DB009B1ADB00604A13441846684905221F
:10AF90002EF065FE07F10C0318462DF0C7FB97F85D
:10AFA0003F201346DB009B1ADB00574A13449C1DCD
:10AFB00007F10C0318462EF003FE0346013307F198
:10AFC0000C02204611461A462EF049FE97F83F30F3
:10AFD000013387F83F3097F83F201346DB009B1A78
:10AFE000DB00494A13441846524905222EF037FE29
:10AFF00007F10C0318462DF0E7FB97F83F201346A6
:10B00000DB009B1ADB00404A13449C1D07F10C0334
:10B0100018462EF0D5FD0346013307F10C022046F9
:10B0200011461A462EF01BFE97F83F30013387F881
:10B030003F3097F83F201346DB009B1ADB00324A73
:10B04000134418463C4905222EF009FE304B93F874
:10B050000C331A4607F10C031846114601F01CFE8A
:10B0600097F83F201346DB009B1ADB00264A134467
:10B070009C1D07F10C0318462EF0A2FD0346013378
:10B0800007F10C02204611461A462EF0E8FD97F80B
:10B090003F30013387F83F3097F83F201346DB00FD
:10B0A0009B1ADB00184A13441846244905222EF047
:10B0B000D6FD174B93F808315AB207F10C0310462E
:10B0C00019460A222EF090FB97F83F201346DB002A
:10B0D0009B1ADB000C4A13449C1D07F10C03184615
:10B0E0002EF06EFD0346013307F10C022046114697
:10B0F0001A462EF0B4FD97F83F30013387F83F3001
:10B1000097F83F2013461BE0F84300102871040015
:10B110000407001030710400387104003C71040011
:10B1200044710400F86F04001C70040050710400A6
:10B1300058710400607104006871040070710400AB
:10B14000DB009B1ADB00E74A13441846E649052258
:10B150002EF085FDE54BB3F80A311AB207F10C0366
:10B16000104619460A222EF03FFB97F83F2013465F
:10B17000DB009B1ADB00DB4A13449C1D07F10C0328
:10B1800018462EF01DFD0346013307F10C02204640
:10B1900011461A462EF063FD97F83F30013387F8C9
:10B1A0003F3097F83F201346DB009B1ADB00CD4A67
:10B1B00013441846CE4905222EF051FDCB4BB3F86F
:10B1C0000C311AB207F10C03104619460A222EF070
:10B1D0000BFB97F83F201346DB009B1ADB00C14AAC
:10B1E00013449C1D07F10C0318462EF0E9FC03469E
:10B1F000013307F10C02204611461A462EF02FFDAE
:10B2000097F83F30013387F83F307868B949092211
:10B210002EF0FBFC0346002B40F09A81002387F8B8
:10B220003F3097F83F201346DB009B1ADB00AD4A06
:10B2300013441846B04905222EF011FDAB4BB3F86C
:10B24000B2311AB207F10C03104619460A222EF049
:10B25000CBFA97F83F201346DB009B1ADB00A14A8C
:10B2600013449C1D07F10C0318462EF0A9FC03465D
:10B27000013307F10C02204611461A462EF0EFFC6E
:10B2800097F83F30013387F83F3097F83F20134657
:10B29000DB009B1ADB00934A1344184697490522AA
:10B2A0002EF0DDFC914B93F8B4311A4607F10C03F4
:10B2B0001846114601F0F0FC97F83F201346DB00DA
:10B2C0009B1ADB00874A13449C1D07F10C031846A8
:10B2D0002EF076FC0346013307F10C02204611469E
:10B2E0001A462EF0BCFC97F83F30013387F83F3008
:10B2F00097F83F201346DB009B1ADB00794A134482
:10B3000018467F4905222EF0AAFC784B93F8B031FD
:10B31000012B06D107F10C0318467A490F222EF0B3
:10B320009EFC724B93F8B031022B06D107F10C034F
:10B33000184675490F222EF092FC6C4B93F8B031F1
:10B34000002B06D107F10C03184670490F222EF08E
:10B3500086FC97F83F201346DB009B1ADB00614A0E
:10B3600013449C1D07F10C0318462EF029FC0346DC
:10B37000013307F10C02204611461A462EF06FFCED
:10B3800097F83F30013387F83F3097F83F20134656
:10B39000DB009B1ADB00534A134418465C49052224
:10B3A0002EF05DFC07F10C0318462CF00DFF97F80A
:10B3B0003F201346DB009B1ADB004A4A13449C1DC6
:10B3C00007F10C0318462EF0FBFB0346013307F18F
:10B3D0000C02204611461A462EF041FC97F83F30E9
:10B3E000013387F83F3097F83F201346DB009B1A64
:10B3F000DB003C4A13441846464905222EF02FFC38
:10B4000007F10C0318462CF02DFF97F83F20134648
:10B41000DB009B1ADB00334A13449C1D07F10C032D
:10B4200018462EF0CDFB0346013307F10C022046EF
:10B4300011461A462EF013FC97F83F30013387F877
:10B440003F3097F83F201346DB009B1ADB00254A6C
:10B4500013441846304905222EF001FC234B93F883
:10B46000B6311A4607F10C03104619460A222EF08F
:10B47000BBF997F83F201346DB009B1ADB00194A03
:10B4800013449C1D07F10C0318462EF099FB03464C
:10B49000013307F10C02204611461A462EF0DFFB5D
:10B4A00097F83F30013387F83F3097F83F20134635
:10B4B000DB009B1ADB000B4A134418461749052290
:10B4C0002EF0CDFB094B93F8B7311A4607F10C0368
:10B4D000104619460A222EF087F997F83F201346A6
:10B4E000DB001DE0F8430010787104000407001031
:10B4F0008071040088710400947104009C71040040
:10B50000A4710400447104001C700400F86F04006E
:10B51000AC710400B4710400BC710400C471040077
:10B520009B1ADB00E54A13449C1D07F10C031846E7
:10B530002EF046FB0346013307F10C02204611466C
:10B540001A462EF08CFB97F83F30013387F83F30D6
:10B550007868DB4903222EF058FB0346002B40F0AD
:10B56000DB81002387F83F3097F83F201346DB004C
:10B570009B1ADB00D14A13441846D24905222EF00B
:10B580006EFBD14BDB891AB207F10C03104619464A
:10B590000A222EF029F997F83F201346DB009B1A68
:10B5A000DB00C64A13449C1D07F10C0318462EF01D
:10B5B00007FB0346013307F10C02204611461A46E9
:10B5C0002EF04DFB97F83F30013387F83F3097F866
:10B5D0003F201346DB009B1ADB00B84A1344184691
:10B5E000BA4905222EF03BFBB94BB3F810311AB221
:10B5F00007F10C03104619460A222EF0F5F897F8C9
:10B600003F201346DB009B1ADB00AC4A13449C1D11
:10B6100007F10C0318462EF0D3FA0346013307F165
:10B620000C02204611461A462EF019FB97F83F30BF
:10B63000013387F83F3097F83F201346DB009B1A11
:10B64000DB009E4A13441846A24905222EF007FB50
:10B650009F4BB3F812311AB207F10C03104619468A
:10B660000A222EF0C1F897F83F201346DB009B1A00
:10B67000DB00924A13449C1D07F10C0318462EF080
:10B680009FFA0346013307F10C02204611461A4681
:10B690002EF0E5FA97F83F30013387F83F3097F8FE
:10B6A0003F201346DB009B1ADB00844A13441846F4
:10B6B000894905222EF0D3FA854BB3F814311AB21A
:10B6C00007F10C03104619460A222EF08DF897F860
:10B6D0003F201346DB009B1ADB00784A13449C1D75
:10B6E00007F10C0318462EF06BFA0346013307F1FD
:10B6F0000C02204611461A462EF0B1FA97F83F3058
:10B70000013387F83F3097F83F201346DB009B1A40
:10B71000DB006A4A13441846704905222EF09FFA4E
:10B720006B4B93F816311A4607F10C031846114675
:10B7300001F0B2FA97F83F201346DB009B1ADB00BA
:10B740005E4A13449C1D07F10C0318462EF038FA8C
:10B750000346013307F10C02204611461A462EF02B
:10B760007EFA97F83F30013387F83F3097F83F2053
:10B770001346DB009B1ADB00504A13441846584915
:10B7800005222EF06CFA524B93F81731012B06D19B
:10B7900007F10C03184653490F222EF060FA4C4B68
:10B7A00093F81731022B06D107F10C0318464E49C6
:10B7B0000F222EF054FA464B93F81731002B06D186
:10B7C00007F10C03184649490F222EF048FA404B66
:10B7D00093F81731032B06D107F10C03184644499F
:10B7E0000F222EF03CFA97F83F201346DB009B1AFD
:10B7F000DB00324A13449C1D07F10C0318462EF05F
:10B80000DFF90346013307F10C02204611461A46C0
:10B810002EF025FA97F83F30013387F83F3097F83C
:10B820003F201346DB009B1ADB00244A13441846D2
:10B83000304905222EF013FA07F10C0318462CF0BC
:10B840006FFB97F83F201346DB009B1ADB001B4A77
:10B8500013449C1D07F10C0318462EF0B1F9034662
:10B86000013307F10C02204611461A462EF0F7F973
:10B8700097F83F30013387F83F3097F83F20134661
:10B88000DB009B1ADB000D4A134418461A490522B7
:10B890002EF0E5F907F10C0318462CF08FFB97F812
:10B8A0003F201346DB009B1ADB00044A13449C1D17
:10B8B00007F10C0318462EF083F91FE0F84300103F
:10B8C000CC710400D0710400C4210010D8710400B0
:10B8D00004070010E0710400E8710400F071040036
:10B8E000F8710400447104001C700400F86F040037
:10B8F000007204000C720400147204000346013349
:10B9000007F10C02204611461A462EF0A8F997F8C6
:10B910003F30013387F83F307868A44907222EF082
:10B9200074F90346002B40F07881002387F83F30FC
:10B9300097F83F201346DB009B1ADB009C4A134418
:10B9400018469C4905222EF08AF99B4BDB79002B87
:10B9500003D1994B5B7C002B01D0012300E0002335
:10B9600007F10C021046194601F096F997F83F20AE
:10B970001346DB009B1ADB008D4A13449C1D07F124
:10B980000C0318462EF01CF90346013307F10C0294
:10B99000204611461A462EF062F997F83F300133DF
:10B9A00087F83F3097F83F201346DB009B1ADB00F7
:10B9B0007F4A13441846814905222EF050F9804BE6
:10B9C0005A6807F10C03104619460A222DF00CFFA5
:10B9D0007B4B9B68002B08D0794B9A6807F10C03CE
:10B9E000104619460A222DF0FFFE97F83F20134615
:10B9F000DB009B1ADB006E4A13449C1D07F10C030D
:10BA000018462EF0DDF80346013307F10C022046FC
:10BA100011461A462EF023F997F83F30013387F884
:10BA20003F3097F83F201346DB009B1ADB00604A4B
:10BA300013441846634905222EF011F95E4B1B781A
:10BA4000002B03D15C4B9B7A002B01D0012300E03B
:10BA5000002307F10C021046194601F01DF997F872
:10BA60003F201346DB009B1ADB00514A13449C1D08
:10BA700007F10C0318462EF0A3F80346013307F133
:10BA80000C02204611461A462EF0E9F897F83F308E
:10BA9000013387F83F3097F83F201346DB009B1AAD
:10BAA000DB00434A13441846474905222EF0D7F8D5
:10BAB000414B5B78002B03D13F4BDB7A002B01D04D
:10BAC000012300E0002307F10C021046194601F0A3
:10BAD000E3F897F83F201346DB009B1ADB00344A5B
:10BAE00013449C1D07F10C0318462EF069F8034619
:10BAF000013307F10C02204611461A462EF0AFF82A
:10BB000097F83F30013387F83F3097F83F201346CE
:10BB1000DB009B1ADB00264A134418462B490522FA
:10BB20002EF09DF8244B9B78002B03D1224B1B7BDE
:10BB3000002B01D0012300E0002307F10C02104686
:10BB4000194601F0A9F897F83F201346DB009B1A2D
:10BB5000DB00174A13449C1D07F10C0318462EF016
:10BB60002FF80346013307F10C02204611461A460E
:10BB70002EF075F897F83F30013387F83F3097F88B
:10BB80003F201346DB009B1ADB00094A134418468A
:10BB90000F4905222EF063F8074BDB78002B03D109
:10BBA000054B5B7B002B15D0012314E01C720400B5
:10BBB000F843001024720400300A00102C720400B4
:10BBC00040220010347204003C72040044720400ED
:10BBD0004C720400002307F10C021046194601F0D4
:10BBE0005BF897F83F201346DB009B1ADB00E34A23
:10BBF00013449C1D07F10C0318462DF0E1FF03468A
:10BC0000013307F10C02204611461A462EF027F8A0
:10BC100097F83F30013387F83F307868D8490B22D6
:10BC20002DF0F3FF0346002B40F08182002387F8BC
:10BC30003F3097F83F201346DB009B1ADB00CF4ACA
:10BC400013441846CF4905222EF009F8CE4B5B89E4
:10BC50001AB207F10C03104619460A222DF0C4FD52
:10BC600097F83F201346DB009B1ADB00C34A1344BE
:10BC70009C1D07F10C0318462DF0A2FF034601336B
:10BC800007F10C02204611461A462DF0E8FF97F8FE
:10BC90003F30013387F83F3097F83F201346DB00F1
:10BCA0009B1ADB00B54A13441846B84905222DF00B
:10BCB000D6FFB54B9B891AB207F10C031046194603
:10BCC0000A222DF091FD97F83F201346DB009B1AC6
:10BCD000DB00AA4A13449C1D07F10C0318462DF003
:10BCE0006FFF0346013307F10C02204611461A4646
:10BCF0002DF0B5FF97F83F30013387F83F3097F8C4
:10BD00003F201346DB009B1ADB009C4A1344184675
:10BD10009F4905222DF0A3FF9E4B1B881AB207F105
:10BD20000C03104619460A222DF05EFD97F83F20BD
:10BD30001346DB009B1ADB00904A13449C1D07F15D
:10BD40000C0318462DF03CFF0346013307F10C02AB
:10BD5000204611461A462DF082FF97F83F300133F6
:10BD600087F83F3097F83F201346DB009B1ADB0033
:10BD7000824A13441846884905222DF070FF824BF1
:10BD8000DB891AB207F10C03104619460A222DF07E
:10BD90002BFD97F83F201346DB009B1ADB00774A08
:10BDA00013449C1D07F10C0318462DF009FF0346B0
:10BDB000013307F10C02204611461A462DF04FFFC1
:10BDC00097F83F30013387F83F3097F83F2013460C
:10BDD000DB009B1ADB00694A134418466F490522B1
:10BDE0002DF03DFF684B1B891AB207F10C0310467A
:10BDF00019460A222DF0F8FC97F83F201346DB0085
:10BE00009B1ADB005D4A13449C1D07F10C03184686
:10BE10002DF0D6FE0346013307F10C0220461146F1
:10BE20001A462DF01CFF97F83F30013387F83F305A
:10BE300097F83F201346DB009B1ADB004F4A134460
:10BE40001846574905222DF00AFF4F4B5A6807F153
:10BE50000C03104619460A222DF0C6FC97F83F2025
:10BE60001346DB009B1ADB00444A13449C1D07F178
:10BE70000C0318462DF0A4FE0346013307F10C0213
:10BE8000204611461A462DF0EAFE97F83F3001335E
:10BE900087F83F3097F83F201346DB009B1ADB0002
:10BEA000364A134418463F4905222DF0D8FE364B3A
:10BEB0009B8A1AB207F10C03104619460A222DF08C
:10BEC00093FC97F83F201346DB009B1ADB002B4ABC
:10BED00013449C1D07F10C0318462DF071FE034618
:10BEE000013307F10C02204611461A462DF0B7FE29
:10BEF00097F83F30013387F83F3097F83F201346DB
:10BF0000DB009B1ADB001D4A134418462649052214
:10BF10002DF0A5FE1F4B5B8D1AB207F10C031046E6
:10BF200019460A222DF060FC97F83F201346DB00EB
:10BF30009B1ADB00114A13449C1D07F10C031846A1
:10BF40002DF03EFE0346013307F10C022046114658
:10BF50001A462DF084FE97F83F30013387F83F30C2
:10BF600097F83F201346DB009B1ADB00034A13447B
:10BF700018460E4905222DF072FE19E0F843001014
:10BF80005472040060720400C4210010687204003E
:10BF90007072040020270010D07104007872040031
:10BFA0008072040088720400907204009872040089
:10BFB000E74B5B8A1AB207F10C03104619460A22B6
:10BFC0002DF012FC97F83F201346DB009B1ADB0094
:10BFD000E04A13449C1D07F10C0318462DF0F0FDB8
:10BFE0000346013307F10C02204611461A462DF094
:10BFF00036FE97F83F30013387F83F3097F83F20FF
:10C000001346DB009B1ADB00D24A13441846D24980
:10C0100005222DF024FED14B1B8D1AB207F10C0323
:10C02000104619460A222DF0DFFB97F83F201346F1
:10C03000DB009B1ADB00C74A13449C1D07F10C036D
:10C0400018462DF0BDFD0346013307F10C022046D2
:10C0500011461A462DF003FE97F83F30013387F85A
:10C060003F3097F83F201346DB009B1ADB00B94AAC
:10C0700013441846BA4905222DF0F1FDB44B1B8A32
:10C080001AB207F10C03104619460A222DF0ACFB38
:10C0900097F83F201346DB009B1ADB00AD4A1344A0
:10C0A0009C1D07F10C0318462DF08AFD0346013351
:10C0B00007F10C02204611461A462DF0D0FD97F8E4
:10C0C0003F30013387F83F3097F83F201346DB00BD
:10C0D0009B1ADB009F4A13441846A24905222DF003
:10C0E000BEFD9E4B9B8E1AB207F10C0310461946FB
:10C0F0000A222DF079FB97F83F201346DB009B1AAC
:10C10000DB00944A13449C1D07F10C0318462DF0E4
:10C1100057FD0346013307F10C02204611461A462B
:10C120002DF09DFD97F83F30013387F83F30786858
:10C130008D4907222DF069FD0346002B40F09385C1
:10C14000002387F83F3097F83F201346DB009B1A07
:10C15000DB00804A13441846844905222DF07FFDF8
:10C16000834B1A6807F10C03104619460A222DF07A
:10C170003BFB97F83F201346DB009B1ADB00754A18
:10C1800013449C1D07F10C0318462DF019FD0346BE
:10C19000013307F10C02204611461A462DF05FFDCF
:10C1A00097F83F201346DB009B1ADB00694A1344D3
:10C1B000063318462BF0B4F997F83F30013387F86F
:10C1C0003F3097F83F201346DB009B1ADB00614AA3
:10C1D00013441846674905222DF041FD5F4B9A6DC7
:10C1E00007F10C03104619460A220CF09DFA97F845
:10C1F0003F201346DB009B1ADB00564A13449C1D6C
:10C2000007F10C0318462DF0DBFC0346013307F160
:10C210000C02204611461A462DF021FD97F83F30BA
:10C22000013387F83F3097F83F201346DB009B1A15
:10C23000DB00484A134418464F4905222DF00FFDF4
:10C2400007F10C031846012103F0BCFE97F83F20CC
:10C250001346DB009B1ADB003E4A13449C1D07F18A
:10C260000C0318462DF0ACFC0346013307F10C0219
:10C27000204611461A462DF0F2FC97F83F30013364
:10C2800087F83F3097F83F201346DB009B1ADB000E
:10C29000304A13441846394905222DF0E0FC07F1D5
:10C2A0000C03184603F00CFF97F83F201346DB0001
:10C2B0009B1ADB00274A13449C1D07F10C03184608
:10C2C0002DF07EFC0346013307F10C022046114697
:10C2D0001A462DF0C4FC97F83F30013387F83F3001
:10C2E00097F83F201346DB009B1ADB00194A1344E2
:10C2F0001846234905222DF0B2FC07F10C0318461D
:10C30000FBF750FB97F83F201346DB009B1ADB003E
:10C31000104A13449C1D07F10C0318462DF050FCE5
:10C320000346013307F10C02204611461A462DF050
:10C3300096FC97F83F30013387F83F3097F83F205D
:10C340001346DB009B1ADB00024A1344184619E02F
:10C35000C4210010F8430010A07204002027001030
:10C36000A8720400B0720400B8720400C072040025
:10C37000E8060010C8720400D0720400D8720400ED
:10C38000E07204005D4905222DF069FC5C4B9B784E
:10C39000012B06D107F10C0318465A490F222DF044
:10C3A0005EFC574B9B78032B06D107F10C03184614
:10C3B00055490F222DF053FC514B9B78002B06D191
:10C3C00007F10C03184651490F222DF048FC4C4B45
:10C3D0009B78042B06D107F10C0318464C490F2219
:10C3E0002DF03DFC464B9B78052B06D107F10C0345
:10C3F000184648490F222DF032FC414B9B78082B00
:10C4000006D107F10C03184643490F222DF027FCF3
:10C410003B4B9B78022B06D107F10C0318463F4992
:10C420000F222DF01CFC364B9B78072B06D107F111
:10C430000C0318463A490F222DF011FC304B9B7823
:10C44000062B06D107F10C03184636490F222DF0B2
:10C4500006FC97F83F201346DB009B1ADB00324AAC
:10C4600013449C1D07F10C0318462DF0A9FB03464D
:10C47000013307F10C02204611461A462DF0EFFB5E
:10C4800097F83F30013387F83F301D4B9B78022BE4
:10C490004ED197F83F201346DB009B1ADB00224A5F
:10C4A00013441846214905222DF0D9FB144B1B8952
:10C4B0001A4607F10C03104619460A222DF094F98A
:10C4C00097F83F201346DB009B1ADB00164A134403
:10C4D0009C1D07F10C0318462DF072FB0346013337
:10C4E00007F10C02204611461A462DF0B8FB97F8CA
:10C4F0003F30013387F83F304AE000BFE872040064
:10C5000020270010F0720400FC720400087304007D
:10C5100010730400147304001C73040028730400D7
:10C52000347304003C730400F843001048730400A3
:10C5300097F83F201346DB009B1ADB00E34A1344C5
:10C540001846E34905222DF08AFB07F10C03002071
:10C5500019460A222DF048F997F83F201346DB00D0
:10C560009B1ADB00D94A13449C1D07F10C031846A3
:10C570002DF026FB0346013307F10C02204611463D
:10C580001A462DF06CFB97F83F30013387F83F30A7
:10C5900097F83F201346DB009B1ADB00CB4A13447D
:10C5A0001846CC4905222DF05AFBCB4B9B881A46E6
:10C5B00007F10C03104619460A222DF015F997F8D9
:10C5C0003F201346DB009B1ADB00C04A13449C1D2E
:10C5D00007F10C0318462DF0F3FA0346013307F177
:10C5E0000C02204611461A462DF039FB97F83F30D1
:10C5F000013387F83F3097F83F201346DB009B1A42
:10C60000DB00B24A13441846B44905222DF027FB3B
:10C61000B14BDB881A4607F10C03104619460A2273
:10C620002DF0E2F897F83F201346DB009B1ADB0061
:10C63000A64A13449C1D07F10C0318462DF0C0FABE
:10C640000346013307F10C02204611461A462DF02D
:10C6500006FB97F83F30013387F83F3097F83F20CB
:10C660001346DB009B1ADB00984A134418469C498A
:10C6700005222DF0F4FA984B1B69184699492EF0C3
:10C680001FFA034618462EF0C9FB024607F10C03B9
:10C69000104619460A220CF047F897F83F20134637
:10C6A000DB009B1ADB00894A13449C1D07F10C0335
:10C6B00018462DF085FA0346013307F10C02204697
:10C6C00011461A462DF0CBFA97F83F30013387F820
:10C6D0003F3097F83F201346DB009B1ADB007B4A74
:10C6E00013441846804905222DF0B9FA7A4BDB68CD
:10C6F00018467C492EF0E4F9034618462EF08EFBCE
:10C70000024607F10C03104619460A220CF00CF8F9
:10C7100097F83F201346DB009B1ADB006B4A13445B
:10C720009C1D07F10C0318462DF04AFA034601330D
:10C7300007F10C02204611461A462DF090FA97F8A0
:10C740003F30013387F83F3097F83F201346DB0036
:10C750009B1ADB005D4A13441846644905222DF0FC
:10C760007EFA5D4B93F861301A4607F10C031046D0
:10C7700019460A222DF038F897F83F201346DB00BF
:10C780009B1ADB00514A13449C1D07F10C03184609
:10C790002DF016FA0346013307F10C02204611462C
:10C7A0001A462DF05CFA97F83F30013387F83F3096
:10C7B00097F83F201346DB009B1ADB00434A1344E3
:10C7C00018464B4905222DF04AFA4A4BDB781A46A7
:10C7D00007F10C031846114600F05EFA97F83F2067
:10C7E0001346DB009B1ADB00384A13449C1D07F1FB
:10C7F0000C0318462DF0E4F90346013307F10C024F
:10C80000204611461A462DF02AFA97F83F30013398
:10C8100087F83F3097F83F201346DB009B1ADB0078
:10C820002A4A13441846344905222DF018FA314B90
:10C830009B781A4607F10C031846114600F02CFAB3
:10C8400097F83F201346DB009B1ADB001F4A134476
:10C850009C1D07F10C0318462DF0B2F90346013375
:10C8600007F10C02204611461A462DF0F8F997F808
:10C870003F30013387F83F3097F83F201346DB0005
:10C880009B1ADB00114A134418461C4905222DF05F
:10C89000E6F91B4B9B6B18461A492EF011F903461B
:10C8A00018462EF0A1FA024607F10C03104619466D
:10C8B0000A220BF039FF97F83F201346DB009B1A42
:10C8C000DB00024A13449C1D1EE000BFF843001029
:10C8D00048730400507304002027001058730400AC
:10C8E000607304000000C8426873040070730400A1
:10C8F0007873040098270010807304008873040084
:10C900001C1E00100000204107F10C0318462DF0FA
:10C9100057F90346013307F10C02204611461A4627
:10C920002DF09DF997F83F30013387F83F3097F8A5
:10C930003F201346DB009B1ADB00CC4A1344184609
:10C94000CB4905222DF08BF9CA4BDB6A18462EF035
:10C950004BFA024607F10C03104619460A222CF046
:10C9600043FF97F83F201346DB009B1ADB00BF4ACA
:10C9700013449C1D07F10C0318462DF021F90346C2
:10C98000013307F10C02204611461A462DF067F9D3
:10C9900097F83F30013387F83F3097F83F20134630
:10C9A000DB009B1ADB00B14A13441846B24905224A
:10C9B0002DF055F9AF4B93F836301A4607F10C03BA
:10C9C0001846114600F068F997F83F201346DB003F
:10C9D0009B1ADB00A54A13449C1D07F10C03184663
:10C9E0002DF0EEF80346013307F10C022046114604
:10C9F0001A462DF034F997F83F30013387F83F306D
:10CA000097F83F201346DB009B1ADB00974A13443C
:10CA100018469A4905222DF022F9994B1B781A469F
:10CA200007F10C031846114600F036F997F83F203D
:10CA30001346DB009B1ADB008C4A13449C1D07F154
:10CA40000C0318462DF0BCF80346013307F10C0225
:10CA5000204611461A462DF002F997F83F3001336F
:10CA600087F83F3097F83F201346DB009B1ADB0026
:10CA70007E4A13441846834905222DF0F0F87D4B79
:10CA800093F851301A4607F10C03104619460A2252
:10CA90002CF0AAFE97F83F201346DB009B1ADB0020
:10CAA000724A13449C1D07F10C0318462DF088F8B8
:10CAB0000346013307F10C02204611461A462DF0B9
:10CAC000CEF897F83F30013387F83F3097F83F2092
:10CAD0001346DB009B1ADB00644A134418466A497C
:10CAE00005222DF0BCF8664B5B781A4607F10C0363
:10CAF0001846114600F0D0F897F83F201346DB00A7
:10CB00009B1ADB00594A13449C1D07F10C0318467D
:10CB10002DF056F80346013307F10C02204611466A
:10CB20001A462DF09CF897F83F30013387F83F30D4
:10CB300097F83F201346DB009B1ADB004B4A134457
:10CB40001846524905222DF08AF84A4B93F85E3078
:10CB50001A4607F10C031846114600F09DF897F8A5
:10CB60003F201346DB009B1ADB00404A13449C1D08
:10CB700007F10C0318462DF023F80346013307F1A3
:10CB80000C02204611461A462DF069F897F83F30FE
:10CB9000013387F83F3097F83F201346DB009B1A9C
:10CBA000DB00324A13441846394905222DF057F864
:10CBB000304BB3F85C301A4607F10C0310461946A7
:10CBC0000A222CF011FE97F83F201346DB009B1A37
:10CBD000DB00264A13449C1D07F10C0318462CF079
:10CBE000EFFF0346013307F10C02204611461A46B7
:10CBF0002DF035F897F83F30013387F83F3097F83C
:10CC00003F201346DB009B1ADB00184A13441846EA
:10CC1000204905222DF023F8164B93F85F301A4671
:10CC200007F10C03104619460A222CF0DDFD97F897
:10CC30003F201346DB009B1ADB000C4A13449C1D6B
:10CC400007F10C0318462CF0BBFF0346013307F134
:10CC50000C02204611461A462DF001F897F83F3095
:10CC6000013387F83F304437BD4690BDF84300108C
:10CC7000907304002027001098730400A073040030
:10CC800098270010A8730400B0730400B873040060
:10CC9000C0730400C873040080B582B000AF786030
:10CCA00039603B68002B05D0786806490A222CF0D1
:10CCB000D6FF04E0786804490A222CF0D0FF083738
:10CCC000BD4680BDD0730400D873040090B597B002
:10CCD00000AF78600B46FB700023A7F856300023A6
:10CCE000A7F854300023A7F85030002387F85330BA
:10CCF0000023FB640023A7F856300CE0B7F8563049
:10CD000007F158021344002203F84C2CB7F85630B0
:10CD10000133A7F85630B7F85630312BEED900233F
:10CD2000A7F85630B7F856305A1CA7F856201A46BE
:10CD3000894B0A219954B7F856305A1CA7F8562047
:10CD40001A46854B3C21995497F9032007F140037B
:10CD5000104619460A222CF047FD0023A7F854304C
:10CD600011E0B7F856305A1CA7F856201A46B7F803
:10CD70005430591CA7F8541007F158010B4413F80C
:10CD8000181C754B9954B7F8543007F158021344E6
:10CD900013F8183C002BE4D1B7F856305A1CA7F80A
:10CDA00056201A466C4B3E219954B7F856305A1CFF
:10CDB000A7F856201A46684B7B219954B7F856308D
:10CDC0005A1CA7F856201A46634B0A21995400238F
:10CDD000A7F854300023FB640023A7F854309AE0EE
:10CDE000002387F85330B7F856305A1CA7F856205E
:10CDF0001A46594B2221995417E0B7F856305A1C5D
:10CE0000A7F856201846B7F8542097F85330591C05
:10CE100087F853101C4651491346DB009B1ADB0070
:10CE200023440B441A784C4B1A54B7F8542097F803
:10CE300053104A481346DB009B1ADB000B440344A3
:10CE40001B78002BD9D1B7F856305A1CA7F85620BA
:10CE50001A46414B22219954B7F856305A1CA7F86C
:10CE600056201A463C4B3A219954B7F856305A1C72
:10CE7000A7F856201A46384B20219954002387F8EA
:10CE8000533017E0B7F856305A1CA7F8562018460A
:10CE9000B7F8542097F85330591C87F853101C46A4
:10CEA0002E491346DB009B1ADB0023440B449A797E
:10CEB000294B1A54B7F8542097F8531027481346B3
:10CEC000DB009B1ADB000B4403449B79002BD9D178
:10CED000B7F854305A1C21491346DB009B1ADB007B
:10CEE0000B441B78002B08D0B7F856305A1CA7F813
:10CEF00056201A46184B2C219954B7F856305A1C14
:10CF0000A7F856201A46144B0A219954B7F8543002
:10CF10000133A7F85430B7F8542010491346DB000A
:10CF20009B1ADB000B441B78002B7FF459AFB7F83A
:10CF300056305A1CA7F856201A46074B7D219954A3
:10CF4000B7F856305A1CA7F856201A46024B0A2149
:10CF500099545C37BD4690BDE84E0010F843001070
:10CF600090B585B000AF786039600023FB60002386
:10CF7000FB720023FB60F8E1FB687A6813441A78BF
:10CF8000974B1A70964B1B785BB218462CF0C0FB7F
:10CF90000346002B00D0E5E1924B1B6803330A2BBC
:10CFA00000F2D58101A252F823F000BFD9CF0000D2
:10CFB000F5CF00004FD30000A7D00000EBD0000059
:10CFC0003DD1000093D100004FD3000019D20000E2
:10CFD0007BD2000023D30000814B1B785BB23C2B3B
:10CFE00007D1804B6FF001021A607F4B00221A605C
:10CFF000B8E1ACE17A4B1B785BB23E2B3BD17A4B6C
:10D000001B687A4A0021D154784805F001F803469C
:10D01000002B06D075482CF0CFFC0246744B1A60EA
:10D0200002E0734BFF221A60714B1B68002B03D088
:10D030006F4B1B68632B19D16A4B00221A606D4B32
:10D0400000221A606C4B00221A606C4B00221A609E
:10D050000023FB7206E0FB7A694A0021D154FB7A77
:10D060000133FB72FB7A1D2BF5D97BE15D4B6FF031
:10D0700002021A600AE05C4B1B68594A11785B4A4D
:10D08000D154594B1B680133574A1360564B1B68E8
:10D09000032B07DD534B6FF002021A60594B00223D
:10D0A0009A7754E153E14E4B1B785BB27B2B1BD13B
:10D0B000544B00229A774E4B1B68002B08D04C4BE8
:10D0C0001B68632B04D0474B6FF002021A6049E1E2
:10D0D000444B01221A60474B00221A604A4B1B68DE
:10D0E0000133494A13603DE131E13D4B1B785BB2AE
:10D0F000222B05D1414B00221A603A4B02221A60C2
:10D10000374B1B785BB27D2B17D13F4B1B68013B24
:10D110003D4A13603C4B1B68002B06D1394B012262
:10D120009A77304B6FF002021A60374B1B68002B66
:10D1300003DD2C4B07221A6009E108E1284B1B781C
:10D140005BB2222B19D12D4B1B68304A0021D154E0
:10D15000284B1A681346DB009B1ADB002C4A9C18EC
:10D160002A482CF02DFD0346204628491A462CF06B
:10D1700076FD1C4B03221A60E9E0204B1B68184A1D
:10D180001178224AD1541D4B1B6801331B4A13608E
:10D19000DDE0134B1B785BB27B2B00D1E2E0104B40
:10D1A0001B785BB23A2B03D1134B00221A60D9E0F3
:10D1B0000B4B1B785BB2222B03D10A4B05221A6062
:10D1C000C5E0084B06221A600B4B1B68044A117815
:10D1D000104AD154084B1B680133074A1360B6E06C
:10D1E0005C010010100000106001001064010010CC
:10D1F000902700106C0100107001001074010010E5
:10D2000078010010A0270010980100109C01001068
:10D2100008390010BC010010584B1B785BB2222B60
:10D220001FD1574B1B68574A0021D154564B1A68DF
:10D230001346DB009B1ADB00544A13449C1D5148E3
:10D240002CF0BEFC034620464E491A462CF007FD42
:10D250004D4B1B6801334C4A13604D4B01221A6041
:10D2600075E0474B1B68454A1178464AD154444BF8
:10D270001B680133424A136069E0404B1B785BB284
:10D280002C2B04D03D4B1B785BB27D2B3CD13C4B0F
:10D290001B683C4A0021D1543B4B1A681346DB0003
:10D2A0009B1ADB00394A13440633184635492CF0E3
:10D2B00067FC354B1B680133334A13602F4B1B78D7
:10D2C0005BB22C2B02D1324B01221A602B4B1B7804
:10D2D0005BB27D2B17D12F4B1B68013B2D4A13608E
:10D2E0002C4B1B68002B06D12B4B01229A77284B25
:10D2F0006FF002021A60274B1B68002B03DD244BE2
:10D3000001221A600CE00BE01D4B1B681B4A1178D0
:10D310001C4AD1541A4B1B680133194A136016E09A
:10D3200015E0164B1B785BB27D2B0FD1194B1B6898
:10D33000013B184A1360174B1B68002B06D1164B94
:10D3400001229A77124B6FF002021A6000BF0E4B57
:10D350001B68302B06DD0C4B00221A600C4B0022A0
:10D360001A6007E0FB680133FB60FA683B689A4289
:10D37000FFF602AE1437BD4690BD00BF5C01001041
:10D3800070010010BC0100106C0100100839001081
:10D390001000001098010010A027001080B590B078
:10D3A00000AF03460A46FB711346BB7107F1080341
:10D3B0002348194601F03AF800F048F87B69DAB2E0
:10D3C000204B1A703B6ADAB21E4B5A707B6ADBB292
:10D3D0003033DAB21B4B9A703B69DAB2194BDA7010
:10D3E000FB68DAB2174B1A71164AFB795371154A6A
:10D3F000BB7993710723BB87002387F83F30114B1C
:10D40000BB63002387F83F300DE097F83F3097F873
:10D410003F20B96B0A4411780B4AD15497F83F303A
:10D42000013387F83F3097F83F309BB2BA8F9A426A
:10D43000EBD8F7F7F9FBF7F7D3FA4037BD4680BDD5
:10D4400000400240102700100003001080B483B099
:10D4500000AF0723BB804FF47A737B807B88013B4E
:10D46000FB800AE0FB88F988BA888A1A0749895C38
:10D47000064AD154FB88013BFB80FA88BB889A425C
:10D48000F0D20C37BD465DF8047B704700030010F6
:10D4900080B592B000AF78600B467B800723A7F879
:10D4A0004230002387F84730604BFB630023A7F826
:10D4B00044307B88B7F8422002FB03F3A7F84430DE
:10D4C000002387F8473011E097F84730FA6B1A4489
:10D4D000B7F84430591CA7F844101946544B5B5C0C
:10D4E000137097F84730013387F8473097F8473083
:10D4F0009BB2B7F842209A42E6D84C4B1B781A46AA
:10D5000007F10C03104619460A222CF06DF97B7BBB
:10D51000002B07D03A7B7B681A707B6801337A7BDB
:10D520001A7006E07B6830221A707B6801333A7B00
:10D530001A707B6802332D221A703C4B5B781A46B6
:10D5400007F10C03104619460A222CF04DF97B7B9B
:10D55000002B08D07B6803333A7B1A707B68043356
:10D560007A7B1A7007E07B68033330221A707B687D
:10D5700004333A7B1A707B6805332D221A702B4BCB
:10D580009B7803F5FA6207F10C03104619460A224C
:10D590002CF02AF97B6806333A7B1A707B680733D4
:10D5A0007A7B1A707B680833BA7B1A707B68093300
:10D5B000FA7B1A707B680A3320221A701B4BDB78C7
:10D5C0001A4607F10C03104619460A222CF00CF9F2
:10D5D0007B7B002B08D07B680B333A7B1A707B680F
:10D5E0000C337A7B1A7007E07B680B3330221A7099
:10D5F0007B680C333A7B1A707B680D333A221A70C1
:10D600000A4B1B791A4607F10C03104619460A22E9
:10D610002CF0EAF87B7B002B0CD07B680E333A7B36
:10D620001A707B680F337A7B1A700BE0581E00105B
:10D63000000300107B680E3330221A707B680F33B2
:10D640003A7B1A707B68103320221A707A4B5B7910
:10D650000D2B05D107F10C031846582129F094FC35
:10D66000754B5B790A2B05D107F10C0318465E2137
:10D6700029F08AFC704B5B79092B05D107F10C036B
:10D680001846592129F080FC6B4B5B79082B05D19A
:10D6900007F10C0318465B2129F076FC664B5B7999
:10D6A000062B05D107F10C031846562129F06CFC16
:10D6B000614B5B79072B05D107F10C0318465F21FD
:10D6C00029F062FC5C4B5B790B2B05D107F10C0355
:10D6D00018465C2129F058FC574B5B790C2B05D17F
:10D6E00007F10C0318465D2129F04EFC524B5B7983
:10D6F000112B05D107F10C031846DC2129F044FC5D
:10D700004D4B5B79012B05D107F10C031846922193
:10D7100029F03AFC484B5B79002B05D107F10C034B
:10D720001846912129F030FC434B5B79022B05D13F
:10D7300007F10C031846572129F026FC3E4B5B7974
:10D74000052B05D107F10C031846542129F01CFCC8
:10D75000394B5B79042B05D107F10C031846552191
:10D7600029F012FC344B5B79032B05D107F10C0334
:10D770001846932129F008FC2F4B5B790E2B05D11D
:10D7800007F10C031846672129F0FEFB2A4B5B7951
:10D790000F2B05D107F10C031846672129F0F4FB84
:10D7A000254B5B79102B05D107F10C031846D421CA
:10D7B00029F0EAFB002387F8473012E097F847305A
:10D7C00011331A467B68134497F8472007F1480144
:10D7D0000A4412F83C2C1A7097F84730013387F846
:10D7E000473097F8473007F14802134413F83C3CA0
:10D7F000002BE3D197F8473011331A467B68134466
:10D8000000221A700C4B9B7803F5FA6340F2DD722C
:10D81000934207DD084B9B7803F5FA6340F602025A
:10D82000934206DD7B6800221A707B680133002278
:10D830001A704837BD4680BD581E001080B485B0B0
:10D8400000AF07233B810023FB73234B7B60002346
:10D85000BB810023BB812EE000237B81BB893A89F9
:10D8600002FB03F37B810023FB730CE0FB7B7A68F4
:10D870001A447B89591C79811946184B5B5C1370DB
:10D88000FB7B0133FB73FB7B9BB23A899A42EDD859
:10D89000114B9B7803F5FA6340F2DD72934213DD7E
:10D8A0000D4B9B7803F5FA6340F6020293420BDCC2
:10D8B000BB890133BB813B894FF47A72B2FBF3F32E
:10D8C0009BB2BA899A42C7D3BB8918461437BD4662
:10D8D0005DF8047B704700BF581E00100003001065
:10D8E00080B485B000AF0723BB810023FB720B4BD4
:10D8F0007B600023FB810023FB8106E0FB89084A53
:10D900000021D154FB890133FB81FB89B3F57A7F78
:10D91000F4D31437BD465DF8047B7047581E0010E1
:10D920000003001080B485B000AF786039607B6878
:10D930001F2B02D97B68203B00E07B68FB607B6883
:10D940001F2B17D81949194BD3F8A831FA680320AF
:10D9500000FA02F2D2431340C1F8A8311348134B26
:10D96000D3F8A821FB68396801FA03F31343C0F820
:10D97000A83116E00D490D4BD3F8AC31FA680320FD
:10D9800000FA02F2D2431340C1F8AC310748074B0A
:10D99000D3F8AC21FB68396801FA03F31343C0F8EC
:10D9A000AC311437BD465DF8047B704700C00F40B2
:10D9B00080B485B000AF78607B681F2B06D87B6889
:10D9C000FB600D4BD3F8A831BB6006E07B68203BC1
:10D9D000FB60094BD3F8AC31BB60FB68BA6822FA34
:10D9E00003F303F00303BB60BB6818461437BD465E
:10D9F0005DF8047B704700BF00C00F4080B584B065
:10DA000000AF7860154B1B68BB607868FFF7D0FFEC
:10DA1000F860FB68032B17D801A252F823F000BF6F
:10DA200031DA000037DA00003DDA000043DA0000A6
:10DA30000423FB6008E00123FB6005E00223FB6098
:10DA400002E00823FB6000BFBA68FB68B2FBF3F397
:10DA5000BB60BB6818461037BD4680BD2000001073
:10DA600080B483B000AF78600B46FB70FB78012B6D
:10DA70000AD10F480E4BD3F8C42079680D4B0B40E8
:10DA80001343C0F8C4300DE0FB78002B0AD10849DD
:10DA9000074BD3F8C4207B68DB431A40054B134087
:10DAA000C1F8C4300C37BD465DF8047B704700BF39
:10DAB00000C00F40DEF7EFEF80B483B000AF034645
:10DAC000FB71084997F907305B09FA7902F01F02E8
:10DAD000012000FA02F241F823200C37BD465DF820
:10DAE000047B704700E100E080B483B000AF0346E0
:10DAF000FB71094997F907305B09FA7902F01F02B7
:10DB0000012000FA02F2203341F823200C37BD46F1
:10DB10005DF8047B704700BF00E100E080B483B093
:10DB200000AF78607B680C4A934201D100230DE07E
:10DB30007B680A4A934201D1012307E07B68084AC7
:10DB4000934201D1022301E04FF0FF3318460C3716
:10DB5000BD465DF8047B704700C0014000C0054031
:10DB600000000A4080B483B000AF78607B68082270
:10DB70009A617B6820221A6000BF7B681B6803F0F3
:10DB80000803002BF9D07B6820229A617B685B68D0
:10DB900003F0F80318460C37BD465DF8047B704768
:10DBA00080B483B000AF78607B681B6803F020030B
:10DBB000002B02D07B6820229A617B6810221A60B9
:10DBC0007B6808229A610C37BD465DF8047B70477C
:10DBD00080B483B000AF78600B46FB707B681B6835
:10DBE00003F02003002B02D07B6820229A61FA7890
:10DBF0007B689A607B6808229A6100BF7B681B681B
:10DC000003F00803002BF9D07B685B6803F0F8038E
:10DC100018460C37BD465DF8047B704780B485B06C
:10DC200000AFF860B9601346FB71FB79012B03D19B
:10DC3000FB6804221A6002E0FB6804229A61FB6818
:10DC400008229A6100BFFB681B6803F00803002BE1
:10DC5000F9D0FB689B68DAB2BB681A70FB685B6836
:10DC600003F0F80318461437BD465DF8047B70478F
:10DC700080B584B000AF786039607B68184A934201
:10DC800008D10E20FFF7BAFE02463B68B2FBF3F361
:10DC9000FB6018E07B68134A934208D12620FFF707
:10DCA000ADFE02463B68B2FBF3F3FB600BE07B6822
:10DCB0000D4A934207D12620FFF7A0FE02463B689B
:10DCC000B2FBF3F3FB60FB685A087B681A617B6860
:10DCD0001B69FA68D21A7B685A611037BD4680BD4D
:10DCE00000C0014000C0054000000A4080B582B07D
:10DCF00000AF786039607B68194A934208D1802070
:10DD00000121FFF7ADFE0E200221FFF70BFE1CE004
:10DD10007B68144A934209D14FF400200121FFF798
:10DD20009FFE26200221FFF7FDFD0EE07B680E4AD4
:10DD3000934209D14FF080600121FFF791FE34201A
:10DD40000221FFF7EFFD00E006E078683968FFF791
:10DD50008FFF7B6864229A610837BD4680BD00BF93
:10DD600000C0014000C0054000000A4080B483B0FC
:10DD700000AF78600B46FB70FB78012B03D17B680A
:10DD800040221A6002E07B6840229A610C37BD464F
:10DD90005DF8047B704700BF80B582B000AF78604B
:10DDA0000B46FB70FB78002B17D07B68184A934218
:10DDB00003D10A20FFF780FE26E07B68154A9342D4
:10DDC00003D10B20FFF778FE1EE07B68124A9342D6
:10DDD0001AD10C20FFF770FE17E07B680C4A9342C3
:10DDE00003D10A20FFF780FE0EE07B68094A9342C8
:10DDF00003D10B20FFF778FE06E07B68064A9342CA
:10DE000002D10C20FFF770FE00BF0837BD4680BD71
:10DE100000C0014000C0054000000A4080B588B045
:10DE200000AFF860B9601346FB71BB685B68FB61CB
:10DE3000BB681B69BB61BB680022DA60BB6800225B
:10DE40009A61BB6800225A62FB79002B40F029815D
:10DE5000BB6800221A62BB685B68FB61BB681B6918
:10DE6000BB61BB680022DA60BB6800229A610023B4
:10DE70007B61F868FFF776FE78617B69082B12D02A
:10DE80007B69102B0FD0BB681B6A5A1CBB681A62D7
:10DE9000BB681A6ABB68DB699A4203D9BB687A69B6
:10DEA0005A62F9E0D7E7BB689B68002B4DD0BB688E
:10DEB0005B68002B49D0BB681B68DBB25B00DBB240
:10DEC000F8681946FFF784FE78617B69182B11D03A
:10DED000BB681B6A5A1CBB681A62BB681A6ABB68BB
:10DEE000DB699A4205D97B6943F40072BB685A62C8
:10DEF000D2E0B0E723E0FB691B78F8681946FFF72A
:10DF000067FE78617B69282B11D0BB681B6A5A1C9D
:10DF1000BB681A62BB681A6ABB68DB699A4205D99A
:10DF20007B6943F40072BB685A62B5E093E7FB6912
:10DF30000133FB61BB68DB685A1CBB68DA60BB68F5
:10DF4000DA68BB689B689A42D5D3BB689B68002B94
:10DF500025D0BB685B68002B21D0BB685B69002BB8
:10DF60001DD0BB681B69002B19D0F868FFF7FAFDBC
:10DF700078617B69082B12D07B69102B0FD0BB68AE
:10DF80001B6A5A1CBB681A62BB681A6ABB68DB69E9
:10DF90009A4203D9BB687A695A627DE05BE7BB6845
:10DFA0005B69002B73D0BB681B69002B6FD0BB680B
:10DFB0001B68DBB25B00DBB243F00103DBB2F86845
:10DFC0001946FFF705FE78617B69402B11D0BB68CD
:10DFD0001B6A5A1CBB681A62BB681A6ABB68DB6999
:10DFE0009A4205D97B6943F40072BB685A6253E0D8
:10DFF00031E746E0BB689A69BB685B69013B9A42BE
:10E000001AD207F11303F86819460122FFF706FE3A
:10E0100078617B69502B2AD0BB681B6A5A1CBB688D
:10E020001A62BB681A6ABB68DB699A4203D9BB688B
:10E030007A695A6230E00EE707F11303F86819466F
:10E040000022FFF7EBFD78617B69582B0FD0BB688E
:10E050001B6A5A1CBB681A62BB681A6ABB68DB6918
:10E060009A4203D9BB687A695A6215E0F3E6BB6944
:10E070005A1CBA61FA7C1A70BB689B695A1CBB684F
:10E080009A61BB689A69BB685B699A42B2D3F868C7
:10E09000FFF786FD012326E0F868FFF781FD0023E6
:10E0A00021E0FB79012B1DD1F868FFF737FD03460E
:10E0B000DBB2FB74FB7C1946BB680D4A42F8313079
:10E0C000FB7C0B4ADB00134400225A60FB680822E9
:10E0D0009A61FB6820221A60F8680121FFF75CFE54
:10E0E000012300E0002318462037BD4680BD00BF55
:10E0F000F001001080B487B000AF0346FB710B46FF
:10E10000BB7113467B71BB797B61FB795B003B6123
:10E11000174BFB607B690F2B05D97B69103B7B613B
:10E120003B6901333B613B699B00FA6813443A69E0
:10E130009200F9680A4411687A6952001046032275
:10E140008240D2430A401A603B699B00FA6813443C
:10E150003A699200F9680A4411687A79786940004E
:10E1600082400A431A601C37BD465DF8047B704745
:10E1700000C0024080B487B000AF0346FB710B467D
:10E18000BB7113467B71BB797B61FB795B003B61A3
:10E19000174BFB607B690F2B05D97B69103B7B61BB
:10E1A0003B6901333B613B699B00FA6813443A6960
:10E1B0009200F9680A4411687A69520010460322F5
:10E1C0008240D2430A401A603B699B00FA681344BC
:10E1D0003A699200F9680A4411687A7978694000CE
:10E1E00082400A431A601C37BD465DF8047B7047C5
:10E1F00040C0024080B485B000AF0346FB710B46BF
:10E20000BB7113467B71154BFB607B79012B0FD1E2
:10E21000FB799B00FA681344FA799200F9680A4482
:10E220001168BA79012000FA02F20A431A600FE07D
:10E23000FB799B00FA681344FA799200F9680A4462
:10E240001168BA79012000FA02F2D2430A401A603A
:10E250001437BD465DF8047B704700BF68C00240BC
:10E2600080B582B000AF78607B6819787B685A7897
:10E270007B689B78084611461A46FFF73BFF7B6890
:10E2800019787B685A787B68DB78084611461A460D
:10E29000FFF770FF7B6819787B685A787B681B7979
:10E2A000084611461A46FFF7A5FF0837BD4680BD50
:10E2B00080B582B000AF78604FF400700121FFF7A5
:10E2C000CFFB7B6800221A707B6800221A727B6881
:10E2D00000221A737B68FF221A747B6800221A647A
:10E2E0000837BD4680BD00BF80B483B000AF786002
:10E2F0007B681B7ADBB243F00203DAB27B681A72E6
:10E300007B681B7ADBB203F01103DAB27B681A7206
:10E310000C37BD465DF8047B704700BF80B483B006
:10E3200000AF78600B46FB70FB78012B08D17B684F
:10E330001B7ADBB243F00103DAB27B681A7207E0A2
:10E340007B681B7ADBB203F01203DAB27B681A72C5
:10E350000C37BD465DF8047B704700BF80B485B0C4
:10E3600000AFF860B9607A60BB68072B58D801A28B
:10E3700052F823F095E30000A7E30000B9E30000A2
:10E38000CBE30000DDE30000EFE30000FFE300006B
:10E3900011E400007B68DBB203F03F03DAB2FB68F4
:10E3A00083F820203CE07B68DBB203F03F03DAB265
:10E3B000FB6883F8242033E07B68DBB203F01F03A3
:10E3C000DAB2FB6883F828202AE07B68DBB203F02E
:10E3D0000703DAB2FB6883F8302021E07B68DBB208
:10E3E00003F01F03DAB2FB6883F82C2018E07B6887
:10E3F0009BB2C3F308039AB2FB689A8610E07B686D
:10E40000DBB203F00F03DAB2FB6883F8382007E0D1
:10E410007B689BB2C3F30B039AB2FB689A8700BF79
:10E420001437BD465DF8047B704700BF80B483B0ED
:10E4300000AF786039607B6893F82C30DBB203F072
:10E440001F023B68DA607B6893F83030DBB203F080
:10E4500007023B681A617B689B8E9BB2C3F308027C
:10E460003B685A617B6893F82830DBB203F01F02E7
:10E470003B689A607B6893F82430DBB203F03F027C
:10E480003B685A607B6893F82030DBB203F03F02B0
:10E490003B681A607B6893F83830DBB203F00F02F8
:10E4A0003B689A617B689B8F9BB2C3F30B023B680E
:10E4B000DA610C37BD465DF8047B704780B483B0E9
:10E4C00000AF78600B46FB70FB78012B08D17B68AE
:10E4D0001B7ADBB203F00303DAB27B681A7207E03F
:10E4E0007B681B7ADBB243F01003DAB27B681A72E6
:10E4F0000C37BD465DF8047B704700BF80B400AFA9
:10E5000062B6BD465DF8047B704700BF80B400AFC3
:10E5100072B6BD465DF8047B704700BF80B584B01D
:10E5200000AF03463960FB710023FB600023BB6032
:10E53000FB79012B1AD0022B69D0002B00D07DE093
:10E54000414BFB60FB68414AA2FB03239B0C3A68EA
:10E55000920802FB03F3BB60BB68FE2B05D94FF0AA
:10E560008042BB685360012369E067E0384B1B6859
:10E570009B08FB60FB68354AA2FB03239B0C3A68AF
:10E58000920802FB03F3BB60BB68FE2B09D9002095
:10E590000021FFF7C7F94FF08042BB6853600123A9
:10E5A0004DE02B4B1B685B08FB60FB68274AA2FB16
:10E5B00003239B0C3A68920802FB03F3BB60BB6821
:10E5C000FE2B09D900200221FFF7ACF94FF0804261
:10E5D000BB685360012332E01D4B1B68FB60FB6886
:10E5E0001A4AA2FB03239B0C3A68920802FB03F32E
:10E5F000BB60BB68FE2B09D900200121FFF792F90F
:10E600004FF08042BB685360012318E016E04FF4DE
:10E610000043FB60FB680D4AA2FB03239B0C3A6896
:10E62000920802FB03F3BB60BB68FE2B05D94FF0D9
:10E630008042BB685360012301E000BF00231846FD
:10E640001037BD4680BD00BF00093D0083DE1B437F
:10E650002000001080B582B000AF03460A46FB716F
:10E660001346BB7100200021FFF75CF94FF0804298
:10E670004FF080431B6923F0030313614FF0804187
:10E680004FF080431A69FB7913430B61BB79012B6F
:10E6900009D14FF080424FF080431B78DBB243F04A
:10E6A0000203DBB213700837BD4680BD80B584B06D
:10E6B00000AF78604FF080431B69FB60FB6803F09C
:10E6C0000303FB60FB68DBB218467968FFF726FF9F
:10E6D0004FF080424FF080431B78DBB243F00103E0
:10E6E000DBB2137000F004F81037BD4680BD00BFE8
:10E6F00080B500AFFFF70AFF4FF08043AA221A72DD
:10E700004FF0804355221A72FFF7F8FE80BD00BF1C
:10E7100080B483B000AF0346FB71094997F9073015
:10E720005B09FA7902F01F02012000FA02F220339D
:10E7300041F823200C37BD465DF8047B704700BFCD
:10E7400000E100E080B483B000AF03463960FB71A4
:10E7500097F90730002B0BDA0D49FB7903F00F0313
:10E76000043B3A68D2B2D200D2B20B441A7609E026
:10E77000084997F907303A68D2B2D200D2B20B44B6
:10E7800083F800230C37BD465DF8047B704700BF5B
:10E7900000ED00E000E100E080B500AF00F066F9B8
:10E7A000804B00221A70804B9B78002B0DD0FFF716
:10E7B0009FFF7E4B93F85F30002B01D005F016FDD4
:10E7C00000F006F9784B00229A70774B9B7B002B68
:10E7D0002CD0774B1B78012B03D1754B00221A707C
:10E7E00002E0734B01221A706E4B5B79002B12D141
:10E7F0006E4B9B78042B0ED06E4B1B7D002B03D0F1
:10E8000000200AF051FB0CE06B4B00225A726A4B5D
:10E8100000221A7205E0684B00225A72664B0022F1
:10E820001A7200F0B9FA604B00229A735E4B9B7A21
:10E83000002B04D001F0AAFD5B4B00229A725A4BC8
:10E84000DB7A002B04D000F0F5FC574B0022DA7283
:10E85000554BDB78002B09D005F072FB02F090FFDE
:10E86000514BDB78013BDAB24F4BDA704E4B1B79E0
:10E87000002B0FD04D4B93F85F30002B02D10520B9
:10E88000F8F7CCFA03F002F8474B1B79013BDAB2F8
:10E89000454B1A71444B1B7A002B07D001F09CFDAD
:10E8A000414B1B7A013BDAB23F4B1A723E4B5B7B0A
:10E8B000002B0FD0F6F72EFAF6F712FA3F48F6F7CC
:10E8C0009BFA3F4B01221A72374B5B7B013BDAB25A
:10E8D000354B5A73344BDB79002B07D001F004FE23
:10E8E000314BDB79013BDAB22F4BDA712E4B9B793E
:10E8F000002B07D001F076FD2B4B9B79013BDAB260
:10E90000294B9A71284B5B7A002B04D002F032FF1E
:10E91000254B00225A72244B5B79002B10D0294AD8
:10E92000284B9B6943F40073936100F035FA254A44
:10E93000244BDB6943F40073D3611B4B00225A71F3
:10E94000194B5B78002B04D002F09AFE164B002284
:10E950005A70154B1B7B002B04D000F071FC124B3E
:10E9600000221A730F4B9B7F012B0AD1164B1B7889
:10E97000002B03D005F0EEFDF9F7C4FC094B002293
:10E980009A77084B5B7F012B0AD1104B1B78002B29
:10E9900003D003F075FBF6F7F1F9024B00225A772A
:10E9A00001E700BFA0270010941E001020270010D0
:10E9B0002C02001004070010300A0010A8A6040062
:10E9C0002C22001000C00920083900103C2800103B
:10E9D00080B400AF204B9B7D002B15D01F4A1F4BEE
:10E9E0009B6943F4002393611B4B9B7D013BDAB28F
:10E9F000194B9A75184B9B7D002B05D1174A174B65
:10EA0000DB6943F40023D361154B5B7C012B08D1F8
:10EA1000124A124B9B6943F4002393610E4B01226F
:10EA20009A75104B1B68002B09D00F4A0E4B9B693F
:10EA300043F0800393610B4B00221A6008E00A4AFE
:10EA4000094BDB6943F08003D361064B01221A6056
:10EA5000BD465DF8047B7047A027001000C0092068
:10EA6000140A00103002001040C0092080B582B0A6
:10EA700000AF28F009FE05200021FFF763FE01200A
:10EA80000121FFF75FFE02200221FFF75BFE00205D
:10EA90000121FFF7DFFD9848FFF708FEFFF728FE8A
:10EAA000964A964B1B6923F440431361944A944B56
:10EAB0001B6843F098031360924A924B1B6843F41F
:10EAC000002343F4407313608E4A8E4B1B6843F45B
:10EAD000003313608B4A8B4B1B6843F07003136049
:10EAE000002001F01BF9874A864B9B6943F4002301
:10EAF0009361854801F054FC824A824BDB6943F400
:10EB00000023D361F5F7BCFE00F02CF901F02AFCDC
:10EB100000204FF461412AF0E1FB01204FF4E13184
:10EB20002AF0DCFB794B00221A6002F08DFE784A55
:10EB3000774B1B6823F0806313600AF0DDF8F5F76C
:10EB400067FE28F0B9F947F2305001F029FCF1F7DF
:10EB5000C9FCF6F743F8F5F7B3FFF5F7E5FF01F069
:10EB6000CFFCF6F797F86B4B5B7F6B481946F1F7D4
:10EB7000F7FA6A48FF21F1F7F3FA694B1B68694A13
:10EB8000D360694BB3F8B821664B1A80614B5B6860
:10EB900066481946F1F744FB5E4B9B68644819468A
:10EBA000F1F73EFB5B4BDB6862481946F1F738FB37
:10EBB000584B1B6960481946F1F732FB554B5B69AE
:10EBC0005E481946F1F72CFB524B9B695C4819468D
:10EBD000F1F726FB544B9B78002B0ED1594B0022AA
:10EBE0009A71504B04229A704B480021F1F7B8FA01
:10EBF0004A480021F1F7B4FA11E04B4B93F8173271
:10EC0000002B06D1474B00229A704E4B00229A717E
:10EC100005E0444B02229A704A4B01229A71F4F7A4
:10EC200021FE404B002283F85020464B00225A73AD
:10EC3000444B00221A73434B0022DA73414B0022EB
:10EC40001A740023FB800023FB8014E0FB883E4AFB
:10EC5000002122F81310FB883B4A03F5347300218E
:10EC600022F81310FB88384A1344002283F8402B03
:10EC7000FB880133FB80FB88B3F5347FE6D32A4B56
:10EC800093F82930022B02D1274B00229A72254B90
:10EC9000002283F85E20244B2C4AC3F85C22224BCE
:10ECA0002B4AC3F86022204B2A4AC3F864221E4B29
:10ECB000264AC3F86822284B00225A72264B0022AB
:10ECC0001A72254B00221A75234B00225A75234BCA
:10ECD0000022DA62214B00225A62204B00229A6203
:10ECE0001E4B00221A621D4B01221A751C4B00227A
:10ECF0001A600837BD4680BD002D310100C00240BA
:10ED000040C0092000C00920A0860100EC020010CC
:10ED100020C00920641E0010C4241000902410009C
:10ED20001C1E001020270010040700101C251000D6
:10ED30002025100024251000282510002C25100067
:10ED400030251000A0270010480A00100000A04144
:10ED50000000404100002041300A0010F421001062
:10ED6000FC02001080B500AF0A48FFF7A1FA11209D
:10ED7000FFF7CEFC11200921FFF7E4FC0548FFF75F
:10ED8000B3FA04480121FFF7C9FA02480021FFF74E
:10ED900095FB80BD0040024080B588B000AF4FF0C9
:10EDA0000003BB61984B5B79002B04D0974B9B68A9
:10EDB000974A136003E0954B5B68954A1360944B48
:10EDC0001B68002B03DC914B00221A6102E08F4B81
:10EDD00001221A618D4B1B69012B06D18D4B1B68DB
:10EDE000002B02D18C4B0A221A608B4B1B68002B24
:10EDF00004D0894B1B68013B874A136032237B6137
:10EE000078692CF01FF80346184684492BF0B6FEAB
:10EE100003463B617E4B1B6818462CF013F80346F3
:10EE2000184639692BF04CFE034618462BF0DCFFE0
:10EE30000346C3F15A03FB60774B1B68002B03D0DA
:10EE4000724B3C22DA6002E0704AFB68D3606F4B81
:10EE5000DB685A2B02DD6D4B5A22DA606B4BDB68A4
:10EE6000272B02DC694B2822DA60684B1B69694A50
:10EE700013600023FB776A4B1B7A002B02D0684B90
:10EE800000225A72664B5B7A002B02D0644B002240
:10EE90001A72634B9B7C002B02D0614B0022DA7408
:10EEA0005F4BDB7C002B02D05D4B00229A745C4BE5
:10EEB000DA795B4B9A71544B5B79002B3BD1584B01
:10EEC0001B78002B03D0FB7F43F00103FB77544BEF
:10EED0009B78002B03D0FB7F43F00203FB77504B62
:10EEE0005B7A002B03D0FB7F43F00403FB774C4B92
:10EEF0001B7A002B03D0FB7F43F00803FB77484BC2
:10EF0000DB79002B03D0FB7F43F01003FB77444BEE
:10EF10005B78002B03D0FB7F43F02003FB77404B53
:10EF2000DB78002B03D0FB7F43F04003FB773C4BA7
:10EF30009B79002B53E03A4B1B78002B03D1384BC5
:10EF40009B7A002B03D0FB7F43F00103FB77344B0C
:10EF50009B78002B03D1324B1B7B002B03D0FB7F14
:10EF600043F00203FB772E4B5B7A002B03D12C4B33
:10EF7000DB7C002B03D0FB7F43F00403FB77284BA3
:10EF80001B7A002B03D1264B9B7C002B03D0FB7FED
:10EF900043F00803FB77224BDB79002B03D1204B96
:10EFA0005B7C002B03D0FB7F43F01003FB771C4BF3
:10EFB0005B78002B03D11A4BDB7A002B03D0FB7F4D
:10EFC00043F02003FB77164BDB78002B03D1144B67
:10EFD0005B7B002B03D0FB7F43F04003FB77FB7F81
:10EFE000184600F09BFE0F4B9B78002B1ED10E4A5B
:10EFF0000D4B9B6943F0080393610B4A0A4BDB6995
:10F0000043F01003D3611DE0A02700104022001040
:10F01000380200103C020010400200100000C842FC
:10F02000300A00100407001040C00920794A794BCB
:10F03000DB6943F00803D361764A764B9B6943F062
:10F0400010039361734B5B6903F02003BB60BB68E3
:10F05000202B03D0704B00221A7002E06E4B01226D
:10F060001A706C4B5B6903F00403BB60BB68042B34
:10F0700003D0694B00225A7002E0674B01225A709C
:10F08000664B5B6903F08063BB60BB68B3F1806F64
:10F0900003D0614B0022DA7002E05F4B0122DA708C
:10F0A0005F4B5B6903F08063BB60BB68B3F1806F4B
:10F0B00009D05C4B1B68002B0EDB5A4B1B68013BD5
:10F0C000584A136008E0574B1B68002B04DC554B73
:10F0D0001B680133534A1360524B1B68002B02DD3F
:10F0E0004D4B01229A704F4B1B68002B02DA4A4BA2
:10F0F00000229A704C4B1B7A002B03D14A4B9B7C0D
:10F10000002B01D0012300E00023FB71464B5B7A0A
:10F11000002B03D1444BDB7C002B01D0012300E00A
:10F120000023BB71404B1B7D002B06D1FB79002BCC
:10F1300003D03E4B1B683E4A13623B4B1B7D002BAA
:10F1400010D0FB79002B0DD1384B1B68384A536225
:10F15000374BDA69364B596A354B1B6ACB1A134465
:10F16000334AD361304B5B7D002B06D1BB79002B3A
:10F1700003D02E4B1B682E4A93622B4B5B7D002BDA
:10F1800010D0BB79002B0DD1284B1B68284AD362C5
:10F19000274BDA69264B996A254BDB6ACB1A134455
:10F1A000234AD361224B1B7D002B02D0204B01222E
:10F1B0005A751D4B1B7D002B23D1FB79002B20D1D1
:10F1C000194B5B7D002B1CD1BB79002B19D1184B3F
:10F1D0005B7D002B15D0164B4FF00002DA60144B0C
:10F1E0000022DA61124B00221A62114B00225A628D
:10F1F0000F4B00229A620E4B0022DA620C4B002267
:10F200005A75094AFB791375074ABB79537520373C
:10F21000BD4680BD40C009209827001000C00920CD
:10F2200060C0092044020010300A0010542200106F
:10F23000F421001080B500AF0CF0FEFD80BD00BFD2
:10F2400080B582B000AF00237B60374B5B6903F071
:10F2500080637B60354B1B78002B05D0344B1B78CB
:10F260000133DAB2324B1A70314B1B78642B05D95B
:10F270002E4B00221A702E4B00221A707B68B3F1BD
:10F28000806F4AD02B4B1B780133DAB2294B1A70AE
:10F29000294B5B7F29481946F0F762FF2848FF2178
:10F2A000F0F75EFF234B1B78012B39D11F4B1B78E6
:10F2B0000133DAB21D4B1A701C4B1B780A2B0DD18F
:10F2C000204B0B221A701D488021F0F749FF1C4883
:10F2D000FF21F0F745FF154B00221A70194B1B78E0
:10F2E0000B2B1DD0174B00225A71174B00229A602E
:10F2F000164B00229A74154B0022DA74114B1B78BE
:10F30000002B03D0124B9B78002B02D119F014F97B
:10F3100006E00C4B00221A7002E0064B00221A7025
:10F320000837BD4680BD00BF20C009205002001034
:10F330005102001052020010641E0010C42410007C
:10F3400090241000A027001040220010300A001066
:10F350000407001090B585B000AF0023FB600023C8
:10F360007B818E4B1B68002B00F0F580002009F09C
:10F37000DFFCF86000237B8110E07C89FB68184685
:10F38000F1F7F2FC034618462BF02EFD0146844AA5
:10F390002301134419607B8901337B817B89312BE5
:10F3A000EBD9012009F0C4FCF86000237B8112E056
:10F3B0007C89FB681846F1F71DFC034618462BF0C4
:10F3C00013FD034699B2764A230113440A469A80F4
:10F3D0007B8901337B817B89312BE9D9022009F0BC
:10F3E000A7FCF86000237B8112E07C89FB6818464B
:10F3F000F1F700FC034618462BF0F6FC034699B2E1
:10F40000674A230113440A46DA807B8901337B81F2
:10F410007B89312BE9D9032009F08AFCF8600023AD
:10F420007B8113E07C89FB681846F1F7E3FB034618
:10F4300018462BF0D9FC034699B2594A23011344CC
:10F4400008330A469A807B8901337B817B89312B83
:10F45000E8D9042009F06CFCF86000237B8113E0FC
:10F460007C89FB681846F1F7C5FB034618462BF06C
:10F47000BBFC034699B24A4A2301134408330A46A7
:10F480005A807B8901337B817B89312BE8D9454BBD
:10F4900093F87432002B04D1052009F049FCF86080
:10F4A00002E04FF4FA63FB6000237B8112E07C8969
:10F4B000FB681846F1F79EFB034618462BF094FCB8
:10F4C000034699B2384AA30013440A465A807B89FE
:10F4D00001337B817B89B3F5967FE8D3062009F061
:10F4E00027FCF86000237B8110E07C89FB681846CC
:10F4F000F1F780FB034618462BF076FC03469AB2E0
:10F50000294B23F824207B8901337B817B89B3F548
:10F51000967FEAD3072009F00BFCF86000237B817B
:10F5200013E07C89FB681846F1F764FB0346184634
:10F530002BF05AFC034699B2194A230113440833AD
:10F540000A461A807B8901337B817B89312BE8D97C
:10F55000124B00221A60002009F0EAFBF860134BFE
:10F560001C68FB681846F1F7FFFB034618462BF0B2
:10F570003BFC01460A4A2301134419600C4BDB781B
:10F58000002B19D00B4B93F82030DBB2DBB20133E8
:10F59000DBB2DAB2074B83F820201EE0180000101F
:10F5A000A41E0010040700105C220010540200107A
:10F5B000A0270010C4210010964B93F820305BB2B6
:10F5C000002B0ADD934B93F82030DBB2DBB2013B1A
:10F5D000DBB2DAB28F4B83F820208E4B93F82030C9
:10F5E0005BB2142B06DD8B4B01221A76894B142259
:10F5F00083F82020874B93F82030002B02D1854BD5
:10F6000000221A76012009F093FBF860824B1C68F7
:10F61000FB681846F1F7EEFA034618462BF0E4FBB8
:10F62000034699B27D4A230113440A469A807C4BD3
:10F63000DB78002B0BD0774B93F82130DBB2DBB2B9
:10F640000133DBB2DAB2734B83F8212010E0714B47
:10F6500093F821305BB2002B0ADD6E4B93F821301A
:10F66000DBB2DBB2013BDBB2DAB26A4B83F82120BA
:10F67000684B93F821305BB2142B06DD654B0122F9
:10F680005A76644B142283F82120624B93F8213080
:10F69000002B02D15F4B00225A76022009F048FB72
:10F6A000F8605D4B1C68FB681846F1F7A3FA034647
:10F6B00018462BF099FB034699B2584A230113448C
:10F6C0000A46DA80564BDB78002B0BD0514B93F86F
:10F6D0002230DBB2DBB20133DBB2DAB24D4B83F85E
:10F6E000222010E04B4B93F822305BB2002B0ADD56
:10F6F000484B93F82230DBB2DBB2013BDBB2DAB22B
:10F70000444B83F82220434B93F822305BB2142BF6
:10F7100006DD404B01229A763E4B142283F82220CC
:10F720003C4B93F82230002B02D13A4B00229A76C0
:10F73000032009F0FDFAF860374B1C68FB68184697
:10F74000F1F758FA034618462BF04EFB034699B2E0
:10F75000324A2301134408330A469A80304BDB783F
:10F76000002B0BD02B4B93F82730DBB2DBB20133ED
:10F77000DBB2DAB2274B83F8272010E0254B93F851
:10F7800027305BB2002B0ADD224B93F82730DBB227
:10F79000DBB2013BDBB2DAB21E4B83F827201D4BF4
:10F7A00093F827305BB2142B06DD1A4B0122DA776F
:10F7B000184B142283F82720164B93F82730002B80
:10F7C00002D1144B0022DA77042009F0B1FAF86074
:10F7D000114B1C68FB681846F1F70CFA03461846F3
:10F7E0002BF002FB034699B20C4A23011344083361
:10F7F0000A465A800A4BDB78002B13D0054B93F84E
:10F800002430DBB2DBB20133DBB2DAB2014B83F876
:10F81000242018E0C421001054020010A41E00107F
:10F82000A02700109B4B93F824305BB2002B0ADD1D
:10F83000984B93F82430DBB2DBB2013BDBB2DAB297
:10F84000944B83F82420934B93F824305BB2142B11
:10F8500006DD904B01221A778E4B142283F8242068
:10F860008C4B93F82430002B02D18A4B00221A775C
:10F87000894B93F87432002B0CD0884B0022DA703D
:10F88000874B1B68874A1188874A9B0013440A46A6
:10F890005A8014E0052009F04BFAF860804B1C6890
:10F8A000FB681846F1F7A6F9034618462BF09CFAB8
:10F8B000034699B27C4AA30013440A465A80774B08
:10F8C000DB78002B0BD0734B93F82630DBB2DBB226
:10F8D0000133DBB2DAB26F4B83F8262010E06D4BB8
:10F8E00093F826305BB2002B0ADD6A4B93F8263082
:10F8F000DBB2DBB2013BDBB2DAB2664B83F8262027
:10F90000644B93F826305BB2142B06DD614B012269
:10F910009A77604B142283F826205E4B93F82630AA
:10F92000002B02D15B4B00229A77062009F000FAE7
:10F93000F8605B4B1C68FB681846F1F75BF90346FF
:10F9400018462BF051FA03469AB2574B23F824205D
:10F95000524BDB78002B0BD04E4B93F82530DBB2AB
:10F96000DBB20133DBB2DAB24A4B83F8252010E078
:10F97000484B93F825305BB2002B0ADD454B93F8DA
:10F980002530DBB2DBB2013BDBB2DAB2414B83F8AC
:10F990002520404B93F825305BB2142B06DD3D4B00
:10F9A00001225A773B4B142283F82520394B93F8D8
:10F9B0002530002B02D1374B00225A77072009F05F
:10F9C000B7F9F860394B1C68FB681846F1F712F973
:10F9D000034618462BF008FA034699B2344A23012D
:10F9E000134408330A461A802C4BDB78002B0BD0CB
:10F9F000284B93F82330DBB2DBB20133DBB2DAB24F
:10FA0000244B83F8232010E0224B93F823305BB281
:10FA1000002B0ADD1F4B93F82330DBB2DBB2013B36
:10FA2000DBB2DAB21B4B83F823201A4B93F8233056
:10FA30005BB2142B06DD174B0122DA76154B14222C
:10FA400083F82320134B93F82330002B02D1114B62
:10FA50000022DA76154B1B680133144A1360134BEE
:10FA60001B68312B02DD114B00221A600C4B1B6806
:10FA700001330B4A13600A4B1B68B3F5967F02DB18
:10FA8000074B00221A6000237B6000237B60002369
:10FA90003B811AE0C421001004070010A0270010C9
:10FAA00058020010020700105C22001054020010DF
:10FAB000A41E00103B89934A1B0113441B687A68FB
:10FAC00013447B603B8901333B813B89312BF1D966
:10FAD0007B688D4A82FB03121211DB17D31A7B60FD
:10FAE0008A4A7B68536000237B6000233B810BE0E4
:10FAF0003B89844A1B0113449B881BB27A681344D8
:10FB00007B603B8901333B813B89312BF0D97B689A
:10FB10007D4A82FB03121211DB17D31A7B607B68CC
:10FB20009AB27A4B1A8100237B6000233B810BE061
:10FB30003B89744A1B011344DB881BB27A68134467
:10FB40007B603B8901333B813B89312BF0D97B685A
:10FB50006D4A82FB03121211DB17D31A7B606C4BC8
:10FB6000B3F87C329AB27B689BB213449BB29AB2D0
:10FB7000664B5A8100237B6000233B810CE03B896C
:10FB8000604A1B01134408335B881BB27A68134434
:10FB90007B603B8901333B813B89312BEFD97B680B
:10FBA000594A82FB03121211DB17D31A7B607B6860
:10FBB0009AB2564BDA8100237B6000233B810CE034
:10FBC0003B89504A1B01134408339B881BB27A6857
:10FBD00013447B603B8901333B813B89312BEFD957
:10FBE0007B68494A82FB03121211DB17D31A7B6030
:10FBF000474BB3F87E329AB27B689BB213449BB2F8
:10FC00009AB2424B9A8200237B6000233B810CE036
:10FC10003B893C4A1B01134408331B881BB27A689A
:10FC200013447B603B8901333B813B89312BEFD906
:10FC30007B68354A82FB03121211DB17D31A7B60F3
:10FC4000334BB3F87A329AB27B689BB213449BB2BF
:10FC50009AB22E4B9A8100237B6000233B810BE0FC
:10FC60003B892C4A9B0013445B881BB27A6813447F
:10FC70007B603B8901333B813B89B3F5967FEFD3B2
:10FC80007B68254A82FB03125211DB17D31A7B6073
:10FC90001F4BB3F876329AB27B689BB213449BB287
:10FCA0009AB21A4B5A8200237B6000233B810AE000
:10FCB0003B89184A32F823301BB27A6813447B60C0
:10FCC0003B8901333B813B89B3F5967FF0D37B6859
:10FCD000114A82FB03125211DB17D31A7B600C4BC3
:10FCE000B3F878329AB27B689BB213449BB29AB253
:10FCF000064B1A82054B9A8A044BDA821437BD46AA
:10FD000090BD00BFA41E00101F85EB51C421001040
:10FD1000040700105C220010B5814E1B80B584B032
:10FD200000AF0346FB71FB79FB730023BB73254ACD
:10FD3000244BDB6943F02003D361224A214BDB696A
:10FD400043F04003D3610023BB7325E0FB7B5BB230
:10FD5000002B06DA1B4A1B4B9B6943F0100393618F
:10FD600005E0184A174BDB6943F01003D361FB7BB6
:10FD70005B00FB73134A134B9B6943F020039361B1
:10FD8000022000F00DFB0F4A0E4BDB6943F020030D
:10FD9000D361BB7B0133BB73BB7B072BD6D9094A2D
:10FDA000084B9B6943F040039361022000F0F8FA8E
:10FDB000044A044BDB6943F04003D3611037BD466E
:10FDC00080BD00BF00C0092080B58EB000AF786054
:10FDD0000B46FB7007F10C033D481946FEF726FB66
:10FDE0007B691A4607F12C03104619460A2229F0AE
:10FDF000FBFC97F82D30002B09D097F82C207B685E
:10FE00001A707B68013397F82D201A7007E07B6821
:10FE100030221A707B68013397F82C201A707B68A7
:10FE200002333A221A703B691A4607F12C03104636
:10FE300019460A2229F0D8FC97F82D30002B0AD059
:10FE40007B68033397F82C201A707B68043397F88B
:10FE50002D201A7008E07B68033330221A707B680B
:10FE6000043397F82C201A707B6805333A221A70F5
:10FE7000FB78002B25D0FB681A4607F12C031046AF
:10FE800019460A2229F0B0FC97F82D30002B0AD031
:10FE90007B68063397F82C201A707B68073397F835
:10FEA0002D201A7008E07B68063330221A707B68B8
:10FEB000073397F82C201A707B68083300221A70D9
:10FEC00003E07B68053300221A703837BD4680BDD9
:10FED0000040024080B58EB000AF786007F10C039F
:10FEE00037481946FEF7A2FABB691A4607F12C03F8
:10FEF000104619460A2229F077FC97F82D30002B7E
:10FF000009D097F82C207B681A707B68013397F82A
:10FF10002D201A7007E07B6830221A707B6801334D
:10FF200097F82C201A707B6802332D221A707B6A96
:10FF30001A4607F12C03104619460A2229F054FCF0
:10FF400097F82D30002B0AD07B68033397F82C20CC
:10FF50001A707B68043397F82D201A7008E07B68CC
:10FF6000033330221A707B68043397F82C201A7000
:10FF70007B6805332D221A70BB6A1A4607F12C03E1
:10FF8000104619460A2229F02FFC7B68063397F8A1
:10FF90002C201A707B68073397F82D201A707B6825
:10FFA000083397F82E201A707B68093397F82F20B2
:10FFB0001A707B680A3300221A703837BD4680BD3C
:10FFC0000040024080B58EB000AF78600B46FB70F9
:10FFD00007F10C0339481946FEF728FA7B691A46DF
:10FFE00007F12C03104619460A2229F0FDFB97F869
:10FFF0002D30002B09D097F82C207B681A707B6875
:020000021000EC
:10000000013397F82D201A7007E07B6830221A70B0
:100010007B68013397F82C201A703B691A4607F168
:100020002C03104619460A2229F0DEFB97F82D30E2
:10003000002B0AD07B68023397F82C201A707B685B
:10004000033397F82D201A7008E07B6802333022C2
:100050001A707B68033397F82C201A70FB78002BFA
:1000600025D0FB681A4607F12C03104619460A22D0
:1000700029F0BAFB97F82D30002B0AD07B680433A7
:1000800097F82C201A707B68053397F82D201A708A
:1000900008E07B68043330221A707B68053397F8D8
:1000A0002C201A707B68063300221A7003E07B68EC
:1000B000043300221A703837BD4680BD004002402C
:1000C00080B58EB000AF786007F10C033A4819464E
:1000D000FEF7ACF9BB691A4607F12C031046194626
:1000E0000A2229F081FB97F82D30002B09D097F8D0
:1000F0002C207B681A707B68013397F82D201A70CA
:1001000007E07B6830221A707B68013397F82C2057
:100110001A707B6A1A4607F12C03104619460A2208
:1001200029F062FB97F82D30002B0AD07B68023350
:1001300097F82C201A707B68033397F82D201A70DB
:1001400008E07B68023330221A707B68033397F82B
:100150002C201A70BB6A1A4607F12C031046194668
:100160000A2229F041FB7B68043397F82C201A708F
:100170007B68053397F82D201A707B68063397F853
:100180002E201A707B68073397F82F201A70FB69AE
:100190001A4607F12C03104619460A2229F024FBBF
:1001A0007B68083397F82C201A707B68093300228B
:1001B0001A703837BD4680BD0040024080B58EB011
:1001C00000AF786007F1140325481946FEF72EF9B1
:1001D0007B681B783B737B685B787B730023BB7306
:1001E00007F10C03184629F0E7FB034687F8373080
:1001F00097F837301A4802211A46FEF7AFF87B68A5
:100200009B783B737B68DB787B730023BB7307F1C0
:100210000C03184629F0D0FB034687F8373097F8CF
:1002200037300F4801211A46FEF798F87B681B7992
:100230003B737B685B797B730023BB7307F10C0313
:10024000184629F0B9FB034687F8373097F837305E
:10025000034800211A46FEF781F83837BD4680BDB5
:100260000040024080B58EB000AF786007F1140303
:100270002E481946FEF7DAF87B681B783B737B68DB
:100280005B787B730023BB7307F10C03184629F0DE
:1002900093FB0346FB86FB8E244804211A46FEF797
:1002A0005DF87B689B783B737B68DB787B7300230E
:1002B000BB7307F10C03184629F07EFB0346FB864F
:1002C000FB8E1A4806211A46FEF748F87B681B7910
:1002D0003B737B685B797B737B689B79BB737B68C3
:1002E000DB79FB7300233B7407F10C03184629F0FC
:1002F00063FB0346FB86FB8E0C4807211A46FEF77C
:100300002DF87B681B7A3B7300237B7307F10C038A
:10031000184629F051FB0346FB86FB8E0348032158
:100320001A46FEF71BF83837BD4680BD0040024034
:1003300080B58EB000AF786007F10C03084819460D
:10034000FEF774F8FB69DBB27868194626F01CFEEC
:100350007B68023300221A703837BD4680BD00BF6B
:100360000040024080B500AF002040F6C41127F0E5
:100370006FFA002027F040FA0120034927F068FABD
:10038000012027F039FA80BD90D0030080B500AF7E
:10039000024B1B6818460EF0E3FB80BD28020010DC
:1003A00080B485B000AF78600023FB600023BB60A1
:1003B0000023FB6006E000BFBB680133BB60FB6845
:1003C0000133FB60FA687B689A42F4DB1437BD4660
:1003D0005DF8047B704700BF80B500AFF0F748FDC3
:1003E00080BD00BF80B500AFF3F7B4FC334B9B6D0D
:1003F0000133324A9365324B1B680133304A136034
:100400002F4B1B68092B07D92C4B002283F85E2049
:100410002A4B0022A3F85C202A4B1B680133294A8F
:100420001360284B1B68772B07D903F08DFE02461B
:10043000254B1A60234B00221A60244B9B78002B1B
:1004400002D0F2F7B5FA05E0214A214BDB6943F40B
:100450000023D3611F4B1B68002B0ED01D4B1B6864
:10046000013B1C4A13601B4B1B68002B05D11A4B28
:1004700000221A73184B00225A73174B1B78192B42
:100480001BD0124B9B78002B17D0144B1B68002BF2
:1004900013D0124B1B68013B104A13600F4B1B68B3
:1004A000002B0AD10E4B1B7F002B03D00D482621B9
:1004B000EFF756FE084B01225A7480BD202700102A
:1004C0000C2700105C0200102C2200100407001002
:1004D00000C009208C1E0010A0270010901E0010E4
:1004E000641E0010C424100080B500AF034B9B783D
:1004F000002B01D0F3F7FCF980BD00BF040700100A
:1005000080B582B000AFBB4B5B7F272B02D8B94BC5
:1005100080225A77B74B5B7F802B02D9B54B802264
:100520005A77B54BB3F8B8311BB240F6AB52934291
:1005300004DCB14B41F28832A3F8B821AE4BB3F8DA
:10054000B8311BB242F23412934204DDAA4B41F29D
:100550008832A3F8B821A84BB3F8BA311BB2632B89
:1005600004DCA54B4FF4FA72A3F8BA21A24BB3F8FE
:10057000BA311BB240F2DC52934204DD9E4B4FF481
:10058000FA72A3F8BA219C4BB3F812311BB2632B59
:1005900004DC994B4FF4FA72A3F81221964BB3F88E
:1005A00012311BB240F2DC52934204DD924B4FF405
:1005B000FA72A3F81221904BB3F810311BB240F637
:1005C000C312934204DC8C4B41F28832A3F8102111
:1005D000894BB3F810311BB242F22832934204DD4A
:1005E000854B41F28832A3F81021834B93F8B63142
:1005F000002B03D1804B052283F8B6217E4B93F864
:10060000B631142B03D97C4B052283F8B6217A4BE3
:1006100093F8B7311E2B03D9774B002283F8B7210B
:10062000754BB3F81432132B03D8734B4622A3F83F
:100630001422714BB3F814325A2B03D96E4B462255
:10064000A3F814226C4BD3F81C3218464FF08041AB
:100650002AF03EFC0346002B03D0674B674AC3F8E1
:100660001C22654BD3F81C32184665492AF04EFC13
:100670000346002B03D0604B604AC3F81C225E4B3C
:1006800093F821325BB2642B03DD5B4B0A2283F8C3
:100690002122594B93F821325BB2012B03DC564BDC
:1006A0000A2283F82122544B93F822325BB2642B46
:1006B00003DD514B502283F822224F4B93F8223214
:1006C0005BB2092B03DC4C4B502283F822224A4BAD
:1006D00093F823325BB2142B03DD474B002283F8DF
:1006E0002322454B93F823325BB213F1140F03DA44
:1006F000414B002283F823223F4B93F824325BB214
:10070000142B03DD3C4B002283F824223A4B93F850
:1007100024325BB213F1140F03DA374B002283F853
:100720002422354B93F826325BB2142B03DD324B77
:10073000002283F82622304B93F826325BB213F165
:10074000140F03DA2C4B002283F826222A4B93F84D
:1007500028325BB2142B03DD274B002283F82822BA
:10076000254B93F828325BB213F1140F03DA224BB6
:10077000002283F82822204B93F82A325BB2142BF4
:1007800003DD1D4B002283F82A221B4B93F82A32EB
:100790005BB213F1140F03DA174B002283F82A22FD
:1007A000154B93F83D32042B03D8134B052283F8E5
:1007B0003D22114B93F83D32642B03D90E4B052299
:1007C00083F83D220C4B93F83E32042B03D80A4B9E
:1007D000642283F83E22084B93F83E32642B03D9FF
:1007E000054B642283F83E22034B93F84232002BE0
:1007F00008E000BF641E0010040700100000404124
:100800000000484303D1B74B042283F84222B54B82
:1008100093F84232072B03D9B24B042283F84222C9
:10082000B04B93F83C321E2B03D9AE4B052283F814
:100830003C22AC4B93F83C32002B03D1A94B052250
:1008400083F83C22A74B93F81332012B03D9A54B15
:10085000012283F81322A34BB3F84E321BB21E2B96
:1008600003DDA04B0022A3F84E229E4BB3F84E327C
:100870001BB213F11E0F03DA9A4B0022A3F84E228B
:10088000984B93F81632082B08D0964B93F81632F3
:10089000072B03D0934B082283F81622914BB3F811
:1008A0005032092B05D98F4BB3F85032B3F5167F70
:1008B00003D98C4B7822A3F850228A4BB3F84432E8
:1008C000142B03D9874B0F22A3F84422854BD3F86E
:1008D0005C32184684492AF0FBFA0346002B03D009
:1008E000804B824AC3F85C227E4BD3F85C321846B8
:1008F0007F492AF00BFB0346002B03D0794B7B4A40
:10090000C3F85C22774BD3F86032184679492AF055
:10091000DFFA0346002B03D0724B774AC3F86022FC
:10092000704BD3F86032184670492AF0EFFA03464C
:10093000002B03D06B4B704AC3F86022694BD3F88D
:10094000643218466B492AF0C3FA0346002B03D0E1
:10095000644B684AC3F86422624BD3F86432184689
:1009600062492AF0D3FA0346002B03D05D4B614A5B
:10097000C3F864225B4BD3F8683218465D492AF00D
:10098000A7FA0346002B03D0564B5C4AC3F86822F3
:10099000544BD3F86832184655492AF0B7FA034643
:1009A000002B03D04F4B554AC3F868224D4B9B7820
:1009B000012B02D94B4B01229A704A4B93F8173204
:1009C000092B03D9474B002283F81722454BB3F874
:1009D0001832962B03D9434B1922A3F81822414B06
:1009E000B3F81832072B03D83E4B1922A3F818226C
:1009F0003C4B93F856320F2B03D93A4B052283F820
:100A00005622384BB3F83232782B03D9354B0F22AC
:100A1000A3F83222334BB3F834323C2B03D9314B99
:100A20001422A3F834222F4BB3F83632642B03D9A7
:100A30002C4B1E22A3F836222A4B93F838320F2B68
:100A400003D9284B032283F838222D4800214FF484
:100A50009672002303F010FD224B9B7A032B02D9E0
:100A6000204B00229A721F4B93F86C32002B08D057
:100A70001C4B93F86C32012B03D01A4B002283F8E5
:100A80006C22184B93F86E32022B03D9154B0122BE
:100A900083F86E22134B93F86D32032B03D9114B5D
:100AA000012283F86D22174B1B6818464FF0000196
:100AB0002AF00EFA0346002B05D0124B4FF07E525F
:100AC0001A60F4F765F8074B9B7D012B02D9054BA3
:100AD00001229A75034B1B7E642B15D9014B6422AE
:100AE0001A7611E0040700100000A0400000A041A9
:100AF0000000F04100002041000040410000C841DA
:100B00003E0900101C1E0010B24B1B7E092B02D8A0
:100B1000B04B64221A76AF4BDB7D5A2B02D9AD4B1A
:100B20000A22DA75AB4B5B8AB3F5967F02D9A94BE3
:100B300078225A82A74B5B8A1D2B02D8A54B7822BC
:100B40005A82A44B5A8AA44BA3FB021399080B4662
:100B50009B000B44D31A9BB2002B02D09D4B7822F2
:100B60005A829C4B5B7EF02B02D99A4B1E225A76FE
:100B7000984B5B7E0E2B02D8964B1E225A76954BD5
:100B8000B3F878321BB2B3F5FA7F06DC914BB3F8B9
:100B900078321BB213F5FA7F03DA8E4B0022A3F8EA
:100BA00078228C4BB3F876321BB2B3F5FA7F06DCB1
:100BB000884BB3F876321BB213F5FA7F03DA854B14
:100BC0000022A3F87622834BB3F87A321BB2B3F536
:100BD000FA7F06DC7F4BB3F87A321BB213F5FA7F4B
:100BE00003DA7C4B0022A3F87A227A4BB3F87C32EA
:100BF0001BB2B3F5FA7F06DC764BB3F87C321BB23E
:100C000013F5FA7F03DA734B0022A3F87C22714BB1
:100C1000B3F87E321BB2B3F5FA7F06DC6D4BB3F846
:100C20007E321BB213F5FA7F03DA6A4B0022A3F877
:100C30007E22684B93F80B33012B03D9654B0022BE
:100C400083F80B23634B93F80C33012B03D9614BCF
:100C5000002283F80C235F4B93F80D33012B03D94B
:100C60005C4B002283F80D235A4B93F80E33B42BC0
:100C700003D9584B782283F80E23564B93F80F3341
:100C8000002B03D1534B142283F80F23514B93F8BD
:100C90000F33282B03D94F4B142283F80F234F48CF
:100CA00064214FF47A72C82303F0E6FB4C4840F607
:100CB000B8314FF4FA5240F6B83303F0DDFB49483F
:100CC00000210122002303F0FDFB474800214FF4DF
:100CD000FA62002303F0D0FB4448322143F6982205
:100CE000962303F0C9FB424800214FF47A721E2379
:100CF00003F0C2FB3F484049404A4FF0000303F075
:100D000007FC3F4807F0B0FE0346002B04D13C48E7
:100D10003C49122228F0A3FF3B4807F0A5FE0346FA
:100D2000002B04D138483949122228F098FF38485E
:100D300007F09AFE0346002B04D1354835491222AC
:100D400028F08DFF344807F08FFE0346002B04D1B6
:100D500031483249122228F082FF314801F058F917
:100D60000346002B10D02E4828F026FE78607B68C2
:100D7000002B03DD7B68B3F5803F0ADB2848294957
:100D8000032228F06CFF04E025482649032228F0BE
:100D900066FF104B9B78002B0FD1234B1B78182B31
:100DA00015D022480021EFF7DBF921480021EFF7A9
:100DB000D7F91D4B00221A7009E01E4B5B7F1B48C0
:100DC0001946EFF7CDF91A48FF21EFF7C9F90837AF
:100DD000BD4680BD04070010CDCCCCCC100800105F
:100DE0000E0800100C08001028070010560900100B
:100DF00058090010541E001000606AC600606A4660
:100E0000A2090010ACA60400FA090010BCA6040058
:100E1000BE090010C8A60400E6090010D8A6040008
:100E2000B6090010E8A60400A0270010C424100092
:100E300090241000641E001080B400AF0F4B0022FD
:100E40001A710E4B00225A710C4B0022DA710B4BB7
:100E500000221A70094B00225A70084B00229A7027
:100E6000064B0022DA70054B00229A71044B0022D7
:100E70005A60BD465DF8047B704700BF300A001021
:100E80004022001080B582B000AF0023FB71002328
:100E9000FB717AE0FB79854A1344002283F8342001
:100EA000FB79824A1344002283F83B20FB797F4A76
:100EB0001344002283F84220FB797C4A1344002229
:100EC00083F84920FB79794A1344002283F8BA2039
:100ED000FB79764A1344002283F8C120FB79734AD8
:100EE0001344002283F8C820FB79704A134400227F
:100EF00083F8CF20FB796D4A1344002283F8182130
:100F0000FB796A4A1344002283F81F21FB79674A60
:100F10001344002283F82621FB79644A13440022FB
:100F200083F82D21FB79614A1344002283F8642160
:100F3000FB795E4A1344002283F86B21FB795B4AFC
:100F40001344002283F87221FB79584A134400228B
:100F500083F87921FB79554A1344012283F8BE2195
:100F6000FB79524A1344002283F8C521FB794F4A8A
:100F70001344002283F8CC21FB794C4A134400220D
:100F800083F8D321FB790133FB71FB79062B81D9DF
:100F90000023FB7182E0FB791846002145220023E3
:100FA00026F05AFFFB79184601214522002326F03E
:100FB00053FFFB79184602214522002326F04CFFFF
:100FC000FB79184603214522002326F045FFFB79D3
:100FD000184600214522012326F03EFFFB791846E2
:100FE00001214522012326F037FFFB791846022113
:100FF0004522012326F030FFFB79184603214522C4
:10100000012326F029FFFB7918460021452226F00E
:1010100021FEFB7918460121452226F01BFEFB79B3
:1010200018460221452226F015FEFB7918460321B9
:10103000452226F00FFEFB7918460021452226F0B6
:1010400087FEFB7918460121452226F081FEFB79B7
:1010500018460221452226F07BFEFB791846032123
:10106000452226F075FEFB79184600214B2227F019
:10107000C9FEFB7918460121452227F0C3FEFB7902
:1010800018460221452227F0BDFEFB7918460321B0
:10109000452227F0B7FEFB790133FB71FB792F2B3B
:1010A0007FF679AF0023FB7102E100BF0407001057
:1010B000FB79C84A862101FB03F313442033012244
:1010C0005A72FB79C34A862101FB03F3134432228F
:1010D0001A81FB79BF4A862101FB03F313440833CD
:1010E00078225A81FB79BB4A862101FB03F3134422
:1010F00010330A225A71FB79B64A862101FB03F3A9
:101100001344103300221A71FB79B24A862101FB85
:1011100003F31344103301229A71FB79AD4A8621FF
:1011200001FB03F31344203300229A72FB79A94A8E
:10113000862101FB03F313440022DA72FB79A54AEE
:10114000862101FB03F3134400229A72FB79A14A22
:10115000862101FB03F3134440F26C72DA80FB79C1
:101160009C4A862101FB03F3134440F634029A8023
:10117000FB79984A862101FB03F3134420330022B4
:101180001A72FB79934A862101FB03F3134420333F
:101190004FF47A62DA80FB798E4A862101FB03F3F1
:1011A000134408334FF47A629A80FB79894A862186
:1011B00001FB03F31344103364221A72FB79854A4E
:1011C000862101FB03F3134410330A22DA71FB7901
:1011D000804A862101FB03F31344103314225A7210
:1011E000FB797C4A862101FB03F313442033002260
:1011F0009A80FB79774A862101FB03F3134410336D
:1012000004229A72FB79734A862101FB03F313448B
:1012100018333222DA80FB796E4A862101FB03F310
:101220001344183396229A80FB796A4A862101FB7F
:1012300003F31344183330229A72FB79654A8621EE
:1012400001FB03F31344183314221A81FB79614A1A
:10125000862101FB03F31344783340F6AC521A8124
:10126000FB795C4A862101FB03F31344083340F603
:10127000C412DA80FB79574A862101FB03F3134439
:10128000083341F288321A81FB79524A862101FBE8
:1012900003F313440022DA72FB794E4A862101FBE4
:1012A00003F31344783300229A72FB790133FB7104
:1012B000FB79012B7FF6FCAE464B0022A3F8782287
:1012C000444B0022A3F87622424B002283F8B0213F
:1012D000404B012283F8B4213E4B4FF47A62A3F8CD
:1012E000B2213C4B01229A703A4B41F28832A3F86A
:1012F000B821384BB3F8B821374B1A80354B4FF42F
:10130000FA72A3F8BA21334B41F65832A3F8BC2144
:10131000304B012283F80D222E4B0022A3F80A2223
:101320002C4B42F22832A3F80E222A4B002283F8DB
:101330000C22284B012283F81322264B4322A3F8C8
:101340001422244B012283F81721224B41F29412DC
:10135000A3F810211F4B4FF4FA72A3F812211D4B72
:10136000002283F816211B4B4FF47A72A3F8142144
:10137000184B052283F8B621164B002283F8B721BB
:10138000144B002283F8B021124B082283F8162256
:10139000104B002283F817220E4B1422A3F81822B8
:1013A0000C4B0E4AC3F81C220A4B052283F83C2240
:1013B000084B0A2283F82022064B0A2283F83D229A
:1013C000044B642283F83E22024B042283F842221B
:1013D00006E000BF04070010202700100000704145
:1013E000924B0F22A3F84022904B0F22A3F83222F7
:1013F0008E4B1E22A3F836228C4B052283F838220E
:101400008A4B1422A3F83422884B1422A3F83A22E0
:10141000864B0822A3F82C22844B1922A3F83022F1
:10142000824B002283F82322804B002283F824225F
:101430007E4B002283F825227C4B002283F8262253
:101440007A4B002283F82722784B002283F8282247
:10145000764B002283F82922744B002283F82A223B
:10146000724B0A2283F82122704B1E2283F822221B
:101470006E4B4622A3F82E226C4B0F22A3F8442277
:101480006A4B7822A3F85022694B1E221A77684BC8
:1014900080225A77654B674AC3F85C22634B664AE1
:1014A000C3F86022614B654AC3F864225F4B614A0E
:1014B000C3F868225D4B012283F86E225B4B022247
:1014C00083F86D22594B4B2283F81022574B202270
:1014D00083F81122554B002283F81222534B40F619
:1014E000B832A3F88420514B002283F882204F4B5E
:1014F0000022A3F888204D4B40F6B832A3F80A2109
:101500004A4B002283F80821484BC822A3F80C213B
:10151000464B46F2A812A3F84C22444B012283F812
:101520004A22424B0022A3F84E22404B002283F86D
:1015300074223E4B002283F80B233C4B002283F89D
:101540000C233A4B002283F80D23384B0022A3F8DA
:101550007C22364B0022A3F87E22344B0022A3F8D3
:101560008022324B0022A3F87822304B0022A3F8CD
:1015700076222E4B0022A3F87A222C4B0022A3F8CD
:1015800084222A4B0022A3F88222284B782283F857
:101590000E23264B142283F80F23244B9622A3F804
:1015A0005222224B1E22A3F85422204BB3F852326F
:1015B0001BB2184629F046FC0246214B9A63F3F70A
:1015C000E7FA1A4B012283F80A23184B012283F809
:1015D000B9221C481C490A2228F041FB1B481C491F
:1015E0000B2228F03CFB1B481B49122228F037FB3A
:1015F0001A481B49032228F032FB1A481A490F22C5
:1016000028F02DFB19481A49122228F028FB194806
:101610001949122228F023FB054B5B7F1748194616
:10162000EEF79EFD0837BD4680BD00BF04070010E1
:10163000641E00100000A041000040410000204155
:101640001C1E00108A090010ECA604009609001068
:10165000F8A60400BE090010C8A60400B6090010D0
:10166000E8A60400E6090010D8A60400A2090010AC
:10167000ACA60400FA090010BCA60400C4241000A3
:1016800080B483B000AF0023FB800023FB8031E0F7
:10169000FB88FA880132334931F81210314A22F8B6
:1016A0001310FB88FA8801322E4902F5347231F8A2
:1016B00012102C4A03F5347322F81310FB88FA88B1
:1016C000013228490A4492F8401B264A13440A462C
:1016D00083F8402BFB88FA880132224902F5E16247
:1016E00031F812101F4A03F5E16322F81310FB884A
:1016F0000133FB80FB8840F2CE229342C8D91A4BBB
:101700005B891BB2194A82FB03129210DB17D31AB2
:101710009AB2144BA3F89E25134B5B68134A82FBC5
:1017200003129210DB17D31A9AB20E4BA3F83E2B7A
:101730000F4B1B89DAB20B4B83F80F2E0A4B9B8A97
:101740001BB20A4A82FB03129210DB17D31A9AB219
:10175000044B03F59D530E331A800C37BD465DF8DC
:10176000047B7047480A0010C42100106766666653
:101770002027001080B400AFBD465DF8047B7047A1
:1017800080B5ADF57C7D00AF0023A7F8EC331B4B93
:101790001B68002B2DD00023A7F8EE33184B062230
:1017A0005A600023A7F8EE3310E0B7F9EE33B7F92B
:1017B000EE2314498A5CD2B2D1B23A1DD154B7F8A3
:1017C000EE339BB201339BB2A7F8EE33B7F9EE23A9
:1017D0000A4B1B689A42E8D3084B00221A60084B58
:1017E00007225A60B7F9EE333A1D10461946FBF747
:1017F000B7FB07F57C77BD4680BD00BFEC0200104B
:1018000000000140A05A001080B483B000AF002354
:101810007B6002E07B6801337B60094B1B7DDBB2A0
:1018200003F00103002BF5D1064A064B9B6943F4F4
:10183000003393610C37BD465DF8047B704700BFF1
:101840000000014000C0092080B582B000AF002335
:101850007B6002E07B6801337B600A4B1B7DDBB25F
:1018600003F02003002BF5D04FF47A70FEF798FDBB
:10187000054A054BDB6943F40033D3610837BD46A5
:1018800080BD00BF0000014000C0092080B588B0C5
:1018900000AFBC4B1B68002B40F0D58106F0E2FF87
:1018A0000346002B1CD0F6F7EDFCF6F7CFFCB6484C
:1018B000F6F768FDB5486321FBF708FAFFF7A4FFC8
:1018C0004FF47A70FEF76CFDB14828F079F90346C1
:1018D0000120AF491A4627F06DFEFFF7B5FFB2E1D0
:1018E000AC4B1B780133DAB2AA4B1A70A94B1B78A8
:1018F000062B02D9A74B00221A70A64B1B78013B7E
:10190000052B00F2A08101A252F823F02519010055
:101910005F190100C91B0100471C0100471C0100A1
:101920000D1C0100F6F7AEFCF6F790FC9A48F6F7AE
:1019300029FD96486321FBF7C9F9FFF765FF4FF4CE
:101940007A70FEF72DFD924828F03AF903460120FF
:101950008F491A4627F02EFEFFF776FF73E18F4B73
:101960001B78032B17D1F6F78DFCF6F76FFC8C482C
:10197000F6F708FD85480321FBF7A8F9FFF744FFB8
:10198000834828F01DF90346012081491A4627F0B3
:1019900011FEFFF759FF814B1B78052B17D1F6F786
:1019A00071FCF6F753FC7F48F6F7ECFC774803210F
:1019B000FBF78CF9FFF728FF754828F001F903467B
:1019C000012073491A4627F0F5FDFFF73DFF734BE1
:1019D0001B78012B17D1F6F755FCF6F737FC724848
:1019E000F6F7D0FC69480321FBF770F9FFF70CFF0D
:1019F000674828F0E5F80346012065491A4627F0B4
:101A0000D9FDFFF721FF654B1B78082B17D1F6F79F
:101A100039FCF6F71BFC6548F6F7B4FC5B4803217C
:101A2000FBF754F9FFF7F0FE594828F0C9F80346D0
:101A3000012057491A4627F0BDFDFFF705FF574B18
:101A40001B780A2B17D1F6F71DFCF6F7FFFB584859
:101A5000F6F798FC4D480321FBF738F9FFF7D4FE61
:101A60004B4828F0ADF80346012049491A4627F0B3
:101A7000A1FDFFF7E9FE494B1B780E2B17D1F6F7B6
:101A800001FCF6F7E3FB4B48F6F77CFC3F480321EB
:101A9000FBF71CF9FFF7B8FE3D4828F091F8034624
:101AA00001203B491A4627F085FDFFF7CDFE3B4B51
:101AB0001B78112B17D1F6F7E5FBF6F7C7FB3E486D
:101AC000F6F760FC31480321FBF700F9FFF79CFEB5
:101AD0002F4828F075F8034601202D491A4627F0B3
:101AE00069FDFFF7B1FE2D4B1B78122B17D1F6F7CE
:101AF000C9FBF6F7ABFB3148F6F744FC234803215A
:101B0000FBF7E4F8FFF780FE214828F059F8034678
:101B100001201F491A4627F04DFDFFF795FE1F4B88
:101B20001B78502B08D1FFF76FFE012024492D228E
:101B300027F040FDFFF788FE184B1B78512B08D18A
:101B4000FFF762FE01201F492A2227F033FDFFF72D
:101B50007BFE124B5A78114B1A70104B9A780F4B30
:101B60005A700E4BDA780D4B9A700C4B1A790B4B5E
:101B7000DA700A4B5A79094B1A71084B00225A71D4
:101B800061E000BFEC02001004A704000CA70400F1
:101B9000E84E00106802001014A70400F8060010B8
:101BA00020A7040024A7040028A704002CA70400F1
:101BB00038A7040040A7040048A7040054A7040065
:101BC0005CA704008CA7040002F0BEFA02461F4B7B
:101BD0001A60F6F757FBF6F739FB1D48F6F7D2FB0C
:101BE0001C480321FBF772F8FFF70EFE4FF47A70E2
:101BF000FEF7D6FB184827F0E3FF034601201649FD
:101C00001A4627F0D7FCFFF71FFE1CE0F6F73AFB59
